:0400000057EF00F0C6
:100008002B002B002B002B002B002B002B002B0090
:100018004E632B002B002B002B002B002B002B00FA
:100028002B002B002B002B002B002B002B002B0070
:100038002B002B002B00F4672B002B002B002B0030
:100048002B002B00A66D2B002B002B002B002B0068
:100058002B002B002B002B002B002B002B002B0040
:100068002B002B002B002B002B002B002B002B0030
:100078002B002B002B002B002B002B002B002B0020
:100088002B002B002B002B002B002B002B002B0010
:100098002B002B002B002B002B002B002B002B0000
:0A00A8002B002B00FF00DFEFCCF06F
:10F574000000000000001B1B0000181818181B1BBB
:10F584000000030303031B1B00001B1B1B1B1B1B93
:10F5940000040E1F0404040400040404041F0E04E5
:10F5A400001112140B110203000E0A0E00000000D9
:10F5B40000EAB60194B301FCB501E28501D69B01D2
:10F5C40082A101869E01DCB6018CB70188B7016C6B
:10F5D400B40134B7013CB701CEB6012CB701BEB6B5
:10F5E40001ACA5017AA201AEB6010024744C00243A
:10F5F400744C0000FA460024F4480000FA460080E7
:10F60400C094D4204F544845525320204C43445F67
:10F6140034626974735F4932435F323032342D305F
:10F62400312E682C2055415254315F46756E6374F7
:10F63400696F6E735F3436303830306264732E68AD
:10F644000D0A20416666696368655F4E454D415FFA
:10F654004C43445F323032342E696E63202C44694B
:10F66400616C6F6775655F4E454D415F3230323472
:10F674002E696E630D0A0045434F2E2E2E2E004236
:10F68400415252455F470042415252455F44004255
:10F6940041525245474400464C45434820480046A1
:10F6A4004C4543485F4200312F324865757200442F
:10F6B40045475245432000204469726563746F7264
:10F6C40079203A433A5C4D504C4142585F50726F36
:10F6D4006A656374735C5F31384632374B34325F2A
:10F6E400546573745F4E454D4132335F323032346A
:10F6F4002E580D0A002031384632374B343220550B
:10F704004152543120343630383030206264732C06
:10F71400204144433132622C204E434F312C436C00
:10F724006B6F75740D0A0020436C6F636B6F757497
:10F73400205241363D464F53432F343D31364D68B8
:10F744007A20776974682020534C52434F4E412EDF
:10F7540042363D30202100205445535420204E434E
:10F764004F3120656E206D6F64652046726571753A
:10F77400656E6365203A204F7570757420737572D9
:10F78400205243350D0A0020536F75726365203A89
:10F79400206D61696E2E630D0A2056657273696F60
:10F7A4006E203A323032342D3031330D0A0020507D
:10F7B400726F6A6574203A5F31384632374B34329F
:10F7C4005F546573745F4E454D4132335F3230325E
:10F7D400340D0A002054657374204241534520506F
:10F7E400494331384632374B343220200D0A002049
:10F7F400204D46494E544F53432028353030206B1A
:10F80400487A2900204D46494E544F53432F342003
:10F81400283332206B487A2900204D504C414258FD
:10F824002056362E30202B205843380D0A00202035
:10F8340020202020202020202020202020202020C4
:10F8440020200020464F53433A36342E30204D4872
:10F854007A0D0A00204846494E544F534320002055
:10F864004C46494E544F53430020464F53430020C7
:10F87400002043686F697820766961204D6F646564
:10F884005F4364653D30202D3E20766961204B65E1
:10F89400796F617264206F75204D6F64655F436496
:10F8A400653D312028706172206465666175742934
:10F8B4006176656320506F74617220737572205293
:10F8C40041310D0A0056616C6575722064652046ED
:10F8D40072657175656E636520617520636C617610
:10F8E40069657220463D7878787820206176656372
:10F8F400207878787820646520303030362000789D
:10F904004530203939393920487A0D0A000D0A204A
:10F914004D6F646520636F6D6D616E6465206D6FFE
:10F92400746575723A204D6F643D30202D3E204B36
:10F934006579626F617264202C204D6F643D3120C3
:10F944002D3E2020506F74617220737572205241D5
:10F95400310D0A0020506F74617220E020646F69D9
:10F964007465202876657273206C65206D617869F2
:10F97400292053656E7320486F7261697265206532
:10F984007420467265712070726F706F7274696F43
:10F994006E656C6C650D0A0020506F74617220E016
:10F9A400206761756368652876657273206C6520CD
:10F9B4006D696E69292053656E7320547269676F8F
:10F9C4002020657420467265712070726F706F72AA
:10F9D40074696F6E656C6C650D0A00204672657102
:10F9E4003D25352E316620202C436F756E74203DE5
:10F9F400253564202C2031547220656E2025356411
:10FA0400206D5320736F69742025332E3266205481
:10FA1400722F7365630D0A002053656E732064654D
:10FA240020726F746174696F6E203C483E20706F61
:10FA3400757220486F726169726520203C543E20C3
:10FA4400706F757220547269676F200D0A000D0A79
:10FA54002053656E7320486F726169726520204E71
:10FA640065772046726571203D2535642020204E3F
:10FA7400657720496E6372656D656E743D25756C9E
:10FA84000D0A002044656C6179203530306D5320B7
:10FA94006368726F6E6F207669612054696D657258
:10FAA4002032203D3E20437074323D253564206D64
:10FAB40053200D0A00205465737420617665632019
:10FAC400636F6D6D616E6465204672657120766941
:10FAD40061204B6579626F617264206F7520506F8D
:10FAE4007461720D0A00204672657175656E6365F6
:10FAF40020463D7878787820617665632078787838
:10FB040078203D20303030362020007845302036B3
:10FB14003030300D0A002052415A20706F75722027
:10FB240052415A20647520636F6D707274657572EA
:10FB340020642065546F757220436F756E745F5234
:10FB440042300D0A00200D0A53657175656E6365B8
:10FB5400206427496E6974204C4344203478323041
:10FB64002076696120493243312050434638353785
:10FB7400340D0A00203C4D3E20706F7572204D619B
:10FB84007263686520203C413E20706F757220418D
:10FB94007272657420202820456E61626C65290D9F
:10FBA4000A00204020646563696D616C202325345C
:10FBB400752020736F6974204044657669636520FD
:10FBC4003762697473203D20305825303258200044
:10FBD40020436F6D70696C65642025732061742007
:10FBE400257320555443202076657273696F6E2007
:10FBF400584338203A2564200D0A00204D6F643D97
:10FC04007820206176656320783D303D3E204B6549
:10FC140079626F6172642C2020783D3120506F74BA
:10FC240061720D0A000D0A204D6F646520636F6DCB
:10FC34006D616E6465203D204B6579626F6172640D
:10FC4400207465726D696E616C0D0A000D0A204E98
:10FC540065772046726571203D2535642020204E4D
:10FC6400657720496E6372656D656E743D25756CAC
:10FC74000D0A0020546573742070726573656E6399
:10FC840065206465766963657320737572204275B7
:10FC94007320493243310D0A000D0A204572726502
:10FCA4007572207361697369652076616C6575721C
:10FCB40020646520426176617264200D0A00205040
:10FCC4006F746172206175206D696C696575203D82
:10FCD400204172726574206D6F746575720D0A002F
:10FCE400204572726F722073616973696520463DA5
:10FCF40030313030200078453020363030300D0A35
:10FD040000204241563D3034207072696E74206187
:10FD14007420696E74657272757074205242300D6D
:10FD24000A00204241563D3032207072696E7420C0
:10FD34006461746173206173796E6368726F6E6558
:10FD44000D0A002061647265737365204C43443D61
:10FD540020256420736F6974203058253032582070
:10FD64000D0A002072617070656C203A206169642C
:10FD7400652076696120636465202048656C700D98
:10FD84000A0020436E74203D253564202C20315414
:10FD94007220656E20253564206D530D0A0045657B
:10FDA40070726F6D2032344C437878782032353657
:10FDB4006B206F75203531324B00205465737420ED
:10FDC4006D6573757265202041444331202852418A
:10FDD40031290D0A00414443313D2025356420205A
:10FDE400736F6974202025332E326620560D0A0065
:10FDF4000D0A2048656C7020436F6D6D616E6465FB
:10FE040073203A2048656C700D0A00202020467249
:10FE14006571204F75747075743D202025362E3120
:10FE240066200D0A00205043463837353420666F6B
:10FE340072204C4344203278313663617273000D72
:10FE44000A20526573657420766F6C6F6E746169F5
:10FE54007265200D0A002041726D6520696E74651B
:10FE64007272757074696F6E73200D0A00204241BE
:10FE7400563D303020706173206465207072696E65
:10FE8400740D0A0020496E69745F493243282920A1
:10FE94003130304B687A3B0D0A00436C636B20466B
:10FEA4005245512E202520352E306620487A2000D8
:10FEB4000D0A2050726573656E746174696F6E20EB
:10FEC4003A200D0A00204E434F315F496E69745F3A
:10FED4004C6F6E6775650D0A0050434638353734EC
:10FEE4004120386269747320492F4F00204E434FDC
:10FEF40031434C4B2063686F6978203D2000436494
:10FF0400652025732054723A20253564206D5300F2
:10FF14004C434420323131392032783136636172B6
:10FF2400730053656E733A202573204D6F643D252D
:10FF3400632000504346383537342038626974737F
:10FF440020494F004E62542025356420446973745F
:10FF54002025356400454550524F4D2035313262DD
:10FF640079746573002054455354204E434F312017
:10FF74000D0A004F4C45442053534431333036006E
:10FF84006E6F6E20726563656E731B39004F637408
:10FF9400203133203230323400525443204453331E
:10FFA4003233310020202020736F697420002048F0
:10FFB400656C70200D0A0031393A32383A35340014
:10FFC400545249474F202E00484F52414952450050
:10FFD40052656375203A00494E46004E414E006911
:10FFE4006E66006E616E006C6C73004F46460020B6
:0BFFF4004F4E00202E31006C66000014
:020000040001F9
:10000000000E0001756F000E746F30C086F031C0B5
:1000100087F032C088F033C089F089BF14EF80F0D8
:1000200012EF80F02AEF80F0000E756F010E746FF2
:1000300086C001F087C002F088C003F089C004F0D8
:10004000B5ECD8F001C086F002C087F003C088F09C
:1000500004C089F0000E00018D6F000E8C6FEEC1A0
:1000600078F0EFC179F074517511D8A43AEF80F0AF
:100070003CEF80F044EF80F00101F2A542EF80F008
:1000800044EF80F05FEF80F0000174517511D8A447
:100090004CEF80F04EEF80F054EF80F0000E616F77
:1000A0002B0E606F58EF80F0000E616F2D0E606FA9
:1000B00060C082F28C4B8D2B7807D8A0790786C060
:1000C00001F087C002F088C003F089C004F01CEC86
:1000D000C6F001040210D8A470EF80F072EF80F037
:1000E000BDEF80F0BF0E356EFF0E366E3450376EAA
:1000F000386A3550372636503822385007E11A0E04
:10010000375CD8B086EF80F088EF80F097EF80F012
:10011000820E00018C25016E020E8D21026EDB0E17
:10012000036EFF0E046EB1ECD3F0A4EF80F0820EEC
:1001300000018C25016E020E8D21026EE30E036E0E
:10014000FF0E046EB1ECD3F00001FD0E7827FF0E18
:1001500079232EC011F02FC012F0820E136E020E02
:10016000146E78C015F079C016F0B9ECCBF011C060
:100170002EF012C02FF013EF86F086C001F087C07A
:1001800002F088C003F089C004F01CECC6F00150F6
:100190000210D8A4CEEF80F0D0EF80F004EF81F011
:1001A000BF0E356EFF0E366E3450376E386A3550DE
:1001B000372636503822385007E11A0E375CD8B04F
:1001C000E4EF80F0E6EF80F0F5EF80F0820E0001C2
:1001D0008C25016E020E8D21026EDF0E036EFF0E66
:1001E000046EB1ECD3F0A4EF80F0820E00018C25F8
:1001F000016E020E8D21026EE70E036EFF0E046E7D
:10020000B1ECD3F0A4EF80F0000E00018E6F000E71
:100210008F6F800E906F3F0E916F000E8B6F000EF0
:100220008A6F86C001F087C002F088C003F089C0E1
:1002300004F0000E056E000E066E000E076E000E36
:10024000086EEEECCEF0D8B028EF81F02AEF81F006
:10025000ADEF81F049EF81F08EC001F08FC002F068
:1002600090C003F091C004F0000E056E000E066E03
:10027000200E076E410E086ED9ECA7F001C08EF07B
:1002800002C08FF003C090F004C091F000018A4BCF
:100290008B2B86C01AF087C01BF088C01CF089C069
:1002A0001DF0000E056E000E066E200E076E410E4C
:1002B000086E8EC001F08FC002F090C003F091C0B4
:1002C00004F0D9ECA7F001C01EF002C01FF003C07B
:1002D00020F004C021F01AECC5F0D8B072EF81F024
:1002E00074EF81F02CEF81F094EF81F08EC001F07B
:1002F0008FC002F090C003F091C004F0000E056EB4
:10030000000E066E200E076E410E086ECEECABF0AE
:1003100001C08EF002C08FF003C090F004C091F0D5
:1003200000018A07D8A08B0786C01AF087C01BF08F
:1003300088C01CF089C01DF08EC01EF08FC01FF059
:1003400090C020F091C021F01AECC5F0D8A0ABEF1E
:1003500081F0ADEF81F076EF81F034C003F0046AF4
:1003600035ECD7F0035000017B6F7BC07AF0670E4D
:100370007B19D8A4BEEF81F0C0EF81F0E8EF81F0E7
:100380000101F051F111D8A4C8EF81F0CAEF81F05A
:10039000CEEF81F0000EF16F010EF06FF1BFDBEFD9
:1003A00081F0F15106E1F005D8B0D9EF81F0DBEF33
:1003B00081F0E2EF81F0000E0001776F060E766F9C
:1003C000F2EF81F0F0C176F0F1C177F0F2EF81F059
:1003D0000101F1BFEEEF81F0F0EF81F0DBEF81F092
:1003E000E2EF81F0670E00017B19D8A4FAEF81F0EB
:1003F000FCEF81F02BEF82F08BAF0AEF82F0FC0E66
:100400008A5DFF0E8B59D8A008EF82F00AEF82F0C8
:1004100029EF82F0FF0E356EFF0E366E76C037F094
:1004200077C038F035503726365038228A51375C3D
:100430003850800A396E8B51800A3958D8A023EF82
:1004400082F025EF82F029EF82F0660E7A6F2BEFB3
:1004500082F0650E7A6F76C06CF077C06DF0670E33
:100460007B19D8A436EF82F038EF82F048EF82F0A3
:10047000660E7A19D8A43FEF82F041EF82F04AEF7E
:1004800082F08BBF48EF82F046EF82F04AEF82F0B5
:100490006C4B6D2B660E7A19D8A451EF82F053EF96
:1004A00082F073EF82F08BBF5AEF82F058EF82F048
:1004B00066EF82F0000E8E6F000E8F6F800E906FD1
:1004C0003F0E916F000E8B6F000E8A6F670E7B19C7
:1004D000D8B46DEF82F06FEF82F073EF82F08A5143
:1004E0006C278B516D23000E856F000E846F86C0C4
:1004F0007CF087C07DF088C07EF089C07FF08EC020
:100500006EF08FC06FF090C070F091C071F004EF8A
:1005100083F07CC001F07DC002F07EC003F07FC09C
:1005200004F08EC005F08FC006F090C007F091C0B7
:1005300008F0CEECABF001C01AF002C01BF003C013
:100540001CF004C01DF06EECB5F01AC080F01BC0AA
:1005500081F01CC082F01DC083F080C001F081C01A
:1005600002F082C003F083C004F097ECC4F001C035
:1005700072F002C073F07CC01AF07DC01BF07EC028
:100580001CF07FC01DF08EC005F08FC006F090C03B
:1005900007F091C008F080C001F081C002F082C075
:1005A00003F083C004F0D9ECA7F001C01EF002C034
:1005B0001FF003C020F004C021F058ECD7F01AC09F
:1005C0007CF01BC07DF01CC07EF01DC07FF08EC093
:1005D00001F08FC002F090C003F091C004F0000E53
:1005E000056E000E066E200E076E410E086ECEECF4
:1005F000ABF001C08EF002C08FF003C090F004C0D9
:1006000091F00001844B852B6C51845D8551800AEB
:10061000356E6D51800A3558D8A011EF83F013EF75
:1006200083F089EF82F08EC001F08FC002F090C09D
:1006300003F091C004F0000E056E000E066EA00ED1
:10064000076E400E086ED9ECA7F001C080F002C022
:1006500081F003C082F004C083F07CC01AF07DC03A
:100660001BF07EC01CF07FC01DF080C01EF081C05A
:100670001FF082C020F083C021F01AECC5F0D8B082
:1006800044EF83F046EF83F051EF83F0000E00015A
:10069000806F000E816F000E826F000E836F7AEF05
:1006A00083F07CC001F07DC002F07EC003F07FC00B
:1006B00004F080C005F081C006F082C007F083C05E
:1006C00008F0EEECCEF0D8A068EF83F06AEF83F08C
:1006D0007AEF83F0000172B170EF83F072EF83F074
:1006E0007AEF83F0000E806F000E816F000E826F34
:1006F000000E836F86C001F087C002F088C003F04F
:1007000089C004F080C005F081C006F082C007F007
:1007100083C008F051ECA3F001C07CF002C07DF072
:1007200003C07EF004C07FF07CC01AF07DC01BF0D7
:100730007EC01CF07FC01DF0000E056E000E066E20
:10074000200E076E410E086E6EC001F06FC002F001
:1007500070C003F071C004F0D9ECA7F001C01EF026
:1007600002C01FF003C020F004C021F01AECC5F055
:10077000D8A0BDEF83F0BFEF83F0E8EF83F0000176
:100780008A4B8B2B6EC001F06FC002F070C003F07B
:1007900071C004F0000E056E000E066E200E076E8E
:1007A000410E086ED9ECA7F001C06EF002C06FF0E8
:1007B00003C070F004C071F0660E00017A19D8A46D
:1007C000E4EF83F0E6EF83F0E8EF83F06C4B6D2B02
:1007D0006EC08EF06FC08FF070C090F071C091F05D
:1007E000650E00017A19D8B4F8EF83F0FAEF83F0C0
:1007F00000EF84F08AC06AF08BC06BF004EF84F0E5
:10080000000E6B6F000E6A6F000E696F000E686F4E
:10081000000E676F000E666F000E856F000E846F0E
:1008200001EF85F07CC001F07DC002F07EC003F0D6
:100830007FC004F08EC005F08FC006F090C007F0B6
:1008400091C008F0CEECABF001C01AF002C01BF072
:1008500003C01CF004C01DF06EECB5F01AC080F0AF
:100860001BC081F01CC082F01DC083F080C001F06D
:1008700081C002F082C003F083C004F097ECC4F0A2
:1008800001C072F002C073F00101F2B94AEF84F0C6
:100890004CEF84F06AEF84F0000172517311D8A418
:1008A00054EF84F056EF84F06AEF84F0670E7B1902
:1008B000D8A45DEF84F05FEF84F06AEF84F06BBF43
:1008C00066EF84F064EF84F06AEF84F0664B672B88
:1008D000B5EF84F0000168516911D8A472EF84F07B
:1008E00074EF84F09EEF84F06BBF7BEF84F079EFC0
:1008F00084F09EEF84F0820E8C25D96E020E8D213D
:10090000DA6E2E0EDF6E8C4B8D2B7807D8A0790710
:10091000000E696F010E686F9EEF84F0820E8C25C9
:10092000D96E020E8D21DA6E300EDF6E8C4B8D2B60
:100930007807D8A079076607D8A0670766516711BE
:10094000D8A4A5EF84F0A7EF84F08EEF84F0820E98
:100950008C25D96E020E8D21DA6E7251300FDF6E4A
:100960008C4B8D2B7807D8A079077CC01AF07DC0FE
:100970001BF07EC01CF07FC01DF08EC005F08FC044
:1009800006F090C007F091C008F080C001F081C06F
:1009900002F082C003F083C004F0D9ECA7F001C0DC
:1009A0001EF002C01FF003C020F004C021F058EC7C
:1009B000D7F01AC07CF01BC07DF01CC07EF01DC0BB
:1009C0007FF08EC001F08FC002F090C003F091C0A4
:1009D00004F0000E056E000E066E200E076E410E2E
:1009E000086ECEECABF001C08EF002C08FF003C0F9
:1009F00090F004C091F000016A07D8A06B07844B07
:100A0000852B6C51845D8551800A356E6D51800A4D
:100A10003558D8B00EEF85F010EF85F01EEF85F059
:100A20008DBF1CEF85F08D5109E14B0E8C5DD8A078
:100A30001CEF85F01EEF85F012EF84F0685169110C
:100A4000D8A425EF85F027EF85F03AEF85F0010176
:100A5000F2A92DEF85F02FEF85F03AEF85F0820EA9
:100A600000018C25D96E020E8D21DA6E2E0EDF6EFE
:100A70008C4B8D2B820E00018C25D96E020E8D21A0
:100A8000DA6E000EDF6E650E7A19D8A44AEF85F093
:100A90004CEF85F0A9EF80F0000E856F4F0E846F4C
:100AA000820E8425D96E020E8521DA6E000EDF6E6D
:100AB000000E756F000E746F8BBF63EF85F061EFF2
:100AC00085F06BEF85F0000E756F010E746F8A6D07
:100AD0008B1FD8B08B2B000E776F020E766F9CEFBA
:100AE00085F08407D8A08507820E8425D96E020E72
:100AF0008521DA6E8AC001F08BC002F0000E046E10
:100B00000A0E036E93ECCDF00150300FDF6E8AC0F9
:100B100001F08BC002F0000E046E0A0E036E1CEC96
:100B2000CCF001C08AF002C08BF000017607D8A09B
:100B300077077807D8A079078A518B11D8A4A3EF3B
:100B400085F0A5EF85F071EF85F077BFB2EF85F006
:100B5000775106E17605D8B0B0EF85F0B2EF85F0B9
:100B600071EF85F08407D8A0850774517511D8A45A
:100B7000BCEF85F0BEEF85F0C4EF85F0000E636F2B
:100B80002B0E626FC8EF85F0000E636F2D0E626F43
:100B9000820E8425D96E020E8521DA6E60008BF1FB
:100BA000DFFF7807D8A079078407D8A08507BF0E94
:100BB000356EFF0E366E3450376E386A3550372634
:100BC00036503822385009E11A0E375CD8A0EBEFC6
:100BD00085F0EDEF85F0F3EF85F0000E656F650EA3
:100BE000646FF7EF85F0000E656F450E646F820E3F
:100BF0008425D96E020E8521DA6E600093F1DFFF45
:100C00007807D8A07907820E8C25016E020E8D21FF
:100C1000026E820E8425036E020E8521046EB1ECF5
:100C2000D3F0A9EF80F01200000E01017C6F000EDE
:100C30007B6F5DC18DF15EC18EF15FC18FF160C1CF
:100C400090F190BF28EF86F026EF86F03EEF86F019
:100C5000000E7C6F010E7B6F8DC100F18EC101F122
:100C60008FC102F190C103F17BECD8F000C18DF18E
:100C700001C18EF102C18FF103C190F1000E01019B
:100C8000946F000E936FEEC17FF1EFC180F17B5145
:100C90007C11D8A44EEF86F050EF86F057EF86F027
:100CA000F2A555EF86F057EF86F071EF86F07B5195
:100CB0007C11D8A45EEF86F060EF86F066EF86F0D8
:100CC000000E686F2B0E676F6AEF86F0000E686F7C
:100CD0002D0E676F67C182F2934B942B7F07D8A0CC
:100CE00080078DC100F18EC101F18FC102F190C169
:100CF00003F19CECC5F0010100050111D8A483EFBC
:100D000086F085EF86F0CFEF86F0BF0E626FFF0EA4
:100D1000636F6151646F656B625164276351652332
:100D2000655107E11A0E645DD8B099EF86F09BEF2C
:100D300086F0A9EF86F0820E9325046F020E9421AF
:100D4000056FDB0E066FFF0E076F46ECD3F0B5EFB5
:100D500086F0820E9325046F020E9421056FE30E38
:100D6000066FFF0E076F46ECD3F00101FD0E7F27E3
:100D7000FF0E80235BC110F15CC111F1820E0101F5
:100D8000126F020E136F7FC114F180C115F1F1ECE7
:100D9000CAF010C15BF111C15CF120EF8CF08DC184
:100DA00000F18EC101F18FC102F190C103F19CEC01
:100DB000C5F0010100510111D8A4E1EF86F0E3EF85
:100DC00086F015EF87F0BF0E626FFF0E636F615103
:100DD000646F656B6251642763516523655107E158
:100DE0001A0E645DD8B0F7EF86F0F9EF86F007EFE2
:100DF00087F0820E9325046F020E9421056FDF0E9B
:100E0000066FFF0E076F46ECD3F0B5EF86F0820E4B
:100E10009325046F020E9421056FE70E066FFF0EF7
:100E2000076F46ECD3F0B5EF86F0000E956F000E1D
:100E3000966F800E976F3F0E986F000E926F000EA8
:100E4000916F8DC100F18EC101F18FC102F190C18E
:100E500003F1000E046F000E056F000E066F000E0A
:100E6000076F42ECCEF00101D8B039EF87F03BEFCD
:100E700087F0C0EF87F05AEF87F095C115F196C162
:100E800016F197C117F198C118F1000E196F000EF5
:100E90001A6F200E1B6F410E1C6FB1ECA5F015C12F
:100EA00095F116C196F117C197F118C198F101019A
:100EB000914B922B8DC12EF18EC12FF18FC130F14C
:100EC00090C131F1000E196F000E1A6F200E1B6FCA
:100ED000410E1C6F95C115F196C116F197C117F11E
:100EE00098C118F1B1ECA5F015C132F116C133F17A
:100EF00017C134F118C135F114ECC4F00101D8B0B8
:100F000084EF87F086EF87F03DEF87F0A6EF87F05C
:100F100095C12EF196C12FF197C130F198C131F1F1
:100F2000000E326F000E336F200E346F410E356F9E
:100F300000ECAAF02EC195F12FC196F130C197F1C6
:100F400031C198F101019107D8A092078DC12EF10E
:100F50008EC12FF18FC130F190C131F195C132F1C5
:100F600096C133F197C134F198C135F114ECC4F056
:100F70000101D8A0BEEF87F0C0EF87F088EF87F0BF
:100F800061C106F1076BA6ECD6F001010651826F34
:100F900082C181F1670E8219D8A4D1EF87F0D3EF17
:100FA00087F0F9EF87F0F051F111D8A4DAEF87F06C
:100FB000DCEF87F0E0EF87F0000EF16F010EF06FCD
:100FC000F1BFEDEF87F0F15106E1F005D8B0EBEF9E
:100FD00087F0EDEF87F0F3EF87F0000E7E6F060EDF
:100FE0007D6F02EF88F0F0C17DF1F1C17EF102EF7B
:100FF00088F0F1BFFEEF87F000EF88F0EDEF87F0AB
:10100000F3EF87F0670E8219D8A409EF88F00BEF91
:1010100088F03AEF88F092AF19EF88F0FC0E915DFE
:10102000FF0E9259D8A017EF88F019EF88F038EF2B
:1010300088F0FF0E626FFF0E636F7DC164F17EC1A9
:1010400065F162516427635165239151645D655177
:10105000800A666F9251800A6659D8A032EF88F0F4
:1010600034EF88F038EF88F0660E816F3AEF88F041
:10107000650E816F7DC173F17EC174F1670E8219B7
:10108000D8A445EF88F047EF88F057EF88F0660E58
:101090008119D8A44EEF88F050EF88F059EF88F00E
:1010A00092BF57EF88F055EF88F059EF88F0734BF7
:1010B000742B660E8119D8A460EF88F062EF88F077
:1010C00082EF88F092BF69EF88F067EF88F075EFE4
:1010D00088F0000E956F000E966F800E976F3F0E92
:1010E000986F000E926F000E916F670E8219D8B440
:1010F0007CEF88F07EEF88F082EF88F091517327C3
:1011000092517423000E8C6F000E8B6F8DC183F192
:101110008EC184F18FC185F190C186F195C175F1C1
:1011200096C176F197C177F198C178F114EF89F003
:1011300083C12EF184C12FF185C130F186C131F117
:1011400095C132F196C133F197C134F198C135F1AF
:1011500000ECAAF02EC147F12FC148F130C149F18E
:1011600031C14AF163ECB4F047C187F148C188F15D
:1011700049C189F14AC18AF187C147F188C148F163
:1011800089C149F18AC14AF190ECC3F047C179F1B4
:1011900048C17AF183C12EF184C12FF185C130F1AC
:1011A00086C131F195C119F196C11AF197C11BF1B0
:1011B00098C11CF187C115F188C116F189C117F1D9
:1011C0008AC118F1B1ECA5F015C132F116C133F1A5
:1011D00017C134F118C135F1CAECD6F02EC183F134
:1011E0002FC184F130C185F131C186F195C12EF155
:1011F00096C12FF197C130F198C131F1000E010174
:10120000326F000E336F200E346F410E356F00ECDD
:10121000AAF02EC195F12FC196F130C197F131C1DD
:1012200098F101018B4B8C2B73518B5D8C51800A93
:10123000626F7451800A6259D8A021EF89F023EFC0
:1012400089F098EF88F095C115F196C116F197C114
:1012500017F198C118F1000E196F000E1A6FA00E49
:101260001B6F400E1C6FB1ECA5F015C187F116C1C4
:1012700088F117C189F118C18AF183C12EF184C1A7
:101280002FF185C130F186C131F187C132F188C1BA
:1012900033F189C134F18AC135F114ECC4F0010194
:1012A000D8B055EF89F057EF89F061EF89F0000E63
:1012B000876F000E886F000E896F000E8A6F8AEFAD
:1012C00089F083C100F184C101F185C102F186C1B9
:1012D00003F187C104F188C105F189C106F18AC112
:1012E00007F142ECCEF00101D8A079EF89F07BEF55
:1012F00089F08AEF89F079B180EF89F082EF89F087
:101300008AEF89F0000E876F000E886F000E896FDC
:10131000000E8A6F8DC100F18EC101F18FC102F103
:1013200090C103F187C104F188C105F189C106F1BB
:101330008AC107F1F0ECA0F000C183F101C184F192
:1013400002C185F103C186F183C12EF184C12FF161
:1013500085C130F186C131F1000E0101196F000E17
:101360001A6F200E1B6F410E1C6F75C115F176C1EF
:1013700016F177C117F178C118F1B1ECA5F015C1DC
:1013800032F116C133F117C134F118C135F114EC43
:10139000C4F00101D8A0CFEF89F0D1EF89F0F9EFC7
:1013A00089F0914B922B75C115F176C116F177C179
:1013B00017F178C118F1000E196F000E1A6F200E88
:1013C0001B6F410E1C6FB1ECA5F015C175F116C174
:1013D00076F117C177F118C178F1660E0101811914
:1013E000D8A4F5EF89F0F7EF89F0F9EF89F0734BA6
:1013F000742B75C195F176C196F177C197F178C1DB
:1014000098F1650E8119D8B408EF8AF00AEF8AF0D6
:1014100010EF8AF091C171F192C172F114EF8AF06C
:10142000000E726F000E716F000E706F000E6F6F06
:10143000000E6E6F000E6D6F000E8C6F000E8B6FC6
:1014400010EF8BF083C12EF184C12FF185C130F1F3
:1014500086C131F195C132F196C133F197C134F1B2
:1014600098C135F100ECAAF02EC147F12FC148F127
:1014700030C149F131C14AF163ECB4F047C187F1A1
:1014800048C188F149C189F14AC18AF187C147F150
:1014900088C148F189C149F18AC14AF190ECC3F091
:1014A00047C179F148C17AF10101F2B95AEF8AF0E6
:1014B0005CEF8AF079EF8AF079517A11D8A463EF62
:1014C0008AF065EF8AF079EF8AF0670E8219D8A466
:1014D0006CEF8AF06EEF8AF079EF8AF072BF75EFE9
:1014E0008AF073EF8AF079EF8AF06D4B6E2BC3EFC1
:1014F0008AF06F517011D8A480EF8AF082EF8AF0E1
:10150000ACEF8AF072BF89EF8AF087EF8AF0ACEF18
:101510008AF0820E9325D96E020E9421DA6E2E0E79
:10152000DF6E934B942B7F07D8A08007000E706F5F
:10153000010E6F6FACEF8AF0820E9325D96E020E0A
:101540009421DA6E300EDF6E934B942B7F07D8A078
:1015500080076D07D8A06E076D516E11D8A4B3EF48
:101560008AF0B5EF8AF09CEF8AF0820E9325D96E4F
:10157000020E9421DA6E7951300FDF6E934B942B6B
:101580007F07D8A0800783C12EF184C12FF185C1C8
:1015900030F186C131F195C119F196C11AF197C1A7
:1015A0001BF198C11CF187C115F188C116F189C1E1
:1015B00017F18AC118F1B1ECA5F015C132F116C1CD
:1015C00033F117C134F118C135F1CAECD6F02EC190
:1015D00083F12FC184F130C185F131C186F195C10C
:1015E0002EF196C12FF197C130F198C131F1000E63
:1015F0000101326F000E336F200E346F410E356FD4
:1016000000ECAAF02EC195F12FC196F130C197F1EF
:1016100031C198F101017107D8A072078B4B8C2B57
:1016200073518B5D8C51800A626F7451800A6259CC
:10163000D8B01DEF8BF01FEF8BF02DEF8BF094BF28
:101640002BEF8BF0945109E14B0E935DD8A02BEF5B
:101650008BF02DEF8BF022EF8AF06F517011D8A430
:1016600034EF8BF036EF8BF047EF8BF0F2A93BEFC6
:101670008BF03DEF8BF047EF8BF0820E9325D96E08
:10168000020E9421DA6E2E0EDF6E934B942B820E97
:101690009325D96E020E9421DA6E000EDF6E650E70
:1016A0008119D8A456EF8BF058EF8BF0BAEF86F083
:1016B000000E8C6F4F0E8B6F820E8B25D96E020E33
:1016C0008C21DA6E000EDF6E000E7C6F000E7B6FD9
:1016D00092BF6FEF8BF06DEF8BF077EF8BF0000E1A
:1016E0007C6F010E7B6F916D921FD8B0922B000E14
:1016F0007E6F020E7D6FA9EF8BF08B07D8A08C0751
:10170000820E8B25D96E020E8C21DA6E91C100F10A
:1017100092C101F1000E036F0A0E026F3AECCDF098
:1017200001010051300FDF6E91C100F192C101F152
:10173000000E036F0A0E026F56ECCBF000C191F160
:1017400001C192F101017D07D8A07E077F07D8A0D3
:10175000800791519211D8A4B0EF8BF0B2EF8BF0CB
:101760007DEF8BF07EBFBFEF8BF07E5106E17D05F4
:10177000D8B0BDEF8BF0BFEF8BF07DEF8BF08B0718
:10178000D8A08C077B517C11D8A4C9EF8BF0CBEF8C
:101790008BF0D1EF8BF0000E6A6F2B0E696FD5EFD7
:1017A0008BF0000E6A6F2D0E696F820E8B25D96E3D
:1017B000020E8C21DA6E6000A7F5DFFF7F07D8A04C
:1017C00080078B07D8A08C07BF0E626FFF0E636F78
:1017D0006151646F656B6251642763516523655184
:1017E00009E11A0E645DD8A0F8EF8BF0FAEF8BF0E8
:1017F00000EF8CF0000E6C6F650E6B6F04EF8CF0D9
:10180000000E6C6F450E6B6F820E8B25D96E020E2B
:101810008C21DA6E6000AFF5DFFF7F07D8A080076C
:10182000820E9325046F020E9421056F820E8B2584
:10183000066F020E8C21076F46ECD3F0BAEF86F0EC
:101840001200600053F2D9FF600057F2DAFF6F0018
:101850007BFFF6FF6F0077FFF7FF000EF86E0800C2
:10186000F550250AD8A437EF8CF039EF8CF0E5EF6E
:1018700091F0600053F2D9FF600057F2DAFFDE2AE0
:10188000000EDD22000E0101EF6F000EEE6FEEC1C3
:10189000F2F1EFC1F3F1F069F169000E0001A36FFD
:1018A000000EA26FA7EF8CF00101F281600053F2ED
:1018B000D9FF600057F2DAFFDE2A000EDD22A7EF23
:1018C0008CF00101F28356EF8CF00101F28556EFA6
:1018D0008CF00101F28756EF8CF00101F28956EF8E
:1018E0008CF0000EA36F010EA26FA7EF8CF06000CA
:1018F00053F2D9FF600057F2DAFF6F007BFFF6FF6B
:101900006F0077FFF7FF000EF86E0800F550406E8D
:10191000416A4150000AD8B490EF8CF071EF8CF01E
:101920004050200AD8B469EF8CF0030AD8B46DEFA8
:101930008CF0080AD8B465EF8CF0060AD8B454EFDE
:101940008CF01D0AD8B461EF8CF071EF8CF00001BF
:10195000A251A311D8B4AFEF8CF0B1EF8CF077EFB8
:101960008CF00101F2A1B7EF8CF0B9EF8CF0BAEF77
:101970008CF0F293600053F2D9FF600057F2DAFF67
:101980006F007BFFF6FF6F0077FFF7FF000EF86E2A
:101990000800F5502A0AD8A4D0EF8CF0D2EF8CF0D2
:1019A00005EF8DF0600053F2D9FF600057F2DAFFC7
:1019B000DE2A000EDD2260005BF2D9FF60005FF2DC
:1019C000DAFF6F007CFF40F0020EDE266F007CFF26
:1019D00041F0000EDD22600003F1D9FF600007F145
:1019E000DAFF6F0078FFEEF16F0074FFEFF1EFBFE9
:1019F000FEEF8CF0FCEF8CF047EF8DF0F281EE6D96
:101A0000EF1FD8B0EF2B47EF8DF0600053F2D9FFF6
:101A1000600057F2DAFF6F0078FF07F06F0074FF85
:101A200008F01FECBEF007C0EEF108C0EFF122EFA6
:101A30008DF0600053F2D9FF600057F2DAFFDE2A22
:101A4000000EDD22D00E406EFF0E416E600053F29C
:101A5000D9FF600057F2DAFF6F007BFFF6FF6F00DF
:101A600077FFF7FF000EF86E0800F550426E436AEC
:101A70004050422641504322435009E10A0E425C45
:101A8000D8A045EF8DF047EF8DF019EF8DF0600095
:101A900053F2D9FF600057F2DAFF6F007BFFF6FFC9
:101AA0006F0077FFF7FF000EF86E0800F5502E0A62
:101AB000D8A45DEF8DF05FEF8DF0EEEF8DF0000EAE
:101AC0000101F16F000EF06F600053F2D9FF60006A
:101AD00057F2DAFFDE2A000EDD22600053F2D9FF52
:101AE000600057F2DAFF6F007BFFF6FF6F0077FFB1
:101AF000F7FF000EF86E0800F5502A0AD8A483EF0D
:101B00008DF085EF8DF0ACEF8DF0600053F2D9FFD2
:101B1000600057F2DAFFDE2A000EDD2260005BF281
:101B2000D9FF60005FF2DAFF6F007CFF40F0020E29
:101B3000DE266F007CFF41F0000EDD22600003F125
:101B4000D9FF600007F1DAFF6F0078FFF0F16F0056
:101B500074FFF1F1EEEF8DF0600053F2D9FF6000F9
:101B600057F2DAFF6F0078FF07F06F0074FF08F09C
:101B70001FECBEF007C0F0F108C0F1F1C9EF8DF025
:101B8000600053F2D9FF600057F2DAFFDE2A000E40
:101B9000DD22D00E406EFF0E416E600053F2D9FF81
:101BA000600057F2DAFF6F007BFFF6FF6F0077FFF0
:101BB000F7FF000EF86E0800F550426E436A405081
:101BC000422641504322435009E10A0E425CD8A00C
:101BD000ECEF8DF0EEEF8DF0C0EF8DF0600053F282
:101BE000D9FF600057F2DAFF6F007BFFF6FF6F004E
:101BF00077FFF7FF000EF86E0800F550036E046AD9
:101C000035ECD7F003500001B26FB251D8B40BEFEE
:101C10008EF00DEF8EF057EF8EF0600053F2D9FF8B
:101C2000600057F2DAFF6F0078FF40F06F0074FF3A
:101C300041F0010E4026000E4122600003F1F6FF44
:101C4000600007F1F7FF000EF86E0800F550036E14
:101C5000046A35ECD7F003500001B36FB351D8B428
:101C600034EF8EF036EF8EF057EF8EF0600053F2C7
:101C7000D9FF600057F2DAFF6F0078FF40F06F0085
:101C800074FF41F0020E4026000E4122600003F175
:101C9000F6FF600007F1F7FF000EF86E0800F55040
:101CA000036E046A35ECD7F003500001B46F600096
:101CB00053F2D9FF600057F2DAFF6F007BFFF6FFA7
:101CC0006F0077FFF7FF000EF86E0800F550630A0B
:101CD000D8A46DEF8EF06FEF8EF09EEF8EF0600067
:101CE00053F2D9FF600057F2DAFFDE2A000EDD2240
:101CF00060005BF2D9FF60005FF2DAFF6F007CFFEB
:101D000040F0020EDE266F007CFF41F0000EDD2267
:101D1000600003F1D9FF600007F1DAFFDF50B56F13
:101D200092C00AF093C00BF0B5C00CF0E3ECC8F021
:101D30000AC092F00BC093F008EF92F0600053F2EB
:101D4000D9FF600057F2DAFF6F007BFFF6FF6F00EC
:101D500077FFF7FF000EF86E0800F550640AD8B45C
:101D6000B4EF8EF0B6EF8EF0CEEF8EF0600053F24F
:101D7000D9FF600057F2DAFF6F007BFFF6FF6F00BC
:101D800077FFF7FF000EF86E0800F550690AD8A437
:101D9000CCEF8EF0CEEF8EF018EF8FF0600053F2A4
:101DA000D9FF600057F2DAFFDE2A000EDD22600064
:101DB0005BF2D9FF60005FF2DAFF6F007CFF40F05A
:101DC000020EDE266F007CFF41F0000EDD22600077
:101DD00003F1D9FF600007F1DAFF6F0078FF98F098
:101DE0006F0074FF99F0000E99BFFF0E9A6F9B6F02
:101DF0009C6F9D6F9E6F9F6F92C01CF093C01DF0F3
:101E000098C01EF099C01FF09AC020F09BC021F02E
:101E10009CC022F09DC023F09EC024F09FC025F0FE
:101E20000EECAFF01CC092F01DC093F008EF92F0E2
:101E3000660EB219D8A41FEF8FF021EF8FF074EF68
:101E40008FF0600053F2D9FF600057F2DAFF6F00A5
:101E50007BFFF6FF6F0077FFF7FF000EF86E0800BC
:101E60006F00D4FFB5F0600053F2D9FF600057F265
:101E7000DAFFDE2A000EDD2260005BF2D9FF60008F
:101E80005FF2DAFF6F007CFF40F0040EDE266F0089
:101E90007CFF41F0000EDD22600003F1D9FF6000FD
:101EA00007F1DAFF6F0078FFAEF06F0078FFAFF058
:101EB0006F0078FFB0F06F0078FFB1F092C02EF0A5
:101EC00093C02FF0AEC030F0AFC031F0B0C032F0F0
:101ED000B1C033F0B5C034F000EC80F02EC092F009
:101EE0002FC093F008EF92F0B20E016E000E026E5A
:101EF000FB0E036EFF0E046E000E066E020E056EE4
:101F000048ECC2F001500210D8A489EF8FF08BEF9B
:101F10008FF01EEF90F0600053F2D9FF600057F28F
:101F2000DAFF6F0078FF40F06F0074FF41F0010EA0
:101F30004026000E4122600003F1F6FF600007F129
:101F4000F7FF000EF86E08006F00D4FFB5F0BF0E6B
:101F5000406EFF0E416E600053F2D9FF600057F2F1
:101F6000DAFF6F007BFFF6FF6F0077FFF7FF000ED1
:101F7000F86E0800F550426E436A405042264150C8
:101F80004322435007E11A0E425CD8B0CAEF8FF0EB
:101F9000CCEF8FF0F0EF8FF060005BF2D9FF6000C4
:101FA0005FF2DAFF6F007CFF40F0040EDE266F0068
:101FB0007CFF41F0000EDD22600003F1D9FF6000DC
:101FC00007F1DAFF6F0078FFAEF06F0078FFAFF037
:101FD0006F0078FFB0F06F0078FFB1F012EF90F073
:101FE00060005BF2D9FF60005FF2DAFF6F007CFFF8
:101FF00040F0040EDE266F007CFF41F0000EDD2273
:10200000600003F1D9FF600007F1DAFF6F0078FF8D
:10201000AEF06F0078FFAFF06F0078FFB0F06F00A8
:1020200078FFB1F0020E600053F2D9FF600057F262
:10203000DAFFDE26000EDD225EEF8FF0600053F245
:10204000D9FF600057F2DAFF6F007BFFF6FF6F00E9
:1020500077FFF7FF000EF86E0800F550730AD8B44A
:1020600034EF90F036EF90F055EF90F0600053F2BF
:10207000D9FF600057F2DAFF6F0078FF01F06F00C0
:1020800074FF02F0EB0E036EFF0E046E000E066E80
:10209000030E056E48ECC2F001500210D8A453EFB5
:1020A00090F055EF90F0AFEF90F0600053F2D9FF51
:1020B000600057F2DAFF6F007BFFF6FF6F0077FFDB
:1020C000F7FF000EF86E0800F550730AD8B46BEFF6
:1020D00090F06DEF90F074EF90F0000E0001A56F9E
:1020E000030EA46F79EF90F0000E0001A56F010EB2
:1020F000A46F600053F2D9FF600057F2DAFFA451D9
:10210000DE26A551DD2260005BF2D9FF60005FF2A0
:10211000DAFF6F007CFF40F0020EDE266F007CFFCE
:1021200041F0000EDD22600003F1D9FF600007F1ED
:10213000DAFF6F0078FFA0F06F0074FFA1F092C08B
:102140000AF093C00BF0A0C00CF0A1C00DF030EC71
:10215000BAF00AC092F00BC093F008EF92F0600062
:1021600053F2D9FF600057F2DAFF6F007BFFF6FFF2
:102170006F0077FFF7FF000EF86E0800F550750A44
:10218000D8A4C5EF90F0C7EF90F013EF91F0600086
:1021900053F2D9FF600057F2DAFFDE2A000EDD228B
:1021A00060005BF2D9FF60005FF2DAFF6F007CFF36
:1021B00040F0020EDE266F007CFF41F0000EDD22B3
:1021C000600003F1D9FF600007F1DAFF6F0078FFCC
:1021D00042F06F0074FF43F042C0A6F043C0A7F086
:1021E0000001A86BA96BAA6BAB6BAC6BAD6B92C01B
:1021F0001CF093C01DF0A6C01EF0A7C01FF0A8C021
:1022000020F0A9C021F0AAC022F0ABC023F0ACC0DE
:1022100024F0ADC025F07AECB7F01CC092F01DC0E0
:1022200093F008EF92F0600053F2D9FF600057F28C
:10223000DAFF6F007BFFF6FF6F0077FFF7FF000EFE
:10224000F86E0800F550780AD8B429EF91F02BEF1A
:1022500091F043EF91F0600053F2D9FF600057F224
:10226000DAFF6F007BFFF6FF6F0077FFF7FF000ECE
:10227000F86E0800F550580AD8A441EF91F043EFEA
:1022800091F0A3EF91F0600053F2D9FF600057F294
:10229000DAFF6F007BFFF6FF6F0077FFF7FF000E9E
:1022A000F86E08006F00D4FFB5F0600053F2D9FF5C
:1022B000600057F2DAFFDE2A000EDD2260005BF2DA
:1022C000D9FF60005FF2DAFF6F007CFF40F0020E82
:1022D000DE266F007CFF41F0000EDD22600003F17E
:1022E000D9FF600007F1DAFF6F0078FF42F06F005E
:1022F00074FF43F042C0A6F043C0A7F00001A86BF2
:10230000A96BAA6BAB6BAC6BAD6B92C01CF093C0AE
:102310001DF0A6C01EF0A7C01FF0A8C020F0A9C0E5
:1023200021F0AAC022F0ABC023F0ACC024F0ADC0B5
:1023300025F0B5C026F0D6ECB1F01CC092F01DC05F
:1023400093F008EF92F0600053F2D9FF600057F26B
:10235000DAFF6F007BFFF6FF6F0077FFF7FF000EDD
:10236000F86E0800F550250AD8A4B9EF91F0BBEF3C
:1023700091F0D5EF91F0600053F2D9FF600057F271
:10238000DAFFDE2A000EDD22000E026E250E016E3F
:1023900092C003F093C004F04FECC9F0000E0001AE
:1023A000936F010E926F08EF92F0600053F2D9FF25
:1023B000600057F2DAFFDE2A000EDD22000E000177
:1023C000936F000E926F08EF92F0600053F2D9FF06
:1023D000600057F2DAFF6F007BFFF6FF6F0077FFB8
:1023E000F7FF000EF86E0800F550016E026A92C009
:1023F00003F093C004F04FECC9F0600053F2D9FF32
:10240000600057F2DAFFDE2A000EDD22CEEF91F0F7
:10241000120060006FF6D9FF600073F6DAFF6F00FC
:102420007BFFF6FF6F0077FFF7FF000EF86E0800E6
:10243000F550250AD8A41FEF92F021EF92F0C3EFD8
:1024400097F060006FF6D9FF600073F6DAFFDE2ABE
:10245000000EDD22000E0101EF6F000EEE6FEEC1E7
:10246000F2F1EFC1F3F1F069F169000EAE6F000E09
:10247000AD6F89EF92F0F28160006FF6D9FF6000D6
:1024800073F6DAFFDE2A000EDD2289EF92F0F28386
:102490003CEF92F0F2853CEF92F0F2873CEF92F045
:1024A000F2893CEF92F0000EAE6F010EAD6F89EF36
:1024B00092F060006FF6D9FF600073F6DAFF6F00EC
:1024C0007BFFF6FF6F0077FFF7FF000EF86E080046
:1024D000F5509F6FA06BA051000AD8B472EF92F034
:1024E00053EF92F09F51200AD8B44DEF92F0030AB7
:1024F000D8B450EF92F0080AD8B44AEF92F0060A26
:10250000D8B43BEF92F01D0AD8B447EF92F053EFE6
:1025100092F0AD51AE11D8B490EF92F092EF92F0EC
:1025200059EF92F0F2A197EF92F099EF92F09AEFB3
:1025300092F0F29360006FF6D9FF600073F6DAFF55
:102540006F007BFFF6FF6F0077FFF7FF000EF86E5E
:102550000800F5502A0AD8A4B0EF92F0B2EF92F03A
:10256000E5EF92F060006FF6D9FF600073F6DAFFD6
:10257000DE2A000EDD22600077F6D9FF60007BF6D0
:10258000DAFF6F007CFF9FF1020EDE266F007CFFFA
:10259000A0F1000EDD2260007FF6D9FF600083F617
:1025A000DAFF6F0078FFEEF16F0074FFEFF1EFBF1D
:1025B000DEEF92F0DCEF92F028EF93F0F281EE6D17
:1025C000EF1FD8B0EF2B28EF93F060006FF6D9FF24
:1025D000600073F6DAFF6F0078FF07F16F0074FF99
:1025E00008F15EECBDF007C1EEF108C1EFF102EFBA
:1025F00093F060006FF6D9FF600073F6DAFFDE2A11
:10260000000EDD22D00E01019F6FFF0EA06F600053
:102610006FF6D9FF600073F6DAFF6F007BFFF6FFFD
:102620006F0077FFF7FF000EF86E0800F550A16FFE
:10263000A26B9F51A127A051A223A25109E10A0E2A
:10264000A15DD8A026EF93F028EF93F0F9EF92F078
:1026500060006FF6D9FF600073F6DAFF6F007BFF52
:10266000F6FF6F0077FFF7FF000EF86E0800F550D9
:102670002E0AD8A43EEF93F040EF93F0CFEF93F003
:10268000000EF16F000EF06F60006FF6D9FF600072
:1026900073F6DAFFDE2A000EDD2260006FF6D9FF46
:1026A000600073F6DAFF6F007BFFF6FF6F0077FFC5
:1026B000F7FF000EF86E0800F5502A0AD8A463EF61
:1026C00093F065EF93F08CEF93F060006FF6D9FF15
:1026D000600073F6DAFFDE2A000EDD22600077F676
:1026E000D9FF60007BF6DAFF6F007CFF9FF1020EDE
:1026F000DE266F007CFFA0F1000EDD2260007FF679
:10270000D9FF600083F6DAFF6F0078FFF0F16F0009
:1027100074FFF1F1CFEF93F060006FF6D9FF600026
:1027200073F6DAFF6F0078FF07F16F0074FF08F1AE
:102730005EECBDF007C1F0F108C1F1F1A9EF93F033
:1027400060006FF6D9FF600073F6DAFFDE2A000E34
:10275000DD22D00E01019F6FFF0EA06F60006FF6AB
:10276000D9FF600073F6DAFF6F007BFFF6FF6F00A2
:1027700077FFF7FF000EF86E0800F550A16FA26B0F
:102780009F51A127A051A223A25109E10A0EA15DE8
:10279000D8A0CDEF93F0CFEF93F0A0EF93F06000CF
:1027A0006FF6D9FF600073F6DAFF6F007BFFF6FF6C
:1027B0006F0077FFF7FF000EF86E0800F550066F08
:1027C000076BA6ECD6F001010651BD6FBD51D8B420
:1027D000ECEF93F0EEEF93F038EF94F060006FF6CB
:1027E000D9FF600073F6DAFF6F0078FF9FF16F008A
:1027F00074FFA0F1010E9F27000EA02360007FF65A
:10280000F6FF600083F6F7FF000EF86E0800F55043
:10281000066F076BA6ECD6F001010651BE6FBE51E4
:10282000D8B415EF94F017EF94F038EF94F06000FF
:102830006FF6D9FF600073F6DAFF6F0078FF9FF143
:102840006F0074FFA0F1020E9F27000EA02360000E
:102850007FF6F6FF600083F6F7FF000EF86E0800C3
:10286000F550066F076BA6ECD6F001010651BF6F5D
:1028700060006FF6D9FF600073F6DAFF6F007BFF30
:10288000F6FF6F0077FFF7FF000EF86E0800F550B7
:10289000630AD8A44EEF94F050EF94F07FEF94F0D9
:1028A00060006FF6D9FF600073F6DAFFDE2A000ED3
:1028B000DD22600077F6D9FF60007BF6DAFF6F005B
:1028C0007CFF9FF1020EDE266F007CFFA0F1000E60
:1028D000DD2260007FF6D9FF600083F6DAFFDF506B
:1028E000C06F99C109F19AC10AF1C0C10BF108EC9E
:1028F000C8F009C199F10AC19AF1E7EF97F06000B9
:102900006FF6D9FF600073F6DAFF6F007BFFF6FF0A
:102910006F0077FFF7FF000EF86E0800F550640AAD
:10292000D8B495EF94F097EF94F0AFEF94F0600087
:102930006FF6D9FF600073F6DAFF6F007BFFF6FFDA
:102940006F0077FFF7FF000EF86E0800F550690A78
:10295000D8A4ADEF94F0AFEF94F0F9EF94F06000ED
:102960006FF6D9FF600073F6DAFFDE2A000EDD2273
:10297000600077F6D9FF60007BF6DAFF6F007CFF1E
:102980009FF1020EDE266F007CFFA0F1000EDD221B
:1029900060007FF6D9FF600083F6DAFF6F0078FFF2
:1029A000A3F16F0074FFA4F1000EA4BFFF0EA56F8A
:1029B000A66FA76FA86FA96FAA6F99C11BF19AC1E3
:1029C0001CF1A3C11DF1A4C11EF1A5C11FF1A6C137
:1029D00020F1A7C121F1A8C122F1A9C123F1AAC107
:1029E00024F19BECADF01BC199F11CC19AF1E7EF0A
:1029F00097F0660EBD19D8A400EF95F002EF95F0A0
:102A000055EF95F060006FF6D9FF600073F6DAFFBE
:102A10006F007BFFF6FF6F0077FFF7FF000EF86E89
:102A200008006F00D4FFC0F160006FF6D9FF6000AE
:102A300073F6DAFFDE2A000EDD22600077F6D9FF9A
:102A400060007BF6DAFF6F007CFF9FF1040EDE264C
:102A50006F007CFFA0F1000EDD2260007FF6D9FF41
:102A6000600083F6DAFF6F0078FFB9F16F0078FF3E
:102A7000BAF16F0078FFBBF16F0078FFBCF199C12C
:102A80005BF19AC15CF1B9C15DF1BAC15EF1BBC144
:102A90005FF1BCC160F1C0C161F114EC86F05BC1B3
:102AA00099F15CC19AF1E7EF97F0BD0E006F010E4E
:102AB000016FFB0E026FFF0E036F000E056F020E1B
:102AC000046FF0ECC0F0010100510111D8A46BEFCC
:102AD00095F06DEF95F000EF96F060006FF6D9FF7E
:102AE000600073F6DAFF6F0078FF9FF16F0074FFEC
:102AF000A0F1010E9F27000EA02360007FF6F6FFD5
:102B0000600083F6F7FF000EF86E08006F00D4FF38
:102B1000C0F1BF0E9F6FFF0EA06F60006FF6D9FF70
:102B2000600073F6DAFF6F007BFFF6FF6F0077FF40
:102B3000F7FF000EF86E0800F550A16FA26B9F51D1
:102B4000A127A051A223A25107E11A0EA15DD8B07E
:102B5000ACEF95F0AEEF95F0D2EF95F0600077F620
:102B6000D9FF60007BF6DAFF6F007CFF9FF1040E57
:102B7000DE266F007CFFA0F1000EDD2260007FF6F4
:102B8000D9FF600083F6DAFF6F0078FFB9F16F00BC
:102B900078FFBAF16F0078FFBBF16F0078FFBCF1EE
:102BA000F4EF95F0600077F6D9FF60007BF6DAFF6E
:102BB0006F007CFF9FF1040EDE266F007CFFA0F10A
:102BC000000EDD2260007FF6D9FF600083F6DAFF99
:102BD0006F0078FFB9F16F0078FFBAF16F0078FFEE
:102BE000BBF16F0078FFBCF1020E60006FF6D9FFF9
:102BF000600073F6DAFFDE26000EDD223FEF95F06F
:102C000060006FF6D9FF600073F6DAFF6F007BFF9C
:102C1000F6FF6F0077FFF7FF000EF86E0800F55023
:102C2000730AD8B416EF96F018EF96F038EF96F0D6
:102C300060006FF6D9FF600073F6DAFF6F0078FF6F
:102C400000F16F0074FF01F1EB0E026FFF0E036FD6
:102C5000000E056F030E046FF0ECC0F0010100518F
:102C60000111D8A436EF96F038EF96F090EF96F079
:102C700060006FF6D9FF600073F6DAFF6F007BFF2C
:102C8000F6FF6F0077FFF7FF000EF86E0800F550B3
:102C9000730AD8B44EEF96F050EF96F056EF96F0D8
:102CA000000EB06F030EAF6F5AEF96F0000EB06FCC
:102CB000010EAF6F60006FF6D9FF600073F6DAFFA8
:102CC000AF51DE26B051DD22600077F6D9FF6000FB
:102CD0007BF6DAFF6F007CFF9FF1020EDE266F00AD
:102CE0007CFFA0F1000EDD2260007FF6D9FF6000BE
:102CF00083F6DAFF6F0078FFABF16F0074FFACF181
:102D000099C109F19AC10AF1ABC10BF1ACC10CF147
:102D100058ECB9F009C199F10AC19AF1E7EF97F0BF
:102D200060006FF6D9FF600073F6DAFF6F007BFF7B
:102D3000F6FF6F0077FFF7FF000EF86E0800F55002
:102D4000750AD8A4A6EF96F0A8EF96F0F3EF96F0E8
:102D500060006FF6D9FF600073F6DAFFDE2A000E1E
:102D6000DD22600077F6D9FF60007BF6DAFF6F00A6
:102D70007CFF9FF1020EDE266F007CFFA0F1000EAB
:102D8000DD2260007FF6D9FF600083F6DAFF6F0076
:102D900078FFA1F16F0074FFA2F1A1C1B1F1A2C14E
:102DA000B2F1B36BB46BB56BB66BB76BB86B99C163
:102DB0001BF19AC11CF1B1C11DF1B2C11EF1B3C129
:102DC0001FF1B4C120F1B5C121F1B6C122F1B7C1E3
:102DD00023F1B8C124F177ECB6F01BC199F11CC105
:102DE0009AF1E7EF97F060006FF6D9FF600073F695
:102DF000DAFF6F007BFFF6FF6F0077FFF7FF000E33
:102E0000F86E0800F550780AD8B409EF97F00BEF88
:102E100097F023EF97F060006FF6D9FF600073F62C
:102E2000DAFF6F007BFFF6FF6F0077FFF7FF000E02
:102E3000F86E0800F550580AD8A421EF97F023EF58
:102E400097F082EF97F060006FF6D9FF600073F69D
:102E5000DAFF6F007BFFF6FF6F0077FFF7FF000ED2
:102E6000F86E08006F00D4FFC0F160006FF6D9FF64
:102E7000600073F6DAFFDE2A000EDD22600077F6CE
:102E8000D9FF60007BF6DAFF6F007CFF9FF1020E36
:102E9000DE266F007CFFA0F1000EDD2260007FF6D1
:102EA000D9FF600083F6DAFF6F0078FFA1F16F00B1
:102EB00074FFA2F1A1C1B1F1A2C1B2F1B36BB46BC5
:102EC000B56BB66BB76BB86B99C11BF19AC11CF1AE
:102ED000B1C11DF1B2C11EF1B3C11FF1B4C120F1E6
:102EE000B5C121F1B6C122F1B7C123F1B8C124F1B6
:102EF000C0C125F181ECB0F01BC199F11CC19AF160
:102F0000E7EF97F060006FF6D9FF600073F6DAFF25
:102F10006F007BFFF6FF6F0077FFF7FF000EF86E84
:102F20000800F550250AD8A498EF97F09AEF97F08B
:102F3000B4EF97F060006FF6D9FF600073F6DAFF28
:102F4000DE2A000EDD22000E016F250E006F99C1F2
:102F500002F19AC103F176ECC8F0000E01019A6FFC
:102F6000010E996FE7EF97F060006FF6D9FF6000F0
:102F700073F6DAFFDE2A000EDD22000E9A6F000ED5
:102F8000996FE7EF97F060006FF6D9FF600073F676
:102F9000DAFF6F007BFFF6FF6F0077FFF7FF000E91
:102FA000F86E0800F5500101006F016B99C102F144
:102FB0009AC103F176ECC8F060006FF6D9FF6000AB
:102FC00073F6DAFFDE2A000EDD22ADEF97F0120075
:102FD00001ECD1F0520E0101E76F2B0EE66F000EEF
:102FE000E82EFED7E62FFCD7E72FFAD700F0000136
:102FF000F405D8A4FEEF97F000EF98F0BAEF9CF03C
:10300000D40E0101006FFF0E016F36ECD5F0800E7B
:103010000101006F040E016FB4ECD1F09CECD9F00B
:10302000800E0101F66F040EF76F6000DBF7D9FF29
:103030006000DFF7DAFF480EDE18D8A422EF98F020
:1030400024EF98F0A4EF98F020EE01F0F651D92685
:10305000F751DA22650EDE18D8A431EF98F033EF7D
:1030600098F0A4EF98F020EE02F0F651D926F7512F
:10307000DA226C0EDE18D8A440EF98F042EF98F0F8
:10308000A4EF98F020EE03F0F651D926F751DA229A
:10309000700EDE18D8A44FEF98F051EF98F0A4EF1F
:1030A00098F0F40E006FFD0E016F36ECD5F0FF0EB8
:1030B0000101006FFB0E016F36ECD5F0780E0101B7
:1030C000006FFB0E016F36ECD5F0EA0E0101006FC8
:1030D000FA0E016F36ECD5F01C0E0101006FFA0EEE
:1030E000016F36ECD5F01A0E0101006FFB0E016F77
:1030F00036ECD5F0260E0101006FFD0E016F36ECA7
:10310000D5F0050E0101006FFD0E016F36ECD5F014
:10311000710E0101006FFE0E016F36ECD5F0B20E9C
:103120000101006FFF0E016F36ECD5F0800E01013A
:10313000006F040E016FB4ECD1F09CECD9F0000EDE
:103140000101F66F000EF76F6000DBF7D9FF60003A
:10315000DFF7DAFF480EDE18D8A4B1EF98F0B3EF2E
:1031600098F0BCEF98F0BC92000E0001EE6F000EDC
:103170000101F66F000EF76F6000DBF7D9FF60000A
:10318000DFF7DAFF540EDE18D8A4C9EF98F0CBEFC2
:1031900098F0D4EF98F0010E0001EE6FBC82000EA3
:1031A0000101F66F000EF76F6000DBF7D9FF6000DA
:1031B000DFF7DAFF4D0EDE18D8A4E1EF98F0E3EF69
:1031C00098F058EF99F020EE01F0F651D926F7511A
:1031D000DA226F0EDE18D8A4F0EF98F0F2EF98F034
:1031E00058EF99F020EE02F0F651D926F751DA2285
:1031F000640EDE18D8A4FFEF98F001EF99F058EFB5
:1032000099F020EE03F0F651D926F751DA223D0E5F
:10321000DE18D8A40EEF99F010EF99F058EF99F05E
:1032200020EE04F0F651D926F751DA22310EDE18DD
:10323000D8A41DEF99F01FEF99F045EF99F0010E1A
:103240000001EB6F110E0101006FF90E016F36ECFA
:10325000D5F0C20E0101006FFC0E016F36ECD5F007
:10326000580E0101006FF90E016F36ECD5F09C0E7F
:103270000101006FF90E016F36ECD5F0000E01016F
:10328000F66F000EF76F58EF99F0000E0001EB6F2C
:10329000290E0101006FFC0E016F36ECD5F0C90E4E
:1032A0000101006FF80E016F36ECD5F03EEF99F09A
:1032B0000001EB51D8A45FEF99F061EF99F017EF9F
:1032C0009BF06000DBF7D9FF6000DFF7DAFF460E06
:1032D000DE18D8A46EEF99F070EF99F017EF9BF01D
:1032E000010120EE01F0F651D926F751DA223D0E08
:1032F000DE18D8A47EEF99F080EF99F017EF9BF0DD
:10330000F6C100F1F7C101F1DAECD4F0060E0101CB
:1033100000190111D8A48FEF99F091EF99F017EFF0
:103320009BF0D00EE66FFF0EE76F20EE02F0F65135
:10333000D926F751DA22DF50E86FE96BE651E8272A
:10334000E751E923E95107E10A0EE85DD8B0ABEF98
:1033500099F0ADEF99F00CEF9BF0D00EE66FFF0EF9
:10336000E76F20EE03F0F651D926F751DA22DF504D
:10337000E86FE96BE651E827E751E923E95107E1F6
:103380000A0EE85DD8B0C7EF99F0C9EF99F00CEFDD
:103390009BF0D00EE66FFF0EE76F20EE04F0F651C3
:1033A000D926F751DA22DF50E86FE96BE651E827BA
:1033B000E751E923E95107E10A0EE85DD8B0E3EFF0
:1033C00099F0E5EF99F00CEF9BF0D00EE66FFF0E51
:1033D000E76F20EE05F0F651D926F751DA22DF50DB
:1033E000E86FE96BE651E827E751E923E95107E186
:1033F0000A0EE85DD8B0FFEF99F001EF9AF00CEFFC
:103400009BF020EE02F0F651D926F751DA22DF5078
:10341000D00FFC6FFCC100F1016B030E036FE80ECF
:10342000026FE1ECD9F000C15BF001C15CF0010179
:1034300020EE03F0F651D926F751DA22DF50D00FF3
:10344000FC6FFC51640D6F00CCFFE6F16F00D0FF04
:10345000E7F15B50E6255B6E5C50E7215C6E20EE89
:1034600004F0F651D926F751DA22DF50D00FFC6F65
:10347000FC510A0D6F00CCFFE6F16F00D0FFE7F1C1
:103480005B50E6255B6E5C50E7215C6E20EE05F03C
:10349000F651D926F751DA22DF50D00FFC6FFC51DC
:1034A0005B245B6E000E5C205C6E5C5009E1C80E14
:1034B0005B5CD8A05EEF9AF060EF9AF012EF9BF0A1
:1034C000710E5B5C170E5C58D8B069EF9AF06BEF29
:1034D0009AF012EF9BF05BC007F15CC008F1096B3A
:1034E0000A6B000E7CECB8F007C1D0F008C1D1F037
:1034F00009C1D2F00AC1D3F05D50040DEE0EF324E1
:10350000F66EF50EF420F76EF86A000EF822090048
:103510006F00D4FF32F109006F00D4FF33F10900CE
:103520006F00D4FF34F10A006F00D4FF35F1000EB4
:103530000101196F000E1A6F000E1B6F4A0E1C6FEF
:10354000D0C015F1D1C016F1D2C017F1D3C018F117
:10355000B1ECA5F015C12EF116C12FF117C130F154
:1035600018C131F100ECAAF02EC147F12FC148F18A
:1035700030C149F131C14AF190ECC3F047C1F9F0D3
:1035800048C1FAF049C1FBF04AC1FCF0300E01011C
:10359000C96F030ECA6F500ECB6FFC0ECC6F5BC0B1
:1035A000CDF15CC0CEF1F9C0CFF1FAC0D0F1FBC0D3
:1035B000D1F1FCC0D2F1E2ECD5F0300E0101006F88
:1035C000030E016FB4ECD1F0BCA0E9EF9AF0EBEF81
:1035D0009AF012EF9BF03F013E9F010120EE02F0B6
:1035E000F451D926F551DA22DF503F013D6F010138
:1035F00020EE01F0F451D926F551DA22DF503F01D7
:103600003C6F6000D3F7D9FF6000D7F7DAFFDF50D7
:103610003B6F3E8F12EF9BF0E40E006FFC0E016FCC
:1036200036ECD5F0000E0101F66F000EF76F60006A
:10363000DBF7D9FF6000DFF7DAFF420EDE18D8A40F
:1036400024EF9BF026EF9BF0C8EF9BF0010120EEEA
:1036500001F0F651D926F751DA22410EDE18D8A42E
:1036600034EF9BF036EF9BF0C8EF9BF020EE02F0BA
:10367000F651D926F751DA22560EDE18D8A443EFB8
:103680009BF045EF9BF0C8EF9BF020EE03F0F65166
:10369000D926F751DA223D0EDE18D8A452EF9BF05E
:1036A00054EF9BF0C8EF9BF020EE06F0F651D926C0
:1036B000F751DA22DF50D8A460EF9BF062EF9BF065
:1036C000C8EF9BF0D00EE66FFF0EE76F20EE04F020
:1036D000F651D926F751DA22DF50E86FE96BE6514F
:1036E000E827E751E923E95107E10A0EE85DD8B080
:1036F0007CEF9BF07EEF9BF0B9EF9BF0D00EE66F76
:10370000FF0EE76F20EE05F0F651D926F751DA22C9
:10371000DF50E86FE96BE651E827E751E923E9510B
:1037200007E10A0EE85DD8B098EF9BF09AEF9BF0A6
:10373000B9EF9BF020EE04F0F651D926F751DA22CA
:10374000DF50FC6FFC51D00F0A0D6F00CCFFF3F07F
:1037500020EE05F0F651D926F751DA22DF50FC6F42
:103760000001F3510101FC25D00F0001F36FC3EFFD
:103770009BF0000E0001F36F9D0E0101006FFC0E27
:10378000016F36ECD5F0000E0101F66F000EF76FF9
:103790006000DBF7D9FF6000DFF7DAFF520EDE18BA
:1037A000D8A4D5EF9BF0D7EF9BF03DEF9CF0010143
:1037B00020EE01F0F651D926F751DA22450EDE1837
:1037C000D8A4E5EF9BF0E7EF9BF03DEF9CF020EEF7
:1037D00002F0F651D926F751DA22530EDE18D8A49A
:1037E000F4EF9BF0F6EF9BF03DEF9CF020EE03F042
:1037F000F651D926F751DA22450EDE18D8A403EF88
:103800009CF005EF9CF03DEF9CF020EE04F0F651AB
:10381000D926F751DA22540EDE18D8A412EF9CF004
:1038200014EF9CF03DEF9CF0F6C100F1F7C101F1FF
:10383000DAECD4F0050E010100190111D8A423EF30
:103840009CF025EF9CF038EF9CF0430E006FFE0ECD
:10385000016F36ECD5F0000E0101F66F000EF76F28
:103860003F013E9F040E7CECD4F0BC90BC92FF0064
:10387000000E0101F66F000EF76F6000DBF7D9FF55
:103880006000DFF7DAFF4D0EDE18D8A44AEF9CF097
:103890004CEF9CF060EF9CF0BC803F013E8FA08E0F
:1038A000000E0001FE6F000EFD6F000E0201636F3F
:1038B000000E626FAC8E000E0101F66F000EF76F06
:1038C0006000DBF7D9FF6000DFF7DAFF410EDE189A
:1038D000D8A46DEF9CF06FEF9CF079EF9CF0BC905A
:1038E0003F013E9FA09EAC9E000E0101F66F000EB0
:1038F000F76F6000DBF7D9FF6000DFF7DAFF520EE9
:10390000DE18D8A486EF9CF088EF9CF0BAEF9CF00C
:10391000010120EE01F0F651D926F751DA22410ECD
:10392000DE18D8A496EF9CF098EF9CF0BAEF9CF0CC
:1039300020EE02F0F651D926F751DA225A0EDE189F
:10394000D8A4A5EF9CF0A7EF9CF0BAEF9CF0000E76
:103950000201536F000E526F000E0001DB6F000E6C
:10396000DA6F000ED96F000ED86F000E0101F66FEE
:10397000000EF76F1200600E3901D96F000EDB6F79
:10398000000EDD6F080EDF6F000EDE6F290E0101E5
:10399000ED6F960EEC6F7F0EE82EFED7EC2FFCD766
:1039A000ED2FFAD78CECCAF0000E3901C16FBC9034
:1039B000BC9282ECD6F0090E0101ED6F1E0EEC6F89
:1039C000E40EE82EFED7EC2FFCD7ED2FFAD700F04F
:1039D0008A0E3D01F56F090E0101ED6F1E0EEC6FB1
:1039E000E40EE82EFED7EC2FFCD7ED2FFAD700F02F
:1039F0009CECD9F0000E0101FB6F000EFA6F000E77
:103A0000FA25D96E040EFB21DA6E000EDF6EFA4B3A
:103A1000FB2BFB5109E1800EFA5DD8A012EF9DF05F
:103A200014EF9DF0FFEF9CF0000EFB6F000EFA6F9D
:103A3000800EFA25D96E040EFB21DA6E000EDF6EC1
:103A4000FA4BFB2BFB5109E1800EFA5DD8A02BEF5E
:103A50009DF02DEF9DF018EF9DF0000EFB6F000E16
:103A6000FA6F300EFA25D96E030EFB21DA6E000EC6
:103A7000DF6EFA4BFB2BFB5109E17F0EFA5DD8A0FC
:103A800044EF9DF046EF9DF031EF9DF0000EF86F92
:103A9000040EF96F9CECD9F0B40E0101006FFE0E1C
:103AA000016F36ECD5F0000E0101FB6F000EFA6FCE
:103AB000D890FA35D96EFB35DA6ED20ED926020EC1
:103AC000DA226F0078FF00F16F0074FF01F136EC2D
:103AD000D5F00101FA4BFB2BFB5109E1090EFA5D10
:103AE000D8A075EF9DF077EF9DF058EF9DF09CEC1E
:103AF000D9F0F8C1C9F1F9C1CAF1D40E0101CB6FF7
:103B0000FB0ECC6F910ECD6FFF0ECE6FBB0ECF6F45
:103B1000FF0ED06F090ED26F380ED16FE2ECD5F0E8
:103B2000F8C100F1F9C101F1B4ECD1F09CECD9F08D
:103B3000000E0101FB6F000EFA6FBA78290E010129
:103B4000ED6F960EEC6F7F0EE82EFED7EC2FFCD7B4
:103B5000ED2FFAD70101FA4BFB2BFB5109E1080EBF
:103B6000FA5DD8A0B6EF9DF0B8EF9DF09DEF9DF007
:103B7000000E0001FE6F000EFD6F880E0101006F48
:103B8000FE0E016F36ECD5F094ECDAF0770E010101
:103B9000006FFC0E016F36ECD5F02BECB3F0270E66
:103BA0000101FD6F000EFF6F140EFE6F300EC96F26
:103BB000030ECA6F470ECB6FFD0ECC6FFDC1CDF16A
:103BC000CE6BFDC1CFF1D06BE2ECD5F0300E010130
:103BD000006F030E016FB4ECD1F03D017589490E01
:103BE0000101006FFB0E016F36ECD5F03D01738FC4
:103BF00043ECC0F09CECD9F0010E96ECCFF05A0EDD
:103C00000101006FFE0E016F36ECD5F04BECD4F0E5
:103C10003901909F000E3A01866F010E556F000E1C
:103C2000566F000E576F3901A09F0001EF9F3901B9
:103C3000A1919181D28E9CECD9F0BE0E0101006F52
:103C4000FD0E016F36ECD5F05EECDAF0000E0001EF
:103C5000E36F000EE26F3E01F88100F000F03E01DC
:103C6000F8B135EF9EF037EF9EF02FEF9EF06F002A
:103C7000C0FB5BF05C6A5B500101EC6F3E01EF51F1
:103C80000001DE6FECC1DFF0DEC007F1DFC008F13C
:103C90000101096B0A6B000E7CECB8F007C115F14D
:103CA00008C116F109C117F10AC118F16F0E01011F
:103CB000196F120E1A6F830E1B6F3A0E1C6FB1EC48
:103CC000A5F015C1CCF016C1CDF017C1CEF018C1CA
:103CD000CFF0300E0101C96F030ECA6FD90ECB6F42
:103CE000FD0ECC6FDEC0CDF1DFC0CEF1CCC0CFF188
:103CF000CDC0D0F1CEC0D1F1CFC0D2F1E2ECD5F041
:103D0000300E0101006F030E016FB4ECD1F0010E13
:103D10007CECD4F00001E24BE32BE35109E1040E0B
:103D2000E25DD8A096EF9EF098EF9EF02BEF9EF00C
:103D3000000E0101F86F040EF96F000E0401006F10
:103D4000690E0101006FFF0E016F36ECD5F0C90E50
:103D50000101006FFE0E016F36ECD5F004ECBBF0F4
:103D6000010E0201576FA40E566F480E0001F96F45
:103D7000030EFA6F000EFB6F000EFC6F3F013E9FBB
:103D8000010120EE02F0F451D926F551DA22DF507C
:103D90003F013D6F010120EE01F0F451D926F551AC
:103DA000DA22DF503F013C6F6000D3F7D9FF60009B
:103DB000D7F7DAFFDF503B6F3E8FBC80020E96ECE8
:103DC000CFF0090E0101ED6F1E0EEC6FE40EE82E30
:103DD000FED7EC2FFCD7ED2FFAD700F0020E000132
:103DE000F36F5DECD6F0AC8E290E0101ED6F960EEF
:103DF000EC6F7F0EE82EFED7EC2FFCD7ED2FFAD715
:103E0000AC9E300E0101C96F030ECA6F870ECB6FD7
:103E1000FA0ECC6FE0C0CDF1E1C0CEF1E2ECD5F00E
:103E2000300E0101006F030E016FB4ECD1F0670E8C
:103E30000101006FFD0E016F36ECD5F0B90E0101E6
:103E4000006FFA0E016F36ECD5F0750E0101006FB0
:103E5000F80E016F36ECD5F0010E0001EB6FBC924D
:103E6000D1ECD8F09DECC1F0BCA039EF9FF03BEF56
:103E70009FF086EFA0F00001EB05D8A442EF9FF081
:103E800044EF9FF003EFA0F0DC51DE1909E1DD51B2
:103E9000DF19D8B44EEF9FF050EF9FF086EFA0F0FF
:103EA000DEC0DCF0DFC0DDF0BC92000EEE6FBC8047
:103EB000C80EDE255B6E000EDF215C6E5BC007F175
:103EC0005CC008F10101096B0A6B000E7CECB8F0D4
:103ED00007C1D0F008C1D1F009C1D2F00AC1D3F0B6
:103EE0005D50040DEE0EF324F66EF50EF420F76E21
:103EF000F86A000EF82209006F00D4FF32F10900C1
:103F00006F00D4FF33F109006F00D4FF34F10A00D1
:103F10006F00D4FF35F1000E0101196F000E1A6F0A
:103F2000000E1B6F4A0E1C6FD0C015F1D1C016F1E8
:103F3000D2C017F1D3C018F1B1ECA5F015C12EF124
:103F400016C12FF117C130F118C131F100ECAAF000
:103F50002EC147F12FC148F130C149F131C14AF1B9
:103F600090ECC3F047C1F9F048C1FAF049C1FBF049
:103F70004AC1FCF0020E0001F319D8A4C2EF9FF071
:103F8000C4EF9FF0E2EF9FF0300E0101C96F030E06
:103F9000CA6F520ECB6FFA0ECC6F5BC0CDF15CC016
:103FA000CEF1F9C0CFF1FAC0D0F1FBC0D1F1FCC025
:103FB000D2F1E2ECD5F0300E0101006F030E016F7B
:103FC000B4ECD1F03F013E9F010120EE02F0F4512C
:103FD000D926F551DA22DF503F013D6F010120EE75
:103FE00001F0F451D926F551DA22DF503F013C6F40
:103FF0006000D3F7D9FF6000D7F7DAFFDF503B6FDF
:104000003E8F86EFA0F0000E01012E6F000E2F6F85
:10401000C60E306F420E316FD0C032F1D1C033F1D5
:10402000D2C034F1D3C035F114ECC4F00101D8B0E2
:104030001CEFA0F01EEFA0F086EFA0F05D50040D85
:10404000EE0EF324F66EF50EF420F76EF86A000E0D
:10405000F82209006F00D4FF32F109006F00D4FF8D
:1040600033F109006F00D4FF34F10A006F00D4FF70
:1040700035F1000E196F000E1A6F000E1B6F4A0EFD
:104080001C6FD0C015F1D1C016F1D2C017F1D3C04A
:1040900018F1B1ECA5F015C12EF116C12FF117C121
:1040A00030F118C131F100ECAAF02EC147F12FC157
:1040B00048F130C149F131C14AF190ECC3F047C138
:1040C000F9F048C1FAF049C1FBF04AC1FCF03F01E8
:1040D0003E9F010120EE02F0F451D926F551DA227B
:1040E000DF503F013D6F010120EE01F0F451D92670
:1040F000F551DA22DF503F013C6F6000D3F7D9FF62
:104100006000D7F7DAFFDF503B6F3E8F020E0001F1
:10411000F319D8A48EEFA0F090EFA0F0EAEFA0F092
:10412000FD51FE11D8B497EFA0F099EFA0F0B8EFD1
:10413000A0F0FDC002F1FEC003F1030E0101016F0A
:10414000E80E006F79ECD1F0010100C107F101C167
:1041500008F1096B0A6B000E7CECB8F007C1CCF0DB
:1041600008C1CDF009C1CEF00AC1CFF0C0EFA0F078
:10417000000ECC6F000ECD6F000ECE6F000ECF6F15
:10418000300E0101C96F030ECA6FDF0ECB6FF90E3F
:10419000CC6FD0C0CDF1D1C0CEF1D2C0CFF1D3C061
:1041A000D0F1DAC0D1F1DBC0D2F1FDC0D3F1FEC055
:1041B000D4F1CCC0D5F1CDC0D6F1CEC0D7F1CFC0AF
:1041C000D8F1E2ECD5F0300E0101006F030E016F63
:1041D000B4ECD1F0E8EC97F030EF9FF057EF00F03F
:1041E00001010351800B0C6F035103250E6F02AFC9
:1041F000FCEFA0F0FEEFA0F0FFEFA0F00E810E515B
:10420000D8B405EFA1F007EFA1F01CEFA1F00E2943
:10421000D8A40DEFA1F00FEFA1F017EFA1F0000E61
:10422000006F000E016F000E026F000E036F028F11
:10423000000E036F24EFA1F0000E006F000E016F5F
:10424000000E026F000E036F0751800B0D6F0C51B3
:104250000D19D8B42EEFA1F030EFA1F031EFA1F09D
:104260000C8D075107250D6F06AF39EFA1F03BEF1D
:10427000A1F03CEFA1F00D810D51D8B442EFA1F0B7
:1042800044EFA1F059EFA1F00D29D8A44AEFA1F015
:104290004CEFA1F054EFA1F0000E046F000E056F7B
:1042A000000E066F000E076F068F000E076F61EF9E
:1042B000A1F0000E046F000E056F000E066F000ED9
:1042C000076F0E510D5DD8B068EFA1F06AEFA1F055
:1042D00091EFA1F00CAD6FEFA1F071EFA1F073EFD2
:1042E000A1F0800E0C1B0EC10FF10DC10EF10FC11C
:1042F0000DF100C10FF104C100F10FC104F101C1C2
:104300000FF105C101F10FC105F102C10FF106C1A5
:1043100002F10FC106F103C10FF107C103F10FC193
:1043200007F1000E0F6F0E510DC108F1096B085F08
:10433000000E095B09BFA6EFA1F0095109E11A0EB1
:10434000085DD8A0A6EFA1F0A8EFA1F0DFEFA1F0E3
:104350000051011102110311D8A4B1EFA1F0B4EF83
:10436000A1F0010EB5EFA1F0000E0F6F000E006F6F
:10437000000E016F000E026F000E036F0DC10EF1F3
:10438000E8EFA1F00FA1C7EFA1F0C9EFA1F0CFEFC7
:10439000A1F0D8900F3101090F6FD1EFA1F0D890A3
:1043A0000F3300A1D6EFA1F0D8EFA1F0D9EFA1F023
:1043B0000F8F033503330233013300330E2B0D51BE
:1043C0000E5DD8A0E6EFA1F0E8EFA1F0C2EFA1F0FA
:1043D0000CBDEDEFA1F0EFEFA1F02FEFA2F00E5129
:1043E000D8A4F5EFA1F0F7EFA1F001EFA2F0000ED5
:1043F000006F000E016F000E026F000E036F50EF92
:10440000A3F004510027055101230651022307514F
:10441000032303A10EEFA2F010EFA2F0BCEFA2F075
:104420000FA115EFA2F017EFA2F01DEFA2F0D890A8
:104430000F3101090F6F1FEFA2F0D8900F3300A1C9
:1044400024EFA2F026EFA2F027EFA2F00F8F0335A2
:1044500003330233013300330E2BBCEFA2F00451BF
:10446000005D05510159065102590351800A086F38
:104470000751800A0859D8B040EFA2F042EFA2F0ED
:104480006DEFA2F00051045D086F01510559096FED
:10449000025106590A6F035107590B6FFF0E082589
:1044A000006FFF0E0921016FFF0E0A21026FFF0E40
:1044B0000B21036F800E0C1B0F6D0F51D8A463EFFF
:1044C000A2F065EFA2F075EFA2F0010E0027000E3A
:1044D00001230223032375EFA2F00451005F05516D
:1044E000015B0651025B0751035B00510111021190
:1044F0000311D8A47EEFA2F080EFA2F0B5EFA2F0F6
:104500000F51D8A486EFA2F088EFA2F0B5EFA2F089
:10451000000E006F000E016F000E026F000E036FA1
:1045200050EFA3F0D89000370137023703370FAFB1
:104530009CEFA2F09EEFA2F09FEFA2F000810FA1EE
:10454000A4EFA2F0A6EFA2F0AAEFA2F0D8800F3756
:10455000ACEFA2F0D8900F370E51D8B4B2EFA2F062
:10456000B4EFA2F0B5EFA2F00E0702AFBAEFA2F0DF
:10457000BCEFA2F092EFA2F0000E0D6F0FAFC3EFF1
:10458000A2F0C5EFA2F0DDEFA2F00FC108F17F0E9F
:104590000817D8B4CEEFA2F0D0EFA2F0D4EFA2F07B
:1045A000010E0D6FDDEFA2F000A1D9EFA2F0DBEF5D
:1045B000A2F0DDEFA2F0D0EFA2F00D51D8B4E3EFFE
:1045C000A2F0E5EFA2F010EFA3F0010E0027000E1D
:1045D00001230223032303A1F0EFA2F0F2EFA2F0E4
:1045E00010EFA3F000C108F101C109F102C10AF105
:1045F00003C10BF10B350B330A330933083308C100
:1046000000F109C101F10AC102F10BC103F10E2948
:10461000D8B40DEFA3F00FEFA3F010EFA3F00E2B23
:104620000E29D8B416EFA3F018EFA3F020EFA3F0F3
:104630000E51D8A41EEFA3F020EFA3F032EFA3F0A9
:10464000000E006F000E016F000E026F000E036F70
:104650000E51D8A42EEFA3F030EFA3F032EFA3F069
:10466000000E0C6F0EA137EFA3F039EFA3F03CEF73
:10467000A3F0028F3DEFA3F0029FD8900E31036F9D
:104680000CAF45EFA3F047EFA3F048EFA3F0038F83
:1046900000C100F101C101F102C102F103C103F146
:1046A00012000450800B0D6E045004240F6E03AEF4
:1046B0005CEFA3F05EEFA3F05FEFA3F00F800F506D
:1046C000D8B465EFA3F067EFA3F07CEFA3F00F2859
:1046D000D8A46DEFA3F06FEFA3F077EFA3F0000E77
:1046E000016E000E026E000E036E000E046E038E4D
:1046F000000E046E84EFA3F0000E016E000E026E39
:10470000000E036E000E046E0850800B0E6E0D50EE
:104710000E18D8B48EEFA3F090EFA3F091EFA3F0B2
:104720000D8C085008240E6E07AE99EFA3F09BEF96
:10473000A3F09CEFA3F00E800E50D8B4A2EFA3F02C
:10474000A4EFA3F0B9EFA3F00E28D8A4AAEFA3F02A
:10475000ACEFA3F0B4EFA3F0000E056E000E066EF2
:10476000000E076E000E086E078E000E086EC1EF79
:10477000A3F0000E056E000E066E000E076E000E12
:10478000086E0F500E5CD8B0C8EFA3F0CAEFA3F0CC
:10479000F1EFA3F00DACCFEFA3F0D1EFA3F0D3EF87
:1047A000A3F0800E0D1A0FC010F00EC00FF010C055
:1047B0000EF001C010F005C001F010C005F002C0FD
:1047C00010F006C002F010C006F003C010F007C0E1
:1047D00003F010C007F004C010F008C004F010C0CF
:1047E00008F0000E106E0F500EC009F00A6A095E44
:1047F000000E0A5A0ABE06EFA4F00A5009E11A0E8A
:10480000095CD8A006EFA4F008EFA4F03FEFA4F0F5
:104810000150021003100410D8A411EFA4F014EFFB
:10482000A4F0010E15EFA4F0000E106E000E016E44
:10483000000E026E000E036E000E046E0EC00FF02E
:1048400048EFA4F010A027EFA4F029EFA4F02FEF79
:10485000A4F0D89010300109106E31EFA4F0D89078
:10486000103201A036EFA4F038EFA4F039EFA4F035
:10487000108E043404320332023201320F2A0E50F9
:104880000F5CD8A046EFA4F048EFA4F022EFA4F00C
:104890000DBC4DEFA4F04FEFA4F08FEFA4F00F503C
:1048A000D8A455EFA4F057EFA4F061EFA4F0000EE8
:1048B000016E000E026E000E036E000E046EB0EF6D
:1048C000A5F0055001260650022207500322085089
:1048D000042204A06EEFA4F070EFA4F01CEFA5F08A
:1048E00010A075EFA4F077EFA4F07DEFA4F0D890BE
:1048F00010300109106E7FEFA4F0D890103201A0A3
:1049000084EFA4F086EFA4F087EFA4F0108E0434B7
:1049100004320332023201320F2A1CEFA5F0055097
:10492000015C06500258075003580450800A096E73
:104930000850800A0958D8B0A0EFA4F0A2EFA4F064
:10494000CDEFA4F00150055C096E025006580A6EC6
:10495000035007580B6E045008580C6EFF0E0924C4
:10496000016EFF0E0A20026EFF0E0B20036EFF0E7B
:104970000C20046E800E0D1A106C1050D8A4C3EFDA
:10498000A4F0C5EFA4F0D5EFA4F0010E0126000EAF
:10499000022203220422D5EFA4F00550015E065046
:1049A000025A0750035A0850045A015002100310CB
:1049B0000410D8A4DEEFA4F0E0EFA4F015EFA5F00A
:1049C0001050D8A4E6EFA4F0E8EFA4F015EFA5F09E
:1049D000000E016E000E026E000E036E000E046EDD
:1049E000B0EFA5F0D890013602360336043610AE8B
:1049F000FCEFA4F0FEEFA4F0FFEFA4F0018010A004
:104A000004EFA5F006EFA5F00AEFA5F0D880103668
:104A10000CEFA5F0D89010360F50D8B412EFA5F0D7
:104A200014EFA5F015EFA5F00F0603AE1AEFA5F0F1
:104A30001CEFA5F0F2EFA4F0000E0E6E10AE23EF07
:104A4000A5F025EFA5F03DEFA5F010C009F07F0E11
:104A50000916D8B42EEFA5F030EFA5F034EFA5F08D
:104A6000010E0E6E3DEFA5F001A039EFA5F03BEF72
:104A7000A5F03DEFA5F030EFA5F00E50D8B443EF10
:104A8000A5F045EFA5F070EFA5F0010E0126000E90
:104A900002220322042204A050EFA5F052EFA5F059
:104AA00070EFA5F001C009F002C00AF003C00BF0DE
:104AB00004C00CF00C340C320B320A32093209C03B
:104AC00001F00AC002F00BC003F00CC004F00F2884
:104AD000D8B46DEFA5F06FEFA5F070EFA5F00F2A39
:104AE0000F28D8B476EFA5F078EFA5F080EFA5F009
:104AF0000F50D8A47EEFA5F080EFA5F092EFA5F0BF
:104B0000000E016E000E026E000E036E000E046EAB
:104B10000F50D8A48EEFA5F090EFA5F092EFA5F07E
:104B2000000E0D6E0FA097EFA5F099EFA5F09CEF8A
:104B3000A5F0038E9DEFA5F0039ED8900F30046E74
:104B40000DAEA5EFA5F0A7EFA5F0A8EFA5F0048E98
:104B500001C001F002C002F003C003F004C004F081
:104B6000120001011851800B216F18511825276F71
:104B700017AFBDEFA5F0BFEFA5F0C0EFA5F02781FF
:104B80002751D8B4C6EFA5F0C8EFA5F0DBEFA5F02C
:104B90002729D8A4CEEFA5F0D0EFA5F0D8EFA5F047
:104BA000000E156F000E166F000E176F000E186FB7
:104BB000178FE3EFA5F0000E156F000E166F000EB5
:104BC000176F000E186F1C51800B211B1C511C25E8
:104BD000266F1BAFEEEFA5F0F0EFA5F0F1EFA5F01B
:104BE00026812651D8B4F7EFA5F0F9EFA5F00CEF28
:104BF000A6F02629D8A4FFEFA5F001EFA6F009EF53
:104C0000A6F0000E196F000E1A6F000E1B6F000E3B
:104C10001C6F1B8F14EFA6F0000E196F000E1A6F99
:104C2000000E1B6F000E1C6F2651D8B41AEFA6F0B1
:104C30001CEFA6F024EFA6F02751D8A422EFA6F08F
:104C400024EFA6F02EEFA6F0000E156F000E166FE3
:104C5000000E176F000E186FD8EFA7F01B51150349
:104C60006F00CCFF2CF16F00D0FF2DF12C51226F83
:104C7000236B246B256B2D51286F296B2A6B2B6BB3
:104C80001A5116036F00CCFF2CF16F00D0FF2DF1ED
:104C90002C512227000E2323242325232D5128279E
:104CA000000E29232A232B23195117036F00CCFF51
:104CB0002CF16F00D0FF2DF12C512227000E232361
:104CC000242325232D512827000E29232A232B2393
:104CD00024C125F123C124F122C123F1226B1951F2
:104CE00016036F00CCFF2CF16F00D0FF2DF12C517B
:104CF00022272D512323000E2423000E25231A5191
:104D000015036F00CCFF2CF16F00D0FF2DF12C515B
:104D100022272D512323000E2423000E252324C1F6
:104D200025F123C124F122C123F1226B195115036E
:104D30006F00CCFF2CF16F00D0FF2DF12C512227FA
:104D40002D512323000E2423000E25231B5116036F
:104D50006F00CCFF2CF16F00D0FF2DF12C512827D4
:104D60002D512923000E2A23000E2B231A5117033D
:104D70006F00CCFF2CF16F00D0FF2DF12C512827B4
:104D80002D512923000E2A23000E2B231B5117031C
:104D90006F00CCFF2CF16F00D0FF2DF12C511D6F57
:104DA0002D511E6F1F6B206B1FC120F11EC11FF103
:104DB0001DC11EF11D6B1D5128271E5129231F5196
:104DC0002A2320512B2322C11DF123C11EF124C10E
:104DD0001FF125C120F1190EF3EFA6F0D890203372
:104DE0001F331E331D33E82EEEEFA6F01D5128278A
:104DF0001E5129231F512A2320512B2324C125F181
:104E000023C124F122C123F1226B265127C11DF1B8
:104E10001E6B1D27000E1E23820E1D252C6FFF0EFC
:104E20001E212D6F29EFA7F0D890283729372A3770
:104E30002B3725AF1EEFA7F020EFA7F021EFA7F04B
:104E40002881D89022372337243725372C07D8A03C
:104E50002D072AAF2EEFA7F030EFA7F014EFA7F041
:104E6000000E266F25AF37EFA7F039EFA7F05DEF03
:104E7000A7F0FF0E22151D6FFF0E23151E6FFF0EEC
:104E800024151F6F7F0E2515206F1D511E111F1138
:104E90002011D8B44EEFA7F050EFA7F054EFA7F0D1
:104EA000010E266F5DEFA7F028A159EFA7F05BEF89
:104EB000A7F05DEFA7F050EFA7F02651D8B463EF4D
:104EC000A7F065EFA7F089EFA7F0010E2827000EE5
:104ED00029232A232B232BA170EFA7F072EFA7F031
:104EE00089EFA7F028C11DF129C11EF12AC11FF1C8
:104EF0002BC120F1203520331F331E331D331DC13C
:104F000028F11EC129F11FC12AF120C12BF12C4B20
:104F10002D2B2DBF94EFA7F02D5108E12C29D8A0FF
:104F200094EFA7F096EFA7F0A0EFA7F0000E286F80
:104F3000000E296F800E2A6F7F0E2B6FCEEFA7F029
:104F40002DBFADEFA7F02D5106E12C05D8B0ABEF8A
:104F5000A7F0ADEFA7F0B9EFA7F0000E286F000E95
:104F6000296F000E2A6F000E2B6F000E216FCEEFFF
:104F7000A7F02CC127F1FF0E2817FF0E29177F0E6F
:104F80002A17000E2B1727A1C8EFA7F0CAEFA7F02A
:104F9000CBEFA7F02A8FD89027312B6F21512B13FD
:104FA00028C115F129C116F12AC117F12BC118F139
:104FB00012000450800B0D6E04500424136E03AED7
:104FC000E4EFA7F0E6EFA7F0E7EFA7F013801350A8
:104FD000D8B4EDEFA7F0EFEFA7F002EFA8F0132899
:104FE000D8A4F5EFA7F0F7EFA7F0FFEFA7F0000EBA
:104FF000016E000E026E000E036E000E046E038E34
:105000000AEFA8F0000E016E000E026E000E036E95
:10501000000E046E0850800B0D1A08500824126E02
:1050200007AE15EFA8F017EFA8F018EFA8F0128060
:105030001250D8B41EEFA8F020EFA8F033EFA8F07C
:105040001228D8A426EFA8F028EFA8F030EFA8F097
:10505000000E056E000E066E000E076E000E086E46
:10506000078E3BEFA8F0000E056E000E066E000ED8
:10507000076E000E086E1250D8B441EFA8F043EF4F
:10508000A8F04BEFA8F01350D8A449EFA8F04BEFCD
:10509000A8F055EFA8F0000E016E000E026E000E93
:1050A000036E000E046EFFEFA9F0075001026F00BF
:1050B000CCFF18F06F00D0FF19F018500E6E0F6A79
:1050C000106A116A1950146E156A166A176A06502A
:1050D00002026F00CCFF18F06F00D0FF19F01850DB
:1050E0000E26000E0F221022112219501426000E37
:1050F000152216221722055003026F00CCFF18F06C
:105100006F00D0FF19F018500E26000E0F2210224B
:10511000112219501426000E15221622172210C033
:1051200011F00FC010F00EC00FF00E6A0550020211
:105130006F00CCFF18F06F00D0FF19F018500E264A
:1051400019500F22000E1022000E112206500102EB
:105150006F00CCFF18F06F00D0FF19F018500E262A
:1051600019500F22000E1022000E112210C011F053
:105170000FC010F00EC00FF00E6A055001026F0054
:10518000CCFF18F06F00D0FF19F018500E26195000
:105190000F22000E1022000E1122075002026F0093
:1051A000CCFF18F06F00D0FF19F0185014261950DA
:1051B0001522000E1622000E1722065003026F0061
:1051C000CCFF18F06F00D0FF19F0185014261950BA
:1051D0001522000E1622000E1722075003026F0040
:1051E000CCFF18F06F00D0FF19F01850096E19505D
:1051F0000A6E0B6A0C6A0BC00CF00AC00BF009C0F7
:105200000AF0096A095014260A5015220B5016227A
:105210000C5017220EC009F00FC00AF010C00BF09E
:1052200011C00CF0190E1AEFA9F0D8900C320B3205
:105230000A320932E82E15EFA9F0095014260A5057
:1052400015220B5016220C50172210C011F00FC05F
:1052500010F00EC00FF00E6A125013C009F00A6A67
:105260000926000E0A22820E0924186EFF0E0A205B
:10527000196E50EFA9F0D890143615361636173639
:1052800011AE45EFA9F047EFA9F048EFA9F014805F
:10529000D8900E360F36103611361806D8A01906DB
:1052A00016AE55EFA9F057EFA9F03BEFA9F0000EAD
:1052B000126E11AE5EEFA9F060EFA9F084EFA9F0D5
:1052C000FF0E0E14096EFF0E0F140A6EFF0E10145F
:1052D0000B6E7F0E11140C6E09500A100B100C107F
:1052E000D8B475EFA9F077EFA9F07BEFA9F0010E24
:1052F000126E84EFA9F014A080EFA9F082EFA9F05C
:1053000084EFA9F077EFA9F01250D8B48AEFA9F092
:105310008CEFA9F0B0EFA9F0010E1426000E1522B3
:105320001622172217A097EFA9F099EFA9F0B0EF76
:10533000A9F014C009F015C00AF016C00BF017C090
:105340000CF00C340C320B320A32093209C014F062
:105350000AC015F00BC016F00CC017F0184A192A35
:1053600019BEBBEFA9F0195008E11828D8A0BBEF6F
:10537000A9F0BDEFA9F0C7EFA9F0000E146E000E62
:10538000156E800E166E7F0E176EF5EFA9F019BE22
:10539000D4EFA9F0195006E11804D8B0D2EFA9F063
:1053A000D4EFA9F0E0EFA9F0000E146E000E156E18
:1053B000000E166E000E176E000E0D6EF5EFA9F0C2
:1053C00018C013F0FF0E1416FF0E15167F0E1616DA
:1053D000000E171613A0EFEFA9F0F1EFA9F0F2EF0E
:1053E000A9F0168ED8901330176E0D50171214C0F6
:1053F00001F015C002F016C003F017C004F012004F
:1054000001013151800B3E6F31513125456F30AF75
:105410000CEFAAF00EEFAAF00FEFAAF0458145516C
:10542000D8B415EFAAF017EFAAF02CEFAAF045298F
:10543000D8A41DEFAAF01FEFAAF027EFAAF0000EE4
:105440002E6F000E2F6F000E306F000E316F308FF9
:10545000000E316F34EFAAF0000E2E6F000E2F6F8A
:10546000000E306F000E316F3551800B3E1B3551F1
:105470003525466F34AF3FEFAAF041EFAAF042EF77
:10548000AAF046814651D8B448EFAAF04AEFAAF0F4
:105490005FEFAAF04629D8A450EFAAF052EFAAF085
:1054A0005AEFAAF0000E326F000E336F000E346F09
:1054B000000E356F348F000E356F67EFAAF0000EC7
:1054C000326F000E336F000E346F000E356F3251A5
:1054D000331134113511D8A470EFAAF072EFAAF08D
:1054E0008AEFAAF0000E2E6F000E2F6F000E306FA5
:1054F000000E316F800E30137F0E31133E51311389
:105500002EC12EF12FC12FF130C130F131C131F157
:10551000CDEFABF04551D8A490EFAAF092EFAAF0EE
:105520009CEFAAF0000E2E6F000E2F6F000E306F52
:10553000000E316FCDEFABF0465145C136F1376B00
:10554000365F000E375B7F0E36253F6F000E37212A
:10555000406F2EC13AF12FC13BF130C13CF131C156
:105560003DF1000E2E6F000E2F6F000E306F000EFB
:10557000316F000E416F000E426F000E436F000E40
:10558000446F000E466FFDEFAAF04651D8B4CBEF42
:10559000AAF0CDEFAAF0E4EFAAF0D8903A373B3763
:1055A0003C373D37D8902E372F373037313744AF1F
:1055B000DCEFAAF0DEEFAAF0DFEFAAF02E81D890A0
:1055C000413742374337443732513A5D33513B59C3
:1055D00034513C5935513D59D8A0F1EFAAF0F3EFC1
:1055E000AAF0FCEFAAF0448D32513A5F33513B5B95
:1055F00034513C5B35513D5B462B190E466503EF3C
:10560000ABF005EFABF0C5EFAAF03A513B113C11FE
:105610003D11D8B40EEFABF010EFABF028EFABF0CC
:10562000418128EFABF0D8902E372F373037313704
:1056300044AF1DEFABF01FEFABF020EFABF02E81CE
:10564000D89041374237433744373F07D8A0400707
:1056500030AF2DEFABF02FEFABF013EFABF0000E50
:10566000466F44AF36EFABF038EFABF05CEFABF02A
:10567000FF0E4115366FFF0E4215376FFF0E4315B3
:10568000386F7F0E4415396F365137113811391183
:10569000D8B44DEFABF04FEFABF053EFABF0010EE2
:1056A000466F5CEFABF02EA158EFABF05AEFABF0CA
:1056B0005CEFABF04FEFABF04651D8B462EFABF01C
:1056C00064EFABF088EFABF0010E2E27000E2F2316
:1056D0003023312331A16FEFABF071EFABF088EFE6
:1056E000ABF02EC136F12FC137F130C138F131C1E5
:1056F00039F13935393338333733363336C12EF152
:1057000037C12FF138C130F139C131F13F4B402B56
:1057100040BF93EFABF0405108E13F29D8A093EF91
:10572000ABF095EFABF0A0EFABF0000E406F3F6930
:10573000000E2E6F000E2F6F000E306F000E316FB7
:1057400040BFADEFABF0405106E13F05D8B0ABEF45
:10575000ABF0ADEFABF0BBEFABF0000E406F000E67
:105760003F6F000E2E6F000E2F6F000E306F000E79
:10577000316F000E3E6F3FC145F145A1C2EFABF066
:10578000C4EFABF0C7EFABF0308FC8EFABF0309F9A
:10579000D8904531316F7EEFAAF012000450800B93
:1057A000116E04500424186E03AED9EFABF0DBEF9A
:1057B000ABF0DCEFABF018801850D8B4E2EFABF0F0
:1057C000E4EFABF0F9EFABF01828D8A4EAEFABF0B8
:1057D000ECEFABF0F4EFABF0000E016E000E026EDA
:1057E000000E036E000E046E038E000E046E01EFB9
:1057F000ACF0000E016E000E026E000E036E000E85
:10580000046E0850800B111A08500824196E07AE58
:105810000CEFACF00EEFACF00FEFACF019801950BC
:10582000D8B415EFACF017EFACF02CEFACF01928B2
:10583000D8A41DEFACF01FEFACF027EFACF0000EDA
:10584000056E000E066E000E076E000E086E078EC7
:10585000000E086E34EFACF0000E056E000E066E02
:10586000000E076E000E086E055006100710081097
:10587000D8A43DEFACF03FEFACF057EFACF0000E2A
:10588000016E000E026E000E036E000E046E800E9E
:1058900003127F0E04121150041201C001F002C065
:1058A00002F003C003F004C004F09AEFADF018500A
:1058B000D8A45DEFACF05FEFACF069EFACF0000E98
:1058C000016E000E026E000E036E000E046E9AEF63
:1058D000ADF0195018C009F00A6A095E000E0A5AA4
:1058E0007F0E0924126E000E0A20136E01C00DF007
:1058F00002C00EF003C00FF004C010F0000E016EE5
:10590000000E026E000E036E000E046E000E146E8A
:10591000000E156E000E166E000E176E000E196E3C
:10592000CAEFACF01950D8B498EFACF09AEFACF0E5
:10593000B1EFACF0D8900D360E360F361036D89049
:10594000013602360336043617AEA9EFACF0ABEFE2
:10595000ACF0ACEFACF00180D890143615361636AA
:10596000173605500D5C06500E5807500F5808505A
:105970001058D8A0BEEFACF0C0EFACF0C9EFACF05F
:10598000178C05500D5E06500E5A07500F5A0850DE
:10599000105A192A190E1964D0EFACF0D2EFACF0FE
:1059A00092EFACF00D500E100F101010D8B4DBEFCA
:1059B000ACF0DDEFACF0F5EFACF01480F5EFACF04F
:1059C000D890013602360336043617AEEAEFACF053
:1059D000ECEFACF0EDEFACF00180D890143615365A
:1059E000163617361206D8A0130603AEFAEFACF03F
:1059F000FCEFACF0E0EFACF0000E196E17AE03EF69
:105A0000ADF005EFADF029EFADF0FF0E1414096E07
:105A1000FF0E15140A6EFF0E16140B6E7F0E171470
:105A20000C6E09500A100B100C10D8B41AEFADF020
:105A30001CEFADF020EFADF0010E196E29EFADF0C7
:105A400001A025EFADF027EFADF029EFADF01CEF91
:105A5000ADF01950D8B42FEFADF031EFADF055EFF8
:105A6000ADF0010E0126000E02220322042204A042
:105A70003CEFADF03EEFADF055EFADF001C009F0F9
:105A800002C00AF003C00BF004C00CF00C340C325E
:105A90000B320A32093209C001F00AC002F00BC011
:105AA00003F00CC004F0124A132A13BE60EFADF0ED
:105AB000135008E11228D8A060EFADF062EFADF00E
:105AC0006DEFADF0000E136E1268000E016E000E49
:105AD000026E000E036E000E046E13BE7AEFADF080
:105AE000135006E11204D8B078EFADF07AEFADF0C4
:105AF00088EFADF0000E136E000E126E000E016EF8
:105B0000000E026E000E036E000E046E000E116E8B
:105B100012C018F018A08FEFADF091EFADF094EF38
:105B2000ADF0038E95EFADF0039ED8901830046E63
:105B30004BEFACF012001DC135F11EC136F11FC193
:105B400037F120C138F121C139F122C13AF123C125
:105B50003BF124C13CF101013CBFB1EFADF0B4EF2A
:105B6000ADF0010EB5EFADF0000E336F346B335175
:105B70003411D8B4BEEFADF0C0EFADF0D0EFADF062
:105B80003C1F3B1F3A1F391F381F371F361F356D0B
:105B9000000E36233723382339233A233B233C2373
:105BA000F1BFD5EFADF0D7EFADF0D8EFADF0F29398
:105BB000F1BFE5EFADF0F15106E1F005D8B0E3EF4C
:105BC000ADF0E5EFADF0EBEFADF0000E306F010E94
:105BD0002F6FEFEFADF0F0C12FF1F1C130F1EEC159
:105BE00031F1EFC132F133513411D8A4FAEFADF0F5
:105BF000FCEFADF003EFAEF0F2A501EFAEF003EF76
:105C0000AEF006EFAEF03107D8A03207000E3E6FBF
:105C10004F0E3D6F000E0201D16F8CEFAEF03D07CD
:105C2000D8A03E07820E3D25D96E020E3E21DA6EC7
:105C300035C100F136C101F137C102F138C103F1BC
:105C400039C104F13AC105F13BC106F13CC107F18C
:105C50000A0E086F000E096F000E0A6F000E0B6F20
:105C6000000E0C6F000E0D6F000E0E6F000E0F6F0A
:105C7000DEECBEF000C125F101C126F102C127F121
:105C800003C128F104C129F105C12AF106C12BF194
:105C900007C12CF125C112F127C113F1E1ECD7F0B6
:105CA00001011251300FDF6E2F07D8A030073107E6
:105CB000D8A0320735C100F136C101F137C102F178
:105CC00038C103F139C104F13AC105F13BC106F114
:105CD0003CC107F10A0E086F000E096F000E0A6F33
:105CE000000E0B6F000E0C6F000E0D6F000E0E6F8E
:105CF000000E0F6FD5ECBBF000C135F101C136F1DC
:105D000002C137F103C138F104C139F105C13AF1DB
:105D100006C13BF107C13CF101013EBF98EFAEF077
:105D20003E5108E13D05D8A098EFAEF09AEFAEF0F5
:105D3000CAEFAEF0355136113711381139113A1119
:105D40003B113C11D8A4A7EFAEF0A9EFAEF00FEFD6
:105D5000AEF030BFB6EFAEF0305106E12F05D8B04F
:105D6000B4EFAEF0B6EFAEF00FEFAEF032BFC1EF72
:105D7000AEF0325108E13105D8A0C1EFAEF0C3EF6B
:105D8000AEF0CAEFAEF0F2B3C8EFAEF0CAEFAEF0CD
:105D90000FEFAEF033513411D8A4D1EFAEF0D3EF02
:105DA000AEF0DAEFAEF0F2A5D8EFAEF0DAEFAEF08B
:105DB000F9EFAEF03D07D8A03E0733513411D8A417
:105DC000E4EFAEF0E6EFAEF0ECEFAEF0000E2E6FCB
:105DD0002B0E2D6FF0EFAEF0000E2E6F2D0E2D6FEF
:105DE000820E3D25D96E020E3E21DA6E6000B7F4B8
:105DF000DFFF1BC110F11CC111F1820E3D25126F96
:105E0000020E3E21136F31C114F132C115F1F1ECD4
:105E1000CAF010C11BF111C11CF112001EC036F0F6
:105E20001FC037F020C038F021C039F022C03AF04E
:105E300023C03BF024C03CF025C03DF03DBE23EF25
:105E4000AFF026EFAFF0010E27EFAFF0000E346E8B
:105E5000356A34503510D8B430EFAFF032EFAFF0D0
:105E600042EFAFF03D1E3C1E3B1E3A1E391E381E4F
:105E7000371E366C000E3722382239223A223B2256
:105E80003C223D220101F1BF48EFAFF04AEFAFF0F5
:105E90004BEFAFF0F293F1BF58EFAFF0F15106E1E5
:105EA000F005D8B056EFAFF058EFAFF05EEFAFF0BF
:105EB000000E316E010E306E62EFAFF0F0C130F0C7
:105EC000F1C131F0EEC132F0EFC133F03450351092
:105ED000D8A46DEFAFF06FEFAFF076EFAFF0F2A5B3
:105EE00074EFAFF076EFAFF079EFAFF03206D8A0F5
:105EF0003306000E3F6E4F0E3E6E000E0201D16F54
:105F0000FEEFAFF03E06D8A03F06820E3E24D96ECB
:105F1000020E3F20DA6E36C001F037C002F038C002
:105F200003F039C004F03AC005F03BC006F03CC0B5
:105F300007F03DC008F00A0E096E000E0A6E000E52
:105F40000B6E000E0C6E000E0D6E000E0E6E000E2F
:105F50000F6E000E106E91ECBFF001C026F002C073
:105F600027F003C028F004C029F005C02AF006C0BD
:105F70002BF007C02CF008C02DF026C013F028C06D
:105F800014F002ECD8F01350300FDF6E3006D8A0BA
:105F900031063206D8A0330636C001F037C002F011
:105FA00038C003F039C004F03AC005F03BC006F039
:105FB0003CC007F03DC008F00A0E096E000E0A6EE4
:105FC000000E0B6E000E0C6E000E0D6E000E0E6EAF
:105FD000000E0F6E000E106E9AECBCF001C036F091
:105FE00002C037F003C038F004C039F005C03AF001
:105FF00006C03BF007C03CF008C03DF03FBE09EFD3
:10600000B0F03F5008E13E04D8A009EFB0F00BEF2C
:10601000B0F03CEFB0F036503710381039103A106D
:106020003B103C103D10D8A418EFB0F01AEFB0F0C0
:1060300082EFAFF031BE27EFB0F0315006E130040F
:10604000D8B025EFB0F027EFB0F082EFAFF033BE5D
:1060500032EFB0F0335008E13204D8A032EFB0F0A4
:1060600034EFB0F03CEFB0F00101F2B33AEFB0F032
:106070003CEFB0F082EFAFF034503510D8A443EFCE
:10608000B0F045EFB0F04DEFB0F00101F2A54BEFED
:10609000B0F04DEFB0F06CEFB0F03E06D8A03F0688
:1060A00034503510D8A457EFB0F059EFB0F05FEF8F
:1060B000B0F0000E2F6E2B0E2E6E63EFB0F0000EC0
:1060C0002F6E2D0E2E6E820E3E24D96E020E3F20B4
:1060D000DA6E6000BBF0DFFF1CC011F01DC012F0D3
:1060E000820E3E24136E020E3F20146E32C015F055
:1060F00033C016F0B9ECCBF011C01CF012C01DF08B
:1061000012000101F1BF87EFB0F089EFB0F08AEF24
:10611000B0F0F293F1BF97EFB0F0F15106E1F00566
:10612000D8B095EFB0F097EFB0F09DEFB0F0000E63
:106130002F6F010E2E6FA1EFB0F0F0C12EF1F1C163
:106140002FF1EEC130F1EFC131F1F2A9AAEFB0F0B9
:10615000ACEFB0F0B0EFB0F0FE0E3027FF0E312301
:106160001DC132F11EC133F11FC134F120C135F11F
:1061700021C136F122C137F123C138F124C139F1EF
:10618000000E3B6F4F0E3A6F000E0201D16F64EFAD
:10619000B1F03A07D8A03B070F0E32153C6F3D6BAC
:1061A0003DBFDCEFB0F03D5109E10A0E3C5DD8A0E7
:1061B000DCEFB0F0DEEFB0F0E6EFB0F0570E3C25CC
:1061C0003C6F000E3D213D6FECEFB0F0300E3C25F2
:1061D0003C6F000E3D213D6FBF0E266FFF0E276FF7
:1061E0002551286F296B265128272751292329510A
:1061F00007E11A0E285DD8B000EFB1F002EFB1F060
:1062000025EFB1F09F0E266FFF0E276F200E3C1179
:10621000286F000E3D11296F265128272751292369
:10622000295107E11A0E285DD8B019EFB1F01BEF24
:10623000B1F025EFB1F03CC106F13DC107F112EC20
:10624000D7F006C13CF107C13DF1820E01013A25AC
:10625000D96E020E3B21DA6E6000F3F4DFFF2E07E9
:10626000D8A02F073007D8A0310732C126F133C19B
:1062700027F134C128F135C129F136C12AF137C1DE
:106280002BF138C12CF139C12DF1050E51EFB1F0D0
:10629000D8902D332C332B332A332933283327330B
:1062A0002633E82E48EFB1F026C132F127C133F191
:1062B00028C134F129C135F12AC136F12BC137F19A
:1062C0002CC138F12DC139F101013BBF71EFB1F0A3
:1062D0003B5109E1020E3A5DD8A071EFB1F073EFC6
:1062E000B1F0A3EFB1F03251331134113511361141
:1062F000371138113911D8A480EFB1F082EFB1F025
:10630000C9EFB0F02FBF8FEFB1F02F5106E12E058E
:10631000D8B08DEFB1F08FEFB1F0C9EFB0F031BF71
:106320009AEFB1F0315108E13005D8A09AEFB1F001
:106330009CEFB1F0A3EFB1F0F2B3A1EFB1F0A3EF96
:10634000B1F0C9EFB0F0F2A9A8EFB1F0AAEFB1F047
:10635000C1EFB1F03A07D8A03B07820E3A25D96EBB
:10636000020E3B21DA6E600097F4DFFF3A07D8A0F7
:106370003B07820E3A25D96E020E3B21DA6E300EB3
:10638000DF6E1BC110F11CC111F1820E3A25126F94
:10639000020E3B21136F30C114F131C115F1F1EC44
:1063A000CAF010C11BF111C11CF112000101F1BFB3
:1063B000DCEFB1F0DEEFB1F0DFEFB1F0F293F1BF5F
:1063C000ECEFB1F0F15106E1F005D8B0EAEFB1F031
:1063D000ECEFB1F0F2EFB1F0000E306E010E2F6E67
:1063E000F6EFB1F0F0C12FF0F1C130F0EEC131F0B5
:1063F000EFC132F0F2A9FFEFB1F001EFB2F005EF1B
:10640000B2F0FE0E3126FF0E32221EC033F01FC046
:1064100034F020C035F021C036F022C037F023C060
:1064200038F024C039F025C03AF0000E3C6E4F0E13
:106430003B6E000E0201D16FB8EFB2F03B06D8A060
:106440003C060F0E33143D6E3E6A3EBE31EFB2F095
:106450003E5009E10A0E3D5CD8A031EFB2F033EFB7
:10646000B2F03BEFB2F0570E3D243D6E000E3E20E1
:106470003E6E41EFB2F0300E3D243D6E000E3E20E8
:106480003E6EBF0E276EFF0E286E2650296E2A6ABA
:106490002750292628502A222A5007E11A0E295C63
:1064A000D8B055EFB2F057EFB2F07AEFB2F09F0EDE
:1064B000276EFF0E286E200E3D10296E000E3E1036
:1064C0002A6E2750292628502A222A5007E11A0E20
:1064D000295CD8B06EEFB2F070EFB2F07AEFB2F0A4
:1064E0003DC003F03EC004F07BECD7F003C03DF0AC
:1064F00004C03EF0820E3B24D96E020E3C20DA6EC0
:106500006000F7F0DFFF2F06D8A030063106D8A0D4
:10651000320633C027F034C028F035C029F036C029
:106520002AF037C02BF038C02CF039C02DF03AC01B
:106530002EF0050EA5EFB2F0D8902E322D322C326F
:106540002B322A32293228322732E82E9CEFB2F041
:1065500027C033F028C034F029C035F02AC036F007
:106560002BC037F02CC038F02DC039F02EC03AF0D7
:106570003CBEC4EFB2F03C5009E1020E3B5CD8A037
:10658000C4EFB2F0C6EFB2F0F7EFB2F03350341010
:10659000351036103710381039103A10D8A4D3EF10
:1065A000B2F0D5EFB2F01EEFB2F030BEE2EFB2F0D3
:1065B000305006E12F04D8B0E0EFB2F0E2EFB2F0D5
:1065C0001EEFB2F032BEEDEFB2F0325008E131040E
:1065D000D8A0EDEFB2F0EFEFB2F0F7EFB2F00101BB
:1065E000F2B3F5EFB2F0F7EFB2F01EEFB2F0010147
:1065F000F2A9FDEFB2F0FFEFB2F016EFB3F03B06F9
:10660000D8A03C06820E3B24D96E020E3C20DA6EE6
:1066100060009BF0DFFF3B06D8A03C06820E3B24C7
:10662000D96E020E3C20DA6E300EDF6E1CC011F007
:106630001DC012F0820E3B24136E020E3C20146E1D
:1066400031C015F032C016F0B9ECCBF011C01CF01F
:1066500012C01DF01200000E0101F86F040EF96F58
:106660006000E3F7D9FF6000E7F7DAFF000EDF6EA6
:106670003D017599738F000E0101EB6F020EEA6FF9
:10668000EAC100F1EBC101F153ECD9F00009D8B433
:106690004CEFB3F04EEFB3F048EFB4F00101EB353F
:1066A000EB31E66FEA315B6EE6C15CF0F8C1C9F12F
:1066B000F9C1CAF1A60ECB6FFB0ECC6FEAC1CDF1CA
:1066C000EBC1CEF15BC0CFF15CC0D0F1E2ECD5F014
:1066D000EDEFB3F0F8C10EF1F9C10FF1290E106F13
:1066E000FE0E116F22ECDAF040EFB4F0300E006FC6
:1066F000030E016F370E026FFF0E036F2AECD2F00C
:10670000F8C100F1F9C101F1DAECD4F000C1E8F10F
:1067100001C1E9F10101E851F825046FE951F921BE
:10672000056F300E066F030E076F46ECD3F040EF97
:10673000B4F0F8C10EF1F9C10FF1140E106FFF0E95
:10674000116F22ECDAF040EFB4F0F8C10EF1F9C1AC
:106750000FF1DD0E106FFE0E116F22ECDAF040EF3C
:10676000B4F0F8C10EF1F9C10FF1770E106FFF0E02
:10677000116F22ECDAF040EFB4F0F8C10EF1F9C17C
:106780000FF1590E106FFF0E116F22ECDAF040EF8F
:10679000B4F0F8C10EF1F9C10FF19D0E106FFF0EAC
:1067A000116F22ECDAF040EFB4F0F8C10EF1F9C14C
:1067B0000FF1A20E106FFD0E116F22ECDAF040EF18
:1067C000B4F0F8C10EF1F9C10FF1840E106FFF0E95
:1067D000116F22ECDAF040EFB4F05BC0E6F15CC080
:1067E000E7F10101E751000AD8B4F9EFB3F0E1EFA6
:1067F000B3F0E651200AD8B46AEFB3F0010AD8B476
:106800006AEFB3F0030AD8B46AEFB3F0010AD8B460
:106810006AEFB3F0040AD8B46AEFB3F00F0AD8B441
:1068200076EFB3F0010AD8B476EFB3F0030AD8B428
:1068300076EFB3F01D0AD8B499EFB3F00F0AD8B4CD
:10684000A5EFB3F0010AD8B4A5EFB3F0030AD8B4AA
:10685000A5EFB3F0010AD8B4A5EFB3F0070AD8B496
:10686000B1EFB3F06B0AD8B4BDEFB3F03F0AD8B4C0
:10687000C9EFB3F0C80AD8B4D5EFB3F0E1EFB3F085
:10688000F8C100F1F9C101F1B4ECD1F09CECD9F000
:10689000020E0101EA25EA6F000EEB21EB6FEBBF60
:1068A0005BEFB4F0EB5109E1FC0EEA5DD8A05BEFC1
:1068B000B4F05DEFB4F040EFB3F03D01739F758924
:1068C0009CECD9F01200C4C057F1C5C058F1C6C045
:1068D00059F1C7C05AF147C157F148C158F149C1F0
:1068E00059F14AC15AF1810E01014B6FFF0E4C6FF5
:1068F00057C14DF158C14EF159C14FF15AC150F134
:10690000180E88EFB4F0D89050334F334E334D33D8
:10691000E82E83EFB4F04D514B25556F000E4C21FE
:10692000566F56BF9DEFB4F0565109E1170E555DF5
:10693000D8A09DEFB4F09FEFB4F0A9EFB4F047C139
:1069400047F148C148F149C149F14AC14AF16DEFE7
:10695000B5F056BFAEEFB4F0B0EFB4F021EFB5F044
:1069600055C14BF1FF0E4C6FFF0E4D6F7F0E4E6FFA
:10697000000E4F6F4B67BFEFB4F0C7EFB4F04F3569
:106980004F334E334D334C334B2FBAEFB4F04CC131
:1069900051F14DC152F14EC153F14FC154F10101BA
:1069A000515157154B6F525158154C6F5351591542
:1069B0004D6F54515A154E6F4B514C114D114E1194
:1069C000D8A4E5EFB4F0E7EFB4F0E9EFB4F09FEF4F
:1069D000B4F057C14BF158C14CF159C14DF15AC1F6
:1069E0004EF1200EF9EFB4F0D8904E334D334C33C6
:1069F0004B33E82EF4EFB4F04B514C114D114E11C6
:106A0000D8B405EFB5F007EFB5F00FEFB5F0515181
:106A10005727525158235351592354515A23511D2A
:106A20004B6F521D4C6F531D4D6F541D4E6F4B518C
:106A300057174C5158174D5159174E515A1765EF6A
:106A4000B5F057C14BF158C14CF159C14DF15AC184
:106A50004EF1200E31EFB5F0D8904E334D334C331C
:106A60004B33E82E2CEFB5F04B514C114D114E111C
:106A7000D8A43DEFB5F03FEFB5F049EFB5F0000E0B
:106A8000576F000E586F000E596F000E5A6F65EF6A
:106A9000B5F0D89057354B6F58354C6F59354D6F11
:106AA0005A354E6F4B514C114D114E11D8B45BEF0E
:106AB000B5F05DEFB5F065EFB5F0000E576F000E65
:106AC000586F800E596FBF0E5A6F57C147F158C1AA
:106AD00048F159C149F15AC14AF11200C4C02AF023
:106AE000C5C02BF0C6C02CF0C7C02DF01AC02AF0CC
:106AF0001BC02BF01CC02CF01DC02DF0810E1E6E93
:106B0000FF0E1F6E2AC020F02BC021F02CC022F0F7
:106B10002DC023F0180E92EFB5F0D8902332223218
:106B200021322032E82E8DEFB5F020501E24286E41
:106B3000000E1F20296E29BEA7EFB5F0295009E1EC
:106B4000170E285CD8A0A7EFB5F0A9EFB5F0B3EF0A
:106B5000B5F01AC01AF01BC01BF01CC01CF01DC001
:106B60001DF076EFB6F029BEB8EFB5F0BAEFB5F08C
:106B70002AEFB6F028C01EF0FF0E1F6EFF0E206E2B
:106B80007F0E216E000E226E1E66C9EFB5F0D1EFAA
:106B9000B5F022342232213220321F321E2EC4EFB1
:106BA000B5F01FC024F020C025F021C026F022C07F
:106BB00027F024502A141E6E25502B141F6E2650C9
:106BC0002C14206E27502D14216E1E501F102010E3
:106BD0002110D8A4EEEFB5F0F0EFB5F0F2EFB5F07C
:106BE000A9EFB5F02AC01EF02BC01FF02CC020F07A
:106BF0002DC021F0200E02EFB6F0D89021322032C5
:106C00001F321E32E82EFDEFB5F01E501F1020106F
:106C10002110D8B40EEFB6F010EFB6F018EFB6F0C2
:106C200024502A2625502B2226502C2227502D2254
:106C3000241C1E6E251C1F6E261C206E271C216E18
:106C40001E502A161F502B1620502C1621502D1680
:106C50006EEFB6F02AC01EF02BC01FF02CC020F043
:106C60002DC021F0200E3AEFB6F0D890213220321C
:106C70001F321E32E82E35EFB6F01E501F102010C6
:106C80002110D8A446EFB6F048EFB6F052EFB6F0B8
:106C9000000E2A6E000E2B6E000E2C6E000E2D6E56
:106CA0006EEFB6F0D8902A341E6E2B341F6E2C3443
:106CB000206E2D34216E1E501F1020102110D8B4CC
:106CC00064EFB6F066EFB6F06EEFB6F0000E2A6E27
:106CD000000E2B6E800E2C6EBF0E2D6E2AC01AF089
:106CE0002BC01BF02CC01CF02DC01DF012000101A8
:106CF000F1BF7DEFB6F07FEFB6F080EFB6F0F29324
:106D0000F1BF8DEFB6F0F15106E1F005D8B08BEF91
:106D1000B6F08DEFB6F093EFB6F0000E2E6F010EC9
:106D20002D6F97EFB6F0F0C12DF1F1C12EF1EEC14C
:106D30002FF1EFC130F11DC131F11EC132F11FC180
:106D400033F120C134F121C135F122C136F123C123
:106D500037F124C138F1000E3A6F4F0E396F000E33
:106D60000201D16F2BEFB7F03907D8A03A07820E96
:106D70003925D96E020E3A21DA6E31C100F132C1E5
:106D800001F133C102F134C103F135C104F136C15F
:106D900005F137C106F138C107F10A0E086F000E80
:106DA000096F000E0A6F000E0B6F000E0C6F000EC5
:106DB0000D6F000E0E6F000E0F6FBBECC9F000C11F
:106DC00025F101C126F102C127F103C128F104C157
:106DD00029F105C12AF106C12BF107C12CF10101EE
:106DE0002551300FDF6E2D07D8A02E072F07D8A012
:106DF000300731C100F132C101F133C102F134C1B8
:106E000003F135C104F136C105F137C106F138C1CE
:106E100007F10A0E086F000E096F000E0A6F000ED0
:106E20000B6F000E0C6F000E0D6F000E0E6F000E3C
:106E30000F6F17ECC7F000C131F101C132F102C18F
:106E400033F103C134F104C135F105C136F106C196
:106E500037F107C138F1010139513A11D8B433EF94
:106E6000B7F035EFB7F065EFB7F0315132113311AC
:106E700034113511361137113811D8A442EFB7F05B
:106E800044EFB7F0B4EFB6F02EBF51EFB7F02E518C
:106E900006E12D05D8B04FEFB7F051EFB7F0B4EFE2
:106EA000B6F030BF5CEFB7F0305108E12F05D8A045
:106EB0005CEFB7F05EEFB7F065EFB7F0F2B363EFFA
:106EC000B7F065EFB7F0B4EFB6F01BC110F11CC11D
:106ED00011F1820E3925126F020E3A21136F2FC164
:106EE00014F130C115F1F1ECCAF010C11BF111C160
:106EF0001CF112000101F1BF80EFB7F082EFB7F093
:106F000083EFB7F0F293F1BF90EFB7F0F15106E1E4
:106F1000F005D8B08EEFB7F090EFB7F096EFB7F07E
:106F2000000E2F6E010E2E6E9AEFB7F0F0C12EF00C
:106F3000F1C12FF0EEC130F0EFC131F01EC032F0E0
:106F40001FC033F020C034F021C035F022C036F02D
:106F500023C037F024C038F025C039F0000E3B6E56
:106F60004F0E3A6E000E0201D16F2DEFB8F03A06C7
:106F7000D8A03B06820E3A24D96E020E3B20DA6E70
:106F800032C001F033C002F034C003F035C004F069
:106F900036C005F037C006F038C007F039C008F039
:106FA0000A0E096E000E0A6E000E0B6E000E0C6EBD
:106FB000000E0D6E000E0E6E000E0F6E000E106EA7
:106FC00024ECCAF001C026F002C027F003C028F06C
:106FD00004C029F005C02AF006C02BF007C02CF031
:106FE00008C02DF02650300FDF6E2E06D8A02F06D9
:106FF0003006D8A0310632C001F033C002F034C0F0
:1070000003F035C004F036C005F037C006F038C0D4
:1070100007F039C008F00A0E096E000E0A6E000E65
:107020000B6E000E0C6E000E0D6E000E0E6E000E3E
:107030000F6E000E106E90ECC7F001C032F002C06F
:1070400033F003C034F004C035F005C036F006C09C
:1070500037F007C038F008C039F03A503B10D8B4C8
:1070600034EFB8F036EFB8F067EFB8F032503310C5
:10707000341035103610371038103910D8A443EFBB
:10708000B8F045EFB8F0B7EFB7F02FBE52EFB8F059
:107090002F5006E12E04D8B050EFB8F052EFB8F000
:1070A000B7EFB7F031BE5DEFB8F0315008E1300412
:1070B000D8A05DEFB8F05FEFB8F067EFB8F001016E
:1070C000F2B365EFB8F067EFB8F0B7EFB7F01CC0F8
:1070D00011F01DC012F0820E3A24136E020E3B20F6
:1070E000146E30C015F031C016F0B9ECCBF011C001
:1070F0001CF012C01DF0120001010F6F01010F51B1
:10710000D8B485EFB8F087EFB8F0A9EFB8F00ABFB0
:107110008EEFB8F08CEFB8F0A9EFB8F007C10BF123
:1071200008C10CF109C10DF10AC10EF10B1F0C1FB2
:107130000D1F0E1F0B2B000E0C230D230E230BC156
:1071400011F10CC112F10DC113F10EC114F1B1EF27
:10715000B8F007C111F108C112F109C113F10AC158
:1071600014F10751081109110A11D8A4BAEFB8F0A7
:10717000BCEFB8F0C6EFB8F0000E076F000E086F56
:10718000000E096F000E0A6F57EFB9F0960E106FE0
:10719000D0EFB8F0102BD8901433133312331133CF
:1071A000000E11150B6F000E12150C6F000E13154B
:1071B0000D6FFE0E14150E6F0B510C110D110E11EB
:1071C000D8A4E5EFB8F0E7EFB8F0CAEFB8F0F5EF04
:1071D000B8F0102B010E1127000E122313231423D5
:1071E000D8901433133312331133000E11150B6F73
:1071F000000E12150C6F000E13150D6FFF0E1415F7
:107200000E6F0B510C110D110E11D8A40AEFB9F02D
:107210000CEFB9F0E9EFB8F014EFB9F01007D8901F
:10722000113712371337143713BF19EFB9F01BEFAB
:10723000B9F023EFB9F0020E106121EFB9F023EF9E
:10724000B9F00EEFB9F010B128EFB9F02AEFB9F0AC
:107250002BEFB9F0139FD890103310C10BF10C6BCA
:107260000D6B0E6B0BC10EF10D6B0C6B0B6B0B51A1
:1072700011130C5112130D5113130E5114130F51FE
:10728000D8B445EFB9F047EFB9F04FEFB9F00ABF06
:107290004EEFB9F04CEFB9F04FEFB9F0148F11C1C8
:1072A00007F112C108F113C109F114C10AF112006A
:1072B00020EEF2F210EE0EF1060E6F006FFFE3FF0C
:1072C000E806FBE20BC119F10CC11AF101011951D9
:1072D0001A11D8A46EEFB9F070EFB9F074EFB9F0ED
:1072E0000E0E196F010E1A6F19C100F11AC101F1CA
:1072F000DAECD4F000C11DF101C11EF1F0C11BF1A7
:10730000F1C11CF101011CBF88EFB9F08AEFB9F09F
:107310009FEFB9F01D511B5D1C51800A0D6F1E516E
:10732000800A0D59D8A097EFB9F099EFB9F09BEF0B
:10733000B9F09FEFB9F01BC11DF11CC11EF11DC1B9
:107340001BF11EC11CF1EEC117F1EFC118F1F2B132
:10735000ACEFB9F0AEEFB9F0CCEFB9F0BDEFB9F0EA
:10736000000E016F200E006F09C102F10AC103F186
:1073700076ECC8F001011D4B1E2B17511D5D1E51EF
:10738000800A0D6F1851800A0D59D8A0CAEFB9F0C4
:10739000CCEFB9F0B0EFB9F0000E166F000E156F1C
:1073A000F7EFB9F0600067F4F6FF60006BF4F7FFE9
:1073B000000EF86E1F0EF76403D00800F55007D0DA
:1073C0006F00DBFFE9FF6F00DFFFEAFFEF50010115
:1073D0000D6F0D51006F016B09C102F10AC103F17C
:1073E00076ECC8F00101194B1A2B154B162B1B51CB
:1073F000155D1651800A0D6F1C51800A0D59D8A0D9
:1074000004EFBAF006EFBAF0D2EFB9F0F2A10BEF49
:10741000BAF00DEFBAF02BEFBAF01CEFBAF0000E95
:10742000016F200E006F09C102F10AC103F176EC71
:10743000C8F001011D4B1E2B17511D5D1E51800A06
:107440000D6F1851800A0D59D8A029EFBAF02BEF13
:10745000BAF00FEFBAF01DC109F11EC10AF1120016
:1074600020EEF2F210EE0FF0060E6F006FFFE3FF5A
:10747000E806FBE20CC01AF00DC01BF01A501B10FE
:10748000D8A445EFBAF047EFBAF04BEFBAF00F0EC1
:107490001A6E000E1B6E1AC001F01BC002F062ECE7
:1074A000D5F001C01EF002C01FF0F0C11CF0F1C108
:1074B0001DF01DBE5EEFBAF060EFBAF075EFBAF0E6
:1074C0001E501C5C1D50800A0E6E1F50800A0E5804
:1074D000D8A06DEFBAF06FEFBAF071EFBAF075EFB8
:1074E000BAF01CC01EF01DC01FF01EC01CF01FC053
:1074F0001DF0EEC118F0EFC119F00101F2B183EFF8
:10750000BAF085EFBAF0A2EFBAF093EFBAF0000E3E
:10751000026E200E016E0AC003F00BC004F04FECA7
:10752000C9F01E4A1F2A18501E5C1F50800A0E6E9A
:107530001950800A0E58D8A0A0EFBAF0A2EFBAF006
:1075400087EFBAF0000E176E000E166ECBEFBAF092
:1075500060006BF0F6FF60006FF0F7FF000EF86E52
:107560001F0EF76403D00800F55007D06F00DBFF53
:10757000E9FF6F00DFFFEAFFEF500E6E0E50016E65
:10758000026A0AC003F00BC004F04FECC9F01A4ABB
:107590001B2A164A172A1C50165C1750800A0E6EBA
:1075A0001D50800A0E58D8A0D8EFBAF0DAEFBAF022
:1075B000A8EFBAF00101F2A1E0EFBAF0E2EFBAF001
:1075C000FFEFBAF0F0EFBAF0000E026E200E016E7F
:1075D0000AC003F00BC004F04FECC9F01E4A1F2A8A
:1075E00018501E5C1F50800A0E6E1950800A0E58EB
:1075F000D8A0FDEFBAF0FFEFBAF0E4EFBAF01EC08A
:107600000AF01FC00BF012003F013E9F3901949B0E
:10761000000E3F013E6F3E91030E3F6F000E0001D2
:10762000ED6F030E5D6EF00E0101006FFE0E016F37
:1076300036ECD5F05D50300F0101FC6FFC5183EC4E
:10764000DAF0A80E0101006FFF0E016F36ECD5F0E5
:107650005D50020DE80EF324D96E020EF420DA6EAE
:107660006F0078FF00F16F0074FF01F136ECD5F088
:107670009CECD9F0600077F13FFF000E3F013A6FBC
:10768000000E396F000E386F630E0001F96F100E97
:10769000FA6F000EFB6F000EFC6FF90E0101F46F24
:1076A000000EF56F20EE02F0F451D926F551DA22E2
:1076B000DF503F013D6F010120EE01F0F451D9266A
:1076C000F551DA22DF503F013C6F6000D3F7D9FF5C
:1076D0006000D7F7DAFFDF503B6F5D50040DEE0E10
:1076E000F324F66EF50EF420F76EF86A000EF82219
:1076F00009006F00D4FF19F109006F00D4FF1AF1DF
:1077000009006F00D4FF1BF10A006F00D4FF1CF1C9
:10771000F9C007F1FAC008F1FBC009F1FCC00AF199
:10772000000E7CECB8F007C115F108C116F109C1D3
:1077300017F10AC118F1B1ECA5F015C12EF116C16F
:107740002FF117C130F118C131F1000E0101326F74
:10775000000E336F000E346F4A0E356F00ECAAF046
:107760002EC1D0F02FC1D1F030C1D2F031C1D3F051
:10777000300E0101C96F030ECA6F0F0ECB6FFE0EE4
:10778000CC6FD0C0CDF1D1C0CEF1D2C0CFF1D3C03B
:10779000D0F1E2ECD5F0300E0101006F030E016F65
:1077A000B4ECD1F03F013E8F1200000E0101116FC9
:1077B0000FBFDFEFBBF0DDEFBBF0F1EFBBF00F1F52
:1077C0000E1F0D1F0C1F0B1F0A1F091F086D000E37
:1077D00009230A230B230C230D230E230F23010E51
:1077E000116F07BFF8EFBBF0F6EFBBF00AEFBCF08C
:1077F000071F061F051F041F031F021F011F006D27
:10780000000E012302230323042305230623072359
:10781000010E111B20EE12F1070EDE6AE806FDE2F2
:10782000085109110A110B110C110D110E110F1134
:10783000D8B41DEFBCF01FEFBCF071EFBCF0010E2F
:10784000106F2DEFBCF0D890083709370A370B3787
:107850000C370D370E370F37102B0FAF32EFBCF050
:1078600034EFBCF023EFBCF0D89012371337143745
:10787000153716371737183719370851005D095172
:1078800001590A5102590B5103590C5104590D5118
:1078900005590E5106590F510759D8A052EFBCF0A7
:1078A00054EFBCF065EFBCF00851005F0951015B7B
:1078B0000A51025B0B51035B0C51045B0D51055BDC
:1078C0000E51065B0F51075B1281D8900F330E33B8
:1078D0000D330C330B330A3309330833102F34EFD5
:1078E000BCF01151D8B477EFBCF079EFBCF089EF60
:1078F000BCF0191F181F171F161F151F141F131F69
:10790000126D000E13231423152316231723182397
:10791000192312C100F113C101F114C102F115C103
:1079200003F116C104F117C105F118C106F119C11F
:1079300007F11200000E126E10BEA3EFBCF0A1EF13
:10794000BCF0B5EFBCF0101E0F1E0E1E0D1E0C1E5F
:107950000B1E0A1E096C000E0A220B220C220D229D
:107960000E220F221022010E126E08BEBCEFBCF0D8
:10797000BAEFBCF0CEEFBCF0081E071E061E051EB7
:10798000041E031E021E016C000E022203220422AA
:107990000522062207220822010E121A20EE13F0F9
:1079A000070EDE6AE806FDE209500A100B100C1003
:1079B0000D100E100F101010D8B4E1EFBCF0E3EF73
:1079C000BCF035EFBDF0010E116EF1EFBCF0D890B8
:1079D00009360A360B360C360D360E360F36103693
:1079E000112A10AEF6EFBCF0F8EFBCF0E7EFBCF0F8
:1079F000D89013361436153616361736183619360B
:107A00001A360950015C0A5002580B5003580C50AA
:107A100004580D5005580E5006580F500758105076
:107A20000858D8A016EFBDF018EFBDF029EFBDF053
:107A30000950015E0A50025A0B50035A0C50045A66
:107A40000D50055A0E50065A0F50075A1050085A3A
:107A50001380D89010320F320E320D320C320B32AE
:107A60000A320932112EF8EFBCF01250D8B43BEFB5
:107A7000BDF03DEFBDF04DEFBDF01A1E191E181EF2
:107A8000171E161E151E141E136C000E142215222E
:107A900016221722182219221A2213C001F014C02C
:107AA00002F015C003F016C004F017C005F018C0AE
:107AB00006F019C007F01AC008F01200000E01010C
:107AC000106F000E0F6F000E0E6F000E0D6F6BEF3C
:107AD000BDF0074B082B60001FF4F6FF600023F495
:107AE000F7FF000EF86E0800F550200AD8B47BEFBF
:107AF000BDF07DEFBDF069EFBDF0F70E096FFF0E31
:107B00000A6F60001FF4F6FF600023F4F7FF000E19
:107B1000F86E0800F5500B6F0C6B09510B270A51DA
:107B20000C230C5109E1050E0B5DD8A09AEFBDF0B6
:107B30009CEFBDF069EFBDF0A6EFBDF0000E0E6F3B
:107B4000010E0D6F074B082BE4EFBDF060001FF432
:107B5000F6FF600023F4F7FF000EF86E0800F55002
:107B6000096F0A6B0A51000AD8B4B9EFBDF0E4EF0F
:107B7000BDF009512B0AD8B4A2EFBDF0060AD8B463
:107B80009EEFBDF0E4EFBDF00FC100F110C101F1B7
:107B9000000E036F0A0E026FE1ECD9F060001FF4D3
:107BA000F6FF600023F4F7FF000EF86E0800F550B2
:107BB0000101005F000E015B300E00250F6F000E0B
:107BC0000121106FA2EFBDF0D00E096FFF0E0A6FFA
:107BD00060001FF4F6FF600023F4F7FF000EF86E5C
:107BE0000800F5500B6F0C6B09510B270A510C2341
:107BF0000C5109E10A0E0B5DD8A001EFBEF003EFB6
:107C0000BEF0C4EFBDF00D510E11D8A40AEFBEF0C6
:107C10000CEFBEF01AEFBEF00FC109F110C10AF16E
:107C2000091F0A1F094B0A2B09C107F10AC108F1F4
:107C30001EEFBEF00FC107F110C108F11200000ED7
:107C4000106E000E0F6E000E0E6E000E0D6E2BEFFE
:107C5000BEF0074A082A60001FF0F6FF600023F01C
:107C6000F7FF000EF86E0800F550200AD8B43BEF7D
:107C7000BEF03DEFBEF029EFBEF0F70E096EFF0E2D
:107C80000A6E60001FF0F6FF600023F0F7FF000EA1
:107C9000F86E0800F5500B6E0C6A09500B260A505E
:107CA0000C220C5009E1050E0B5CD8A05AEFBEF077
:107CB0005CEFBEF029EFBEF066EFBEF0000E0E6E78
:107CC000010E0D6E074A082AA3EFBEF060001FF0F8
:107CD000F6FF600023F0F7FF000EF86E0800F55085
:107CE000096E0A6A0A50000AD8B479EFBEF0A3EF11
:107CF000BEF009502B0AD8B462EFBEF0060AD8B421
:107D00005EEFBEF0A3EFBEF00FC001F010C002F0B6
:107D1000000E046E0A0E036E0DECDAF060001FF028
:107D2000F6FF600023F0F7FF000EF86E0800F55034
:107D3000015E000E025A300E01240F6E000E02206A
:107D4000106E62EFBEF0D00E096EFF0E0A6E60007C
:107D50001FF0F6FF600023F0F7FF000EF86E08003A
:107D6000F5500B6E0C6A09500B260A500C220C5071
:107D700009E10A0E0B5CD8A0C0EFBEF0C2EFBEF066
:107D800084EFBEF00D500E10D8A4C9EFBEF0CBEFBB
:107D9000BEF0D9EFBEF00FC009F010C00AF0091E06
:107DA0000A1E094A0A2A09C007F00AC008F0DDEFD6
:107DB000BEF00FC007F010C008F01200000E010165
:107DC000116F07BFE8EFBEF0E6EFBEF0FAEFBEF0CE
:107DD000071F061F051F041F031F021F011F006D41
:107DE000000E012302230323042305230623072374
:107DF000010E116F0FBF01EFBFF0FFEFBEF011EFEB
:107E0000BFF00F1F0E1F0D1F0C1F0B1F0A1F091F96
:107E1000086D000E09230A230B230C230D230E23C8
:107E20000F23085109110A110B110C110D110E111C
:107E30000F11D8B41EEFBFF020EFBFF068EFBFF016
:107E4000010E106F2EEFBFF0D890083709370A37B0
:107E50000B370C370D370E370F37102B0FAF33EFB3
:107E6000BFF035EFBFF024EFBFF00851005D0951BE
:107E700001590A5102590B5103590C5104590D5122
:107E800005590E5106590F510759D8A04AEFBFF0B6
:107E90004CEFBFF05CEFBFF00851005F0951015B90
:107EA0000A51025B0B51035B0C51045B0D51055BE6
:107EB0000E51065B0F51075BD8900F330E330D3315
:107EC0000C330B330A3309330833102F35EFBFF06F
:107ED0001151D8B46EEFBFF070EFBFF080EFBFF07C
:107EE000071F061F051F041F031F021F011F006D30
:107EF000000E012302230323042305230623072363
:107F000000C100F101C101F102C102F103C103F19D
:107F100004C104F105C105F106C106F107C107F16D
:107F20001200000E126E08BE9AEFBFF098EFBFF07D
:107F3000ACEFBFF0081E071E061E051E041E031E22
:107F4000021E016C000E02220322042205220622D8
:107F500007220822010E126E10BEB3EFBFF0B1EF80
:107F6000BFF0C3EFBFF0101E0F1E0E1E0D1E0C1E25
:107F70000B1E0A1E096C000E0A220B220C220D2277
:107F80000E220F22102209500A100B100C100D1097
:107F90000E100F101010D8B4D0EFBFF0D2EFBFF01A
:107FA0001AEFC0F0010E116EE0EFBFF0D890093665
:107FB0000A360B360C360D360E360F361036112AB1
:107FC00010AEE5EFBFF0E7EFBFF0D6EFBFF009501E
:107FD000015C0A5002580B5003580C5004580D50C5
:107FE00005580E5006580F50075810500858D8A082
:107FF000FCEFBFF0FEEFBFF00EEFC0F00950015EE6
:108000000A50025A0B50035A0C50045A0D50055A8C
:108010000E50065A0F50075A1050085AD890103276
:108020000F320E320D320C320B320A320932112E5F
:10803000E7EFBFF01250D8B420EFC0F022EFC0F04D
:1080400032EFC0F0081E071E061E051E041E031E8A
:10805000021E016C000E02220322042205220622C7
:108060000722082201C001F002C002F003C003F0A1
:1080700004C004F005C005F006C006F007C007F014
:1080800008C008F01200F70E0101006FFF0E016F2B
:1080900036ECD5F0000E01011E6F300E7EECD0F0F4
:1080A000680E0101226FE40EE82EFED7222FFCD7C6
:1080B00000F0320E83ECDAF0000E01011E6F300E7C
:1080C0007EECD0F0150E0101226FC60EE82EFED711
:1080D000222FFCD700F0330E83ECDAF0000E010102
:1080E0001E6F300E7EECD0F0150E0101226FC60E11
:1080F000E82EFED7222FFCD700F0340E83ECDAF006
:10810000000E01011E6F250E7EECD0F0150E010150
:10811000226FC60EE82EFED7222FFCD700F0350EB8
:1081200083ECDAF0010E01011E6F280E7EECD0F018
:10813000150E0101226FC60EE82EFED7222FFCD7A6
:1081400000F0360E83ECDAF0010E01011E6F080E0E
:108150007EECD0F0150E0101226FC60EE82EFED780
:10816000222FFCD700F0370E83ECDAF0010E01016C
:108170001E6F010E7EECD0F0030E0101236F080E7E
:10818000226F770EE82EFED7222FFCD7232FFAD7A7
:10819000380E83ECDAF0010E01011E6F060E7EEC44
:1081A000D0F0150E0101226FC60EE82EFED7222F49
:1081B000FCD700F0390E83ECDAF0010E01011E6FDE
:1081C0000C0E7EECD0F0150E0101226FC60EE82ECB
:1081D000FED7222FFCD700F0410E83ECDAF012001C
:1081E00000C107F101C108F102C109F103C10AF19F
:1081F00001010407D8A00507042906E10529D8A430
:1082000004EFC1F006EFC1F014EFC1F0000E016FF2
:10821000000E006F9CEFC1F00101074B082B094BCA
:108220000A2B0407D8A0050760001FF4F6FF6000C2
:1082300023F4F7FF000EF86E1F0EF76403D008005A
:10824000F55007D06F00DBFFE9FF6F00DFFFEAFFAB
:10825000EF500009D8B42FEFC1F031EFC1F076EF45
:10826000C1F0600027F4F6FF60002BF4F7FF000E6A
:10827000F86E0800F5500009D8B441EFC1F043EFA3
:10828000C1F076EFC1F0010104510511D8B44BEFF4
:10829000C1F04DEFC1F076EFC1F0600027F4F6FFBA
:1082A00060002BF4F7FF000EF86E08006F00D4FF9B
:1082B00006F160001FF4F6FF600023F4F7FF000EE4
:1082C000F86E1F0EF76403D00800F55007D06F005A
:1082D000DBFFE9FF6F00DFFFEAFFEF500619D8B4BC
:1082E00074EFC1F076EFC1F00CEFC1F060001FF445
:1082F000F6FF600023F4F7FF000EF86E1F0EF76420
:1083000003D00800F55007D06F00DBFFE9FF6F00D6
:10831000DFFFEAFFEF500101066F600027F4F6FF70
:1083200060002BF4F7FF000EF86E0800F550065DB4
:10833000006F016BD8A001071200000E0301306F1F
:10834000BCB0A5EFC1F0A7EFC1F0AEEFC1F0EF0EEA
:108350000101E66FFF0EE76FB3EFC1F0F30E01010D
:10836000E66FFF0EE76F300EC96F030ECA6F020E85
:10837000CB6FFF0ECC6FE6C1CDF1E7C1CEF1FDC0F2
:10838000CFF1FEC0D0F1E2ECD5F0010E0101276F74
:10839000300E286F030E296F010EB5ECDAF0000ED7
:1083A0000301306F0001EE51D8B4D9EFC1F0DBEF1B
:1083B000C1F0E2EFC1F0C40E0101E86FFF0EE96FFA
:1083C000E7EFC1F0CC0E0101E86FFF0EE96F300E50
:1083D000C96F030ECA6F260ECB6FFF0ECC6FE8C1BC
:1083E000CDF1E9C1CEF1300E0001EB250101CF6FD7
:1083F000D06B000ED023E2ECD5F0010E0101276F07
:10840000300E286F030E296F020EB5ECDAF0000E65
:108410000301306F300E0101C96F030ECA6F9E0E4B
:10842000CB6FFE0ECC6FD0C0CDF1D1C0CEF1D2C09B
:10843000CFF1D3C0D0F1E2ECD5F0010E0101276FEE
:10844000300E286F030E296F030EB5ECDAF0000E24
:108450000301306F300E0101C96F030ECA6F480E61
:10846000CB6FFF0ECC6FDAC0CDF1DBC0CEF1D8C040
:10847000CFF1D9C0D0F1E2ECD5F0010E0101276FA8
:10848000300E286F030E296F040EB5ECDAF01200DF
:1084900001C008F002C009F003C00AF004C00BF0EC
:1084A0000506D8A00606052806E10628D8A45BEF35
:1084B000C2F05DEFC2F06AEFC2F0000E026E000E75
:1084C000016EF0EFC2F0084A092A0A4A0B2A050693
:1084D000D8A00606600023F0F6FF600027F0F7FF43
:1084E000000EF86E1F0EF76403D00800F55007D099
:1084F0006F00DBFFE9FF6F00DFFFEAFFEF500009CD
:10850000D8B485EFC2F087EFC2F0CBEFC2F06000C5
:108510002BF0F6FF60002FF0F7FF000EF86E08005A
:10852000F5500009D8B497EFC2F099EFC2F0CBEF45
:10853000C2F005500610D8B4A0EFC2F0A2EFC2F00E
:10854000CBEFC2F060002BF0F6FF60002FF0F7FFDA
:10855000000EF86E08006F00D4FF07F0600023F0F3
:10856000F6FF600027F0F7FF000EF86E1F0EF764AD
:1085700003D00800F55007D06F00DBFFE9FF6F0064
:10858000DFFFEAFFEF500718D8B4C9EFC2F0CBEF16
:10859000C2F063EFC2F0600023F0F6FF600027F046
:1085A000F7FF000EF86E1F0EF76403D00800F550B9
:1085B00007D06F00DBFFE9FF6F00DFFFEAFFEF503E
:1085C000076E60002BF0F6FF60002FF0F7FF000E43
:1085D000F86E0800F550075C016E026AD8A002062A
:1085E000120014ECDBF00009D8B4F9EFC2F0FBEF95
:1085F000C2F038EFC3F008EFC3F06EECDBF08FEFA2
:10860000C3F0C6ECDBF08FEFC3F0000E8FEFC3F0CA
:1086100018C20BF119C20CF120EE09F202D81BEFBF
:10862000C3F00500FA6EDE50FD6EDE50FE6EDE50C9
:10863000FF6EFA50120001010D6F0E6B0E51000A11
:10864000D8B425EFC3F005EFC3F00D51010AD8B43B
:1086500005EFC3F0030AD8B4FDEFC2F0010AD8B4A5
:1086600001EFC3F0070AD8B405EFC3F005EFC3F07C
:1086700009ECDBF00009D8B440EFC3F042EFC3F0DF
:108680008EEFC3F002012951030B0009D8B44BEF60
:10869000C3F04DEFC3F05FEFC3F0010E01010D6FAA
:1086A00002012951030B01010E6F0D510E5F0201F2
:1086B000295101010E19FC0B0E190201296F6000EE
:1086C0008FF8D9FF600093F8DAFFDF500101116FD6
:1086D0000201234B242B2507D8A02607255126115C
:1086E000D8A475EFC3F077EFC3F080EFC3F0C1EC0F
:1086F000D0F001010D6F0D510F6F106B85EFC3F0BE
:10870000000E0101106F030E0F6F0FC112F1115116
:108710007BECDBF0010112518FEFC3F0030E12006E
:10872000010149354A35506F5051D8A49AEFC3F032
:108730009CEFC3F0A6EFC3F0000E476F000E486F2A
:10874000000E496F000E4A6F13EFC4F047C14BF1A2
:1087500048C14CF149C14DF14AC14EF1200EB6EF6E
:10876000C3F0D8904E334D334C334B33E82EB1EF3A
:10877000C3F04B514F6F498FFF0E4717FF0E48173D
:10878000FF0E4917000E4A17960E505F50BFCDEFEF
:10879000C3F0CBEFC3F0E3EFC3F05051800A970F63
:1087A000D8B0D5EFC3F0D7EFC3F0D9EFC3F09CEF4B
:1087B000C3F0D8904A33493348334733503FD9EF59
:1087C000C3F0FBEFC3F01F0E5065E9EFC3F0EBEF12
:1087D000C3F0F3EFC3F09CEFC3F0D89047374837AE
:1087E00049374A3750075051D8A4F9EFC3F0FBEF8F
:1087F000C3F0EDEFC3F04F51D8B401EFC4F003EF75
:10880000C4F00BEFC4F04A1F491F481F476D000E0C
:10881000482349234A2347C147F148C148F149C188
:1088200049F14AC14AF11200000E01012E15366FBE
:10883000000E2F15376F800E3015386F7F0E3115F3
:10884000396F3651371138113911D8A42AEFC4F0D5
:108850002CEFC4F034EFC4F0000E2E6F000E2F6F1B
:10886000000E306F000E316F000E3215366F000EA5
:108870003315376F800E3415386F7F0E3515396F0D
:108880003651371138113911D8A449EFC4F04BEFE4
:10889000C4F053EFC4F0000E326F000E336F000EC1
:1088A000346F000E356F31AF58EFC4F05AEFC4F09B
:1088B00063EFC4F02E6D2F1FD8B02F2B301FD8B010
:1088C000302B800E315735AF68EFC4F06AEFC4F03B
:1088D00073EFC4F0326D331FD8B0332B341FD8B0D0
:1088E000342B800E3557000E2E1B000E2F1B000E52
:1088F000301B800E311B000E321B000E331B000E8E
:10890000341B800E351B32512E5D33512F5934519B
:10891000305935513159D8B090EFC4F092EFC4F0CE
:1089200095EFC4F0D89096EFC4F0D88012000334CD
:1089300004340A6E0A50D8A4A0EFC4F0A2EFC4F029
:10894000ACEFC4F0000E016E000E026E000E036E5E
:10895000000E046E19EFC5F001C005F002C006F06C
:1089600003C007F004C008F0200EBCEFC4F0D8909C
:108970000832073206320532E82EB7EFC4F0055050
:10898000096E038EFF0E0116FF0E0216FF0E031670
:10899000000E0416960E0A5E0ABED3EFC4F0D1EFA5
:1089A000C4F0E9EFC4F00A50800A970FD8B0DBEFAB
:1089B000C4F0DDEFC4F0DFEFC4F0A2EFC4F0D89054
:1089C00004320332023201320A3EDFEFC4F001EF1B
:1089D000C5F01F0E0A64EFEFC4F0F1EFC4F0F9EF39
:1089E000C4F0A2EFC4F0D890013602360336043644
:1089F0000A060A50D8A4FFEFC4F001EFC5F0F3EF68
:108A0000C4F00950D8B407EFC5F009EFC5F011EF75
:108A1000C5F0041E031E021E016C000E022203227A
:108A2000042201C001F002C002F003C003F004C040
:108A300004F01200000E1A14226E000E1B14236E96
:108A4000800E1C14246E7F0E1D14256E22502310E0
:108A500024102510D8A42FEFC5F031EFC5F039EF61
:108A6000C5F0000E1A6E000E1B6E000E1C6E000E7E
:108A70001D6E000E1E14226E000E1F14236E800E3B
:108A80002014246E7F0E2114256E225023102410F2
:108A90002510D8A44EEFC5F050EFC5F058EFC5F043
:108AA000000E1E6E000E1F6E000E206E000E216E58
:108AB0001DAE5DEFC5F05FEFC5F068EFC5F01A6C55
:108AC0001B1ED8B01B2A1C1ED8B01C2A800E1D5697
:108AD00021AE6DEFC5F06FEFC5F078EFC5F01E6CFD
:108AE0001F1ED8B01F2A201ED8B0202A800E215663
:108AF000000E1A1A000E1B1A000E1C1A800E1D1AE8
:108B0000000E1E1A000E1F1A000E201A800E211AC7
:108B10001E501A5C1F501B5820501C5821501D58C5
:108B2000D8B095EFC5F097EFC5F09AEFC5F0D890A3
:108B30009BEFC5F0D8801200C8C00AF1C9C00BF184
:108B4000CAC00CF1CBC00DF100C10AF101C10BF19B
:108B500002C10CF103C10DF10AC104F10BC105F111
:108B60000CC106F10DC107F1180EBDEFC5F00101F2
:108B7000D8900733063305330433E82EB7EFC5F03A
:108B80000451086F096B08510911D8A4CAEFC5F048
:108B9000CCEFC5F0ECEFC5F0D8900A35046F0B357B
:108BA000056F0C35066F0D35076F04510511061161
:108BB0000711D8A4DEEFC5F0E0EFC5F0E6EFC5F091
:108BC000000E016F020E006F1BEFC6F0000E016F6A
:108BD000030E006F1BEFC6F008290911D8A4F3EFAC
:108BE000C5F0F5EFC5F017EFC6F00AC104F10BC1EF
:108BF00005F10CC106F10DC107F1090ED89004373B
:108C0000053706370737E82EFEEFC5F0045105118A
:108C100006110711D8B40FEFC6F012EFC6F0010E1F
:108C200013EFC6F0000E006F016B1BEFC6F0000ED5
:108C3000016F040E006F1200C8C00BF0C9C00CF029
:108C4000CAC00DF0CBC00EF001C00BF002C00CF09A
:108C500003C00DF004C00EF00BC005F00CC006F010
:108C60000DC007F00EC008F0180E3CEFC6F0D8900B
:108C70000832073206320532E82E37EFC6F00550CB
:108C8000096E0A6A09500A10D8A449EFC6F04BEFE2
:108C9000C6F06BEFC6F0D8900B34056E0C34066E40
:108CA0000D34076E0E34086E0550061007100810BC
:108CB000D8A45DEFC6F05FEFC6F065EFC6F0000E1A
:108CC000026E020E016E9AEFC6F0000E026E030EE7
:108CD000016E9AEFC6F009280A10D8A472EFC6F008
:108CE00074EFC6F096EFC6F00BC005F00CC006F0AE
:108CF0000DC007F00EC008F0090ED89005360636F4
:108D000007360836E82E7DEFC6F00550061007102E
:108D10000810D8B48EEFC6F091EFC6F0010E92EFB6
:108D2000C6F0000E016E026A9AEFC6F0000E026EE7
:068D3000040E016E1200AA
:108D38006F0060FF54F06F00D8FF55F06F00DCFF44
:108D480056F06F00E0FF57F06F00D4FF58F039017C
:108D580091A1B1EFC6F0B3EFC6F007EFC7F0A1A13C
:108D6800B8EFC6F0BAEFC6F007EFC7F0150E536EAE
:108D7800C60EE82EFED7532EFCD700D0AC9E390184
:108D88009495A4950001DA4BDB2BD890DA35D86F8F
:108D9800DB35D96FE0C0FDF0E1C0FEF0230EA5EC95
:108DA800DAF00D0EA5ECDAF00A0EA5ECDAF0000EFA
:108DB8000001E16F000EE06F040EF319D8A4E7EF8D
:108DC800C6F0E9EFC6F001EFC7F0300EBC6F030E36
:108DD800BD6F860EBE6FFD0EBF6FDAC0C0F0DBC080
:108DE800C1F0FDC0C2F0FEC0C3F034ECD6F0300EC6
:108DF800016E030E026E0EECD3F03901A495A09F0C
:108E08009485AC8EA191600063F1F5FF60005FF17D
:108E1800F8FF60005BF1F7FF600057F1F6FF6000B4
:108E280053F1D8FF110020EE10F1070EDE6AE806B4
:108E3800FDE20101085109110A110B110C110D1164
:108E48000E110F11D8B42BEFC7F02DEFC7F07FEF3D
:108E5800C7F0010E186F3BEFC7F0D89008370937F5
:108E68000A370B370C370D370E370F37182B0FAF64
:108E780040EFC7F042EFC7F031EFC7F0D890103796
:108E88001137123713371437153716371737085174
:108E9800005D095101590A5102590B5103590C51EE
:108EA80004590D5105590E5106590F510759D8A0AB
:108EB80060EFC7F062EFC7F073EFC7F00851005FCB
:108EC8000951015B0A51025B0B51035B0C51045BB6
:108ED8000D51055B0E51065B0F51075B1081D89051
:108EE8000F330E330D330C330B330A330933083386
:108EF800182F42EFC7F010C100F111C101F112C1E2
:108F080002F113C103F114C104F115C105F116C131
:108F180006F117C107F1120020EE11F0070EDE6A04
:108F2800E806FDE209500A100B100C100D100E1087
:108F38000F101010D8B4A3EFC7F0A5EFC7F0F7EFE4
:108F4800C7F0010E196EB3EFC7F0D89009360A368C
:108F58000B360C360D360E360F361036192A10AE73
:108F6800B8EFC7F0BAEFC7F0A9EFC7F0D89011363D
:108F78001236133614361536163617361836095083
:108F8800015C0A5002580B5003580C5004580D50FD
:108F980005580E5006580F50075810500858D8A0BA
:108FA800D8EFC7F0DAEFC7F0EBEFC7F00950015E72
:108FB8000A50025A0B50035A0C50045A0D50055AC5
:108FC8000E50065A0F50075A1050085A1180D89060
:108FD80010320F320E320D320C320B320A32093295
:108FE800192EBAEFC7F011C001F012C002F013C079
:108FF80003F014C004F015C005F016C006F017C041
:1090080007F018C008F012000101EE51EF11D8A4C2
:1090180010EFC8F012EFC8F018EFC8F0EEC10FF16A
:10902800EFC110F11EEFC8F0FF0EEE250F6FFF0E17
:10903800EF21106FF2A123EFC8F025EFC8F02EEF53
:10904800C8F00BC100F1016B09C102F10AC103F1BB
:1090580076ECC8F0010110BF34EFC8F036EFC8F065
:1090680038EFC8F03CEFC8F0000E106F000E0F6F1D
:10907800000E0E6F000E0D6F4FEFC8F0000E016F5F
:10908800200E006F09C102F10AC103F176ECC8F0A5
:1090980001010D4B0E2B0F510D5D0E51800A0C6F07
:1090A8001051800A0C59D8A05CEFC8F05EEFC8F0E8
:1090B80042EFC8F0F2B163EFC8F065EFC8F06EEFA9
:1090C800C8F00BC100F1016B09C102F10AC103F13B
:1090D80076ECC8F0010E01010D25096F000E0E2176
:1090E8000A6F1200010102510311D8B47EEFC8F0D3
:1090F80080EFC8F089EFC8F002510311D8A487EFB8
:10910800C8F089EFC8F08EEFC8F00051CDECDBF065
:10911800E2EFC8F020EE09F00251D9260351DA2215
:10912800DE50DE10D8B49BEFC8F09DEFC8F0B8EF62
:10913800C8F020EE09F00251D9260351DA2210EEC8
:1091480003F00251E1260351E222DE50E65CE650CC
:10915800800A086FDE50800A0859D8B0B6EFC8F008
:10916800B8EFC8F0E2EFC8F020EE03F00251D926BC
:109178000351DA226F0078FF04F16F0074FF05F1E4
:1091880060000BF4D9FF60000FF4DAFF6F0078FF7E
:1091980006F16F0074FF07F104510625D96E0551D9
:1091A8000721DA6E600003F4DFFF20EE03F00251BE
:1091B800D9260351DA22DE2A000EDD22120001012F
:1091C800EE51EF11D8A4EBEFC8F0EDEFC8F0F3EFD4
:1091D800C8F0EEC110F0EFC111F0F9EFC8F0FF0EC2
:1091E800EE25106EFF0EEF21116EF2A1FEEFC8F012
:1091F80000EFC9F009EFC9F00CC001F0026A0AC01B
:1092080003F00BC004F04FECC9F011BE0EEFC9F02B
:1092180010EFC9F012EFC9F016EFC9F0000E116E89
:10922800000E106E000E0F6E000E0E6E28EFC9F0C5
:10923800000E026E200E016E0AC003F00BC004F08F
:109248004FECC9F00E4A0F2A10500E5C0F50800ADE
:109258000D6E1150800A0D58D8A035EFC9F037EFC0
:10926800C9F01CEFC9F00101F2B13DEFC9F03FEFC1
:10927800C9F048EFC9F00CC001F0026A0AC003F057
:109288000BC004F04FECC9F0010E0E240A6E000E5C
:109298000F200B6E120003500410D8B456EFC9F01B
:1092A80058EFC9F061EFC9F003500410D8A45FEF7C
:1092B800C9F061EFC9F066EFC9F00150D1ECDBF0FD
:1092C800BAEFC9F020EE09F00350D9260450DA228B
:1092D800DE50DE10D8B473EFC9F075EFC9F090EF27
:1092E800C9F020EE09F00350D9260450DA2210EE16
:1092F80003F00350E1260450E222DE50E65CE6501B
:10930800800A096EDE50800A0958D8B08EEFC9F07D
:1093180090EFC9F0BAEFC9F020EE03F00350D92658
:109328000450DA226F0078FF05F06F0074FF06F032
:1093380060000FF0D9FF600013F0DAFF6F0078FFCC
:1093480007F06F0074FF08F005500724D96E065027
:109358000820DA6E600007F0DFFF20EE03F003500C
:10936800D9260450DA22DE2A000EDD22120001017D
:10937800085109110A110B110C110D110E110F11C1
:10938800D8B4C9EFC9F0CBEFC9F013EFCAF0010E9A
:10939800106FD9EFC9F0D890083709370A370B375B
:1093A8000C370D370E370F37102B0FAFDEEFC9F024
:1093B800E0EFC9F0CFEFC9F00851005D095101593C
:1093C8000A5102590B5103590C5104590D510559B1
:1093D8000E5106590F510759D8A0F5EFC9F0F7EF0C
:1093E800C9F007EFCAF00851005F0951015B0A5143
:1093F800025B0B51035B0C51045B0D51055B0E5175
:10940800065B0F51075BD8900F330E330D330C33C7
:109418000B330A3309330833102FE0EFC9F000C1CA
:1094280000F101C101F102C102F103C103F104C15C
:1094380004F105C105F106C106F107C107F11200E3
:1094480009500A100B100C100D100E100F101010F0
:10945800D8B431EFCAF033EFCAF07BEFCAF0010E8F
:10946800116E41EFCAF0D89009360A360B360C3621
:109478000D360E360F361036112A10AE46EFCAF0EA
:1094880048EFCAF037EFCAF00950015C0A50025899
:109498000B5003580C5004580D5005580E500658E0
:1094A8000F50075810500858D8A05DEFCAF05FEF6A
:1094B800CAF06FEFCAF00950015E0A50025A0B5009
:1094C800035A0C50045A0D50055A0E50065A0F50A4
:1094D800075A1050085AD89010320F320E320D32F7
:1094E8000C320B320A320932112E48EFCAF001C091
:1094F80001F002C002F003C003F004C004F005C08C
:1095080005F006C006F007C007F008C008F0120012
:10951800000EBA6EBB68BC68020EC26EC368800ECD
:10952800C46E000E3A01606F000E506F020E406F5D
:10953800000E816F5169FC0E416F6169000E006F6A
:10954800000E016F000E026F000E086F000E096F0B
:10955800000E0A6F000E0B6F000E0C6F000E0D6FE1
:10956800000E0E6F000E0F6F070E426F000E526F47
:10957800180E626F43695369636944695469646981
:10958800080E846F000E476F000E466F000E456F81
:10959800000E576F000E566F000E556F000E676F66
:1095A800000E666F000E656F000E106F000E116FD3
:1095B800000E126F000E156F000E176F210E136F3D
:1095C800220E146F260E156F130E166F170EE56F09
:1095D800130EE16F140EE26F12000101F2A1F7EF12
:1095E800CAF0F9EFCAF003EFCBF012C109F113C1C9
:1095F8000AF110C10BF111C10CF1EEECD6F001012A
:1096080015BF09EFCBF00BEFCBF011EFCBF014C186
:1096180019F115C11AF115EFCBF0000E1A6F000EF3
:10962800196F000E186F000E176F28EFCBF0000EA1
:10963800016F200E006F10C102F111C103F176EC29
:10964800C8F00101174B182B1951175D1851800AE2
:10965800166F1A51800A1659D8A035EFCBF037EF9C
:10966800CBF01BEFCBF0F2B13CEFCBF03EEFCBF001
:1096780048EFCBF012C109F113C10AF110C10BF187
:1096880011C10CF1EEECD6F012C100F113C101F1D9
:10969800DAECD4F0010119510025106F1A5101219B
:1096A800116F1200000E0101056F03BF60EFCBF0D0
:1096B8005EEFCBF066EFCBF0026D031FD8B0032B43
:1096C800010E056F01BF6DEFCBF06BEFCBF073EFC1
:1096D800CBF0006D011FD8B0012B010E051B000E49
:1096E800076F000E066F02510311D8B47EEFCBF05E
:1096F80080EFCBF0A8EFCBF0010E046F88EFCBF032
:10970800D89002370337042B03AF8DEFCBF08FEFE0
:10971800CBF084EFCBF0D890063707370251005DC5
:1097280003510159D8A09BEFCBF09DEFCBF0A2EFEE
:10973800CBF00251005F0351015B0681D8900333DF
:109748000233042F8FEFCBF00551D8B4AEEFCBF036
:10975800B0EFCBF0B4EFCBF0066D071FD8B0072BF6
:1097680006C100F107C101F112000101F2A1BFEF2A
:10977800CBF0C1EFCBF0CBEFCBF013C00AF014C0A5
:109788000BF011C00CF012C00DF09DECD7F016BE16
:10979800D0EFCBF0D2EFCBF0D8EFCBF015C01AF06A
:1097A80016C01BF0DCEFCBF0000E1B6E000E1A6E1D
:1097B800000E196E000E186EEEEFCBF0000E026E62
:1097C800200E016E11C003F012C004F04FECC9F076
:1097D800184A192A1A50185C1950800A176E1B501B
:1097E800800A1758D8A0FBEFCBF0FDEFCBF0E2EFE3
:1097F800CBF00101F2B103EFCCF005EFCCF00FEFA5
:10980800CCF013C00AF014C00BF011C00CF012C059
:109818000DF09DECD7F013C001F014C002F062EC1B
:10982800D5F01A500124116E1B500220126E12003E
:10983800000E066E04BE25EFCCF023EFCCF02BEF24
:10984800CCF0036C041ED8B0042A010E066E02BECA
:1098580032EFCCF030EFCCF038EFCCF0016C021ED8
:10986800D8B0022A010E061A000E086E000E076E06
:1098780003500410D8B443EFCCF045EFCCF06DEFB3
:10988800CCF0010E056E4DEFCCF0D89003360436BF
:10989800052A04AE52EFCCF054EFCCF049EFCCF0EF
:1098A800D890073608360350015C04500258D8A0F7
:1098B80060EFCCF062EFCCF067EFCCF00350015EC4
:1098C8000450025A0780D89004320332052E54EF10
:1098D800CCF00650D8B473EFCCF075EFCCF079EF3C
:1098E800CCF0076C081ED8B0082A07C001F008C0E1
:1098F80002F012000101266F01012251D8A487EF5E
:10990800CCF089EFCCF08BEFCCF0010E226F225116
:10991800236F246B2351FE5DFF51800A256F24516C
:10992800800A2559D8B09BEFCCF09DEFCCF09FEF83
:10993800CCF0FE05226F2605D8A4A5EFCCF0A7EF42
:10994800CCF0ABEFCCF022517F0F96ECCFF0020EAB
:1099580001012619D8A4B3EFCCF0B5EFCCF0B9EFDC
:10996800CCF02251BF0F96ECCFF0030E010126195F
:10997800D8A4C1EFCCF0C3EFCCF0C7EFCCF02251A4
:10998800930F96ECCFF0040E01012619D8A4CFEF5F
:10999800CCF0D1EFCCF0D5EFCCF02251D30F96EC30
:1099A800CFF0150E0101236FC60EE82EFED7232F28
:1099B800FCD700F01200940EF66EB40EF76E010E8E
:1099C800F86E00EED2F210EE27F009006F00D7FF14
:1099D800EEFFE550E150F9E1980EF66EB70EF76E1E
:1099E800010EF86E09006F00D4FFFEF109006F0048
:1099F800D4FFFFF1A60EF66EB70EF76E010EF86EE5
:109A080009006F00D4FFFFF001EE00F010EE00F146
:109A1800EE6AE550E150FCE1E250FAE100EE00F3B5
:109A2800B00EEE6AE806FDE100EE00F2D20EEE6A34
:109A3800E806FDE100EEEEF1100EEE6AE806FDE143
:109A480000EEC4F03B0EEE6AE806FDE15F6A5E6A6E
:109A58005D6A5C6A5B6A5A6A596A080ED56E000EBE
:109A6800D66E000ED76E0001BBEF9CF0000E010110
:109A7800056F01BF44EFCDF042EFCDF04AEFCDF0D6
:109A8800006D011FD8B0012B010E056F03BF51EF08
:109A9800CDF04FEFCDF055EFCDF0026D031FD8B0EC
:109AA800032B02510311D8B45CEFCDF05EEFCDF07B
:109AB80082EFCDF0010E046F66EFCDF0D89002373B
:109AC8000337042B03AF6BEFCDF06DEFCDF062EFF2
:109AD800CDF00251005D03510159D8A076EFCDF0C9
:109AE80078EFCDF07CEFCDF00251005F0351015BC0
:109AF800D89003330233042F6DEFCDF00551D8B45D
:109B080088EFCDF08AEFCDF08EEFCDF0006D011F1C
:109B1800D8B0012B00C100F101C101F11200000E03
:109B2800066E02BE9CEFCDF09AEFCDF0A2EFCDF01D
:109B3800016C021ED8B0022A010E066E04BEA9EFFF
:109B4800CDF0A7EFCDF0ADEFCDF0036C041ED8B08B
:109B5800042A03500410D8B4B4EFCDF0B6EFCDF01A
:109B6800DAEFCDF0010E056EBEEFCDF0D8900336DA
:109B78000436052A04AEC3EFCDF0C5EFCDF0BAEF39
:109B8800CDF00350015C04500258D8A0CEEFCDF0C0
:109B9800D0EFCDF0D4EFCDF00350015E0450025A5F
:109BA800D89004320332052EC5EFCDF00650D8B454
:109BB800E0EFCDF0E2EFCDF0E6EFCDF0016C021E64
:109BC800D8B0022A01C001F002C002F012001FEC56
:109BD800DBF00009D8A4F3EFCDF0F5EFCDF0F8EF06
:109BE800CDF0040E41EFCEF002012951030B00091C
:109BF800D8B401EFCEF003EFCEF015EFCEF0010EA2
:109C080001010F6F02012951030B0101106F0F5160
:109C1800105F0201295101011019FC0B10190201F2
:109C2800296F2507D8A0260725512611D8B41FEF7C
:109C3800CEF021EFCEF02FEFCEF0B2ECDBF06000EB
:109C48008FF8D9FF600093F8DAFFDF6E0201234B2B
:109C5800242BF5EFCDF043ECCFF00101116FB2ECFE
:109C6800DBF060008FF8D9FF600093F8DAFFDF6E51
:109C78000201234B242B010111511200000E010196
:109C88000015086F000E0115096F800E02150A6F86
:109C98007F0E03150B6F085109110A110B11D8A477
:109CA80058EFCEF05AEFCEF062EFCEF0000E006F14
:109CB800000E016F000E026F000E036F000E0415F8
:109CC800086F000E0515096F800E06150A6F7F0EC6
:109CD80007150B6F085109110A110B11D8A477EF5A
:109CE800CEF079EFCEF081EFCEF0000E046F000ECB
:109CF800056F000E066F000E076F045100190FE183
:109D0800055101190CE10651021909E1075103191E
:109D1800D8B491EFCEF093EFCEF096EFCEF0D89086
:109D280097EFCEF0D88012000101006F010E0101FB
:109D3800016F020129B7A3EFCEF0A5EFCEF0EBEF4C
:109D4800CEF000C122F229952987FC0E29170F0EA3
:109D5800276F010E216FF40E206F2989940E006F72
:109D6800B70E016F010E026F000E126F000E136F17
:109D7800940E036FB70E046F010E056F000E146F7B
:109D8800000E156F940E066FB70E076F010E086F61
:109D9800000E166F000E176F940E096FB70E0A6F3C
:109DA800010E0B6F000E186F000E196F900E0C6FDE
:109DB800B70E0D6F010E0E6F000E1A6F000E1B6F9F
:109DC800A2ECDBF0B3ECD9F0000E0101016F010148
:109DD80001511200000E0114096E000E02140A6EE1
:109DE800800E03140B6E7F0E04140C6E09500A10BB
:109DF8000B100C10D8A403EFCFF005EFCFF00DEF48
:109E0800CFF0000E016E000E026E000E036E000E03
:109E1800046E000E0514096E000E06140A6E800EFC
:109E280007140B6E7F0E08140C6E09500A100B10E5
:109E38000C10D8A422EFCFF024EFCFF02CEFCFF006
:109E4800000E056E000E066E000E076E000E086E00
:109E5800055001180FE1065002180CE107500318CD
:109E680009E108500418D8B43CEFCFF03EEFCFF02A
:109E780041EFCFF0D89042EFCFF0D8801200020126
:109E8800298967EFCFF0B5ECDBF0080E95EFCFF03E
:109E9800B5ECDBF0070E95EFCFF00201252981EC38
:109EA800DBF0040E95EFCFF0070E02012719D8B4A6
:109EB80060EFCFF062EFCFF064EFCFF0B8ECDBF0FB
:109EC8000F0E95EFCFF012C20BF113C20CF102D8AE
:109ED80078EFCFF00500FA6E0051FD6E0151FE6E6D
:109EE8000251FF6EFA50120001010D6F0E6B0E51F8
:109EF800000AD8B482EFCFF058EFCFF00D51010A25
:109F0800D8B458EFCFF0030AD8B44CEFCFF0010A19
:109F1800D8B447EFCFF0070AD8B451EFCFF058EFD5
:109F2800CFF012000101206F01012051F00B0C0944
:109F3800216F21C11AF1FD51F7ECD9F084ECD9F069
:109F480001012051F00B0809216F21C11AF1FD51BF
:109F5800F7ECD9F084ECD9F020C11EF10F0E010105
:109F68001E171E39F00B0C09216F21C11AF1FD5182
:109F7800F7ECD9F084ECD9F020C11EF10F0E0101E5
:109F88001E171E39F00B0809216F21C11AF1FD5166
:109F9800F7ECD9F084ECD9F001012005D8A4D7EF6B
:109FA800CFF0D9EFCFF0E6EFCFF0090E01011F6F28
:109FB8001E0E1E6FE40EE82EFED71E2FFCD71F2F95
:069FC800FAD700F01200C0
:109FD0003901A3A7EEEFCFF0F0EFCFF034EFD0F0E0
:109FE00093A7F5EFCFF0F7EFCFF034EFD0F06F009D
:109FF000A0F7F8F00D0E0001F819D8B402EFD0F078
:10A0000004EFD0F00FEFD0F05A5009E1800E595C08
:10A01000D8A00DEFD0F00FEFD0F025EFD0F0010E6B
:10A02000F46F800E5924D96E040E5A20DA6E000E99
:10A03000DF6E59C074F25AC075F2000E5A6E000EEF
:10A04000596E3901939734EFD0F0800E5924D96EB0
:10A05000040E5A20DA6E6000E3F3DFFF594A5A2AF1
:10A0600059C074F25AC075F211000101056F010167
:10A07000005101110211D8B440EFD0F042EFD0F0FE
:10A0800063EFD0F00551030D000EF324D96E020EDC
:10A09000F420DA6E600003F4DEFF600007F4DEFFF8
:10A0A00060000BF4DEFF0551020D120EF324D96E91
:10A0B000020EF420DA6E60000FF4DEFF600013F48D
:10A0C000DDFF7DEFD0F00551030D000EF324D96EB6
:10A0D000020EF420DA6E940EDE6EB70EDE6E010E06
:10A0E000DE6E0551020D120EF324D96E020EF4201D
:10A0F000DA6E000EDE6E000EDD6E12000101206FC2
:10A1000001012051F00B0C09216F21C11AF1FD5101
:10A11000F7ECD9F084ECD9F001012051F00B0809DB
:10A12000216F21C11AF1FD51F7ECD9F084ECD9F07F
:10A1300001011E05D8A49FEFD0F0A1EFD0F0C0EF31
:10A14000D0F020C11FF10F0E1F171F39F00B0C09A3
:10A15000216F21C11AF1FD51F7ECD9F084ECD9F04F
:10A1600020C11FF10F0E01011F171F39F00B080945
:10A17000216F21C11AF1FD51F7ECD9F084ECD9F02F
:10A18000120002012989D6EFD0F0B5ECDBF0070E02
:10A1900000EFD1F00201252981ECDBF0030E00EF86
:10A1A000D1F0B8ECDBF00A0E00EFD1F012C20BF1E7
:10A1B00013C20CF102D8E7EFD0F00500FA6E00519F
:10A1C000FD6E0151FE6E0251FF6EFA501200010148
:10A1D0000D6F0E6B0E51000AD8B4F1EFD0F0D1EF35
:10A1E000D0F00D51010AD8B4D1EFD0F0030AD8B4A1
:10A1F000C5EFD0F0060AD8B4CAEFD0F0D1EFD0F056
:10A2000012003901A3A707EFD1F009EFD1F00CEF4D
:10A21000D1F06F00A0F7F8F0000E0101016F000E01
:10A22000006F800E0025D96E040E0121DA6E000E3B
:10A23000DF6E004B012B015109E17F0E005DD8A0BC
:10A2400024EFD1F026EFD1F011EFD1F03D01F289EA
:10A25000000EF96F000EFA6F000E0401806F000E01
:10A260000201756F000E746F000E0001F86F000E92
:10A27000F46F3901938D93871200A2ECDBF0020E8C
:10A280000201286F50EFD1F06EECDBF078EFD1F0E7
:10A29000C6ECDBF078EFD1F05FECDBF078EFD1F0DB
:10A2A00014C20BF115C20CF120EE03F202D863EFD9
:10A2B000D1F00500FA6EDE50FD6EDE50FE6EDE500F
:10A2C000FF6EFA50120001010D6F0E6B0E51000A65
:10A2D000D8B46DEFD1F04CEFD1F00D51020AD8B4E3
:10A2E00044EFD1F0010AD8B448EFD1F04CEFD1F0EF
:10A2F0001200000E0101056F000E046F02510311E0
:10A30000D8B485EFD1F087EFD1F0AFEFD1F0010EE7
:10A31000066F8FEFD1F0D89002370337062B03AFCB
:10A3200094EFD1F096EFD1F08BEFD1F0D8900437C5
:10A3300005370251005D03510159D8A0A2EFD1F0B9
:10A34000A4EFD1F0A9EFD1F00251005F0351015BFE
:10A350000481D89003330233062F96EFD1F004C165
:10A3600000F105C101F11200000E0101036F000EA2
:10A37000026FE0EFD1F03901A3A9C1EFD1F0C3EF33
:10A38000D1F0BBEFD1F0010102510025D96E03518C
:10A390000121DA6EDF503D01EA6F0101024B032B10
:10A3A00003BFDCEFD1F0035109E1810E025DD8A0BB
:10A3B000DCEFD1F0DEEFD1F0E0EFD1F0EEEFD1F055
:10A3C00002510025D96E03510121DA6EDF50D8A465
:10A3D000ECEFD1F0EEEFD1F0BBEFD1F012000101C4
:10A3E0001F6F01011F51F00B0D095E6E5EC01AF167
:10A3F000FD51F7ECD9F084ECD9F001011F51F00BBD
:10A4000009095E6E5EC01AF1FD51F7ECD9F084ECDB
:10A41000D9F01FC11EF10F0E01011E171E39F00BDE
:10A420000D095E6E5EC01AF1FD51F7ECD9F084ECB7
:10A43000D9F01FC11EF10F0E01011E171E39F00BBE
:10A4400009095E6E5EC01AF1FD51F7ECD9F084EC9B
:10A45000D9F0120060000BF4F6FF60000FF4F7FF74
:10A46000000EF86E08006F00D4FFE8F052EFD2F053
:10A4700060000BF4F6FF60000FF4F7FF000EF86EBB
:10A4800008006F00D4FFE8F0600003F4D9FF60001B
:10A4900007F4DAFF6000A3F3DFFF0101004B012B9B
:10A4A000024B032B0001E851D8A459EFD2F05BEF27
:10A4B000D2F038EFD2F0600003F4D9FF600007F467
:10A4C000DAFF000EDF6E1200C3C1C7F1C4C1C8F1CC
:10A4D000000E0001D56F000ED46F86EFD2F0C1C11F
:10A4E00099F1C2C19AF1C70E01019B6F010E9C6FD9
:10A4F000C5C19DF1C6C19EF109EC92F001019951CF
:10A500000001D42701019A510001D52360001FF7F3
:10A51000F6FF600023F7F7FF000EF86E0800F55015
:10A520000009D8A496EFD2F098EFD2F06FEFD2F0F6
:10A53000D4C0C1F1D5C0C2F112000BECD6F00201BB
:10A540002951030B0009D8B4A8EFD2F0AAEFD2F03A
:10A55000B7EFD2F014ECDBF00009D8B4B2EFD2F0D0
:10A56000B4EFD2F0B7EFD2F0100E0201276F020164
:10A570002751030DB50EF324F66EF50EF420F76E99
:10A58000F86A000EF82202D8D3EFD2F00500FA6E76
:10A590000900F550FD6E0900F550FE6E0900F550FA
:10A5A000FF6EFA5012000201276F1200FC0E02012A
:10A5B0002917020E286F2995E5EFD2F0C4ECDBF0E5
:10A5C0000DEFD3F00F0E0DEFD3F016C20BF117C243
:10A5D0000CF120EE06F202D8F8EFD2F00500FA6E88
:10A5E000DE50FD6EDE50FE6EDE50FF6EFA50120041
:10A5F00001010D6F0E6B0E51000AD8B402EFD3F0BB
:10A60000E2EFD2F00D51020AD8B4DEEFD2F0010A27
:10A61000D8B4DEEFD2F0E2EFD2F01200000E046EFA
:10A62000000E036E37EFD3F03901A3A91AEFD3F070
:10A630001CEFD3F014EFD3F003500124D96E045073
:10A640000220DA6EDF503D01EA6F034A042A04BE9D
:10A6500033EFD3F0045009E1810E035CD8A033EF4F
:10A66000D3F035EFD3F037EFD3F045EFD3F003500D
:10A670000124D96E04500220DA6EDF50D8A443EFD3
:10A68000D3F045EFD3F014EFD3F0120006C10AF176
:10A6900007C10BF104C10CF105C10DF101010A5113
:10A6A000086F0B51096F0A4B0B2B600023F4F6FF68
:10A6B000600027F4F7FF000EF86E600033F4D9FF56
:10A6C000600037F4DAFF0C4B0D2B1F0EF76403D03C
:10A6D0000800F55007D06F00DBFFE9FF6F00DFFFD8
:10A6E000EAFFEF50DF6EDF50D8A479EFD3F07BEFB5
:10A6F000D3F04EEFD3F01200B8C044F0B9C045F02B
:10A70000000E0001D56F000ED46F9AEFD3F0B6C0E3
:10A7100092F0B7C093F0440E946F000E956FBAC0DC
:10A7200096F0BBC097F021EC8CF000019251D42739
:10A730009351D523600013F1F6FF600017F1F7FF86
:10A74000000EF86E0800F5500009D8A4AAEFD3F067
:10A75000ACEFD3F087EFD3F0D4C0B6F0D5C0B7F0EC
:10A76000120003C007F004C008F001C009F002C0E5
:10A770000AF00750056E0850066E074A082A600066
:10A7800017F0F6FF60001BF0F7FF000EF86E600098
:10A7900027F0D9FF60002BF0DAFF094A0A2A1F0EC2
:10A7A000F76403D00800F55007D06F00DBFFE9FF26
:10A7B0006F00DFFFEAFFEF50DF6EDF50D8A4E3EF5A
:10A7C000D3F0E5EFD3F0B9EFD3F01200000E0101A2
:10A7D000246F000E236FFBEFD3F023512025D96E99
:10A7E00024512121DA6EDF50EFECD1F084ECD9F066
:10A7F0000101234B242B23512025D96E24512121E3
:10A80000DA6EDF50D8B407EFD4F009EFD4F018EFC8
:10A81000D4F0FE51235D2451800A226FFF51800A3B
:10A820002259D8A016EFD4F018EFD4F0EDEFD3F002
:10A8300012000101196F0101195198ECCEF00009C5
:10A84000D8B425EFD4F027EFD4F01BEFD4F015C126
:10A8500000F116C101F117C102F118C103F171EC49
:10A86000DAF0000E0101066F000E076F000E086F90
:10A87000000E096F000E0A6FE2ECDAF092ECDBF0EA
:10A880006CECD9F0E806D8B448EFD4F04AEFD4F035
:10A8900040EFD4F01200D2BE50EFD4F053EFD4F01A
:10A8A000010E54EFD4F0000E0101006FD29ED28A47
:10A8B000D29ED29CD28A550ED46EAA0ED46ED4905B
:10A8C000000ED76E000ED66E080ED56E550ED46EE5
:10A8D000AA0ED46ED4803901838781818491839FAD
:10A8E00084958791809FD28CD28E010100B102D0D5
:10A8F000D29E01D0D28E12000101036F000E000122
:10A90000D76F000ED66F95EFD4F0520E0101016F94
:10A910002B0E006F000EE82EFED7002FFCD7012F64
:10A92000FAD700F00001D64BD72B01010351006F7D
:10A93000016B00510001D65DD751800A0101026F01
:10A940000151800A0259D8A0A8EFD4F0AAEFD4F0A0
:10A9500085EFD4F012000101136F010E0101146F95
:10A96000020129B5B6EFD4F0B8EFD4F0D7EFD4F0A8
:10A970002985000E0101146F0201255181ECDBF0E5
:10A9800001011351D8B4C7EFD4F0C9EFD4F0D0EF20
:10A99000D4F0040E0201276FCAECD9F0D5EFD4F041
:10A9A000030E0201276FFEECDAF0C4ECDAF00101CD
:10A9B0001451120000C102F101C103F1E3EFD4F020
:10A9C0000101004B012B600003F4F6FF600007F467
:10A9D000F7FF000EF86E1F0EF76403D00800F55065
:10A9E00007D06F00DBFFE9FF6F00DFFFEAFFEF50EA
:10A9F0000009D8A4FEEFD4F000EFD5F0E0EFD4F0DA
:10AA000001010251005D006F03510159016F1200F5
:10AA10003901A3A10EEFD5F010EFD5F012EFD5F06C
:10AA200035EFD5F0A2AF17EFD5F019EFD5F01BEF4A
:10AA3000D5F035EFD5F03D0179A521EFD5F023EF25
:10AA4000D5F025EFD5F035EFD5F079AF2AEFD5F079
:10AA50002CEFD5F02EEFD5F035EFD5F076A933EF0A
:10AA6000D5F035EFD5F008EFD5F012004FEFD5F067
:10AA70003901A3A93EEFD5F040EFD5F038EFD5F07E
:10AA8000600003F4F6FF600007F4F7FF000EF86EB5
:10AA900008006F00D7FFEAFD0101004B012B6000A9
:10AAA00003F4F6FF600007F4F7FF000EF86E0800ED
:10AAB000F5500009D8A45FEFD5F061EFD5F038EF7D
:10AAC000D5F0120001C003F002C004F06AEFD5F027
:10AAD000014A022A600007F0F6FF60000BF0F7FF62
:10AAE000000EF86E1F0EF76403D00800F55007D073
:10AAF0006F00DBFFE9FF6F00DFFFEAFFEF500009A7
:10AB0000D8A485EFD5F087EFD5F068EFD5F00350E6
:10AB1000015C016E04500258026E1200010E010128
:10AB2000066F200E00190111D8B499EFD5F09BEFF4
:10AB3000D5F0B4EFD5F0F70E026FFF0E036F00C132
:10AB400004F101C105F10251042703510523055108
:10AB500009E1050E045DD8A0B0EFD5F0B2EFD5F055
:10AB6000B4EFD5F0000E066F06C100F1016B1200C4
:10AB7000010120EE02F00B51D9260C51DA226F00B0
:10AB800078FF00F16F0074FF01F160002FF4D9FF2E
:10AB9000600033F4DAFF6F0078FF02F16F0074FF9A
:10ABA00003F171ECDAF0000E0101066F000E076F81
:10ABB000000E086F000E096F000E0A6FF0ECDAF05D
:10ABC000020E1200CD0E0101E46F010EE56FC9C146
:10ABD000D9F1CAC1DAF1000EDD6F000EDC6F000E94
:10ABE000E36F000EE26FD90EC16F010EC26FCBC1D1
:10ABF000C3F1CCC1C4F1E40EC56F010EC66F64ECA5
:10AC0000D2F00101DC51C925D96EDD51CA21DA6EBD
:10AC1000000EDF6E120040ECDBF00009D8B413EF39
:10AC2000D6F015EFD6F019EFD6F0C1ECDBF033EF2C
:10AC3000D6F02AECDBF00009D8B421EFD6F023EFF0
:10AC4000D6F027EFD6F0BBECDBF033EFD6F035ECE7
:10AC5000DBF00009D8B42FEFD6F031EFD6F033EFA8
:10AC6000D6F0BEECDBF01200C00E466E000E476E52
:10AC7000BCC048F0BDC049F0000E4C6E000E4B6EDB
:10AC8000000E526E000E516E480E0001B66F000E9F
:10AC9000B76FBEC0B8F0BFC0B9F0460EBA6F000EB5
:10ACA000BB6F7CECD3F04B500001BC25D96E4C50EF
:10ACB000BD21DA6E000EDF6E1200000EAC6E010ECA
:10ACC000AE6EAC8CAC9AAC88AC50F00B0109AC6E9B
:10ACD000F90EAB6E000EAA6E000EAF6E000E0001F4
:10ACE000E16F000EE06FEF95000E0201636F000E42
:10ACF000626F000E5D6F000E5C6F39019485A49544
:10AD0000AC9E1200000E3D01EC6F000EED6F000EC8
:10AD1000EE6F000EEF6F000EF06F000EF16FB00ED1
:10AD2000F26F800EF36F000EF46F220EF56F000EBF
:10AD3000F66F000EF76F000EF86F000EF96F000E41
:10AD4000FA6FF28BF289390193971200BF0E01015D
:10AD5000086FFF0E096F06C10AF107C10BF1085118
:10AD60000A2709510B230B5107E11A0E0A5DD8B0CF
:10AD7000BCEFD6F0BEEFD6F0C5EFD6F0200E061130
:10AD8000066F0751076FC9EFD6F006C106F107C17C
:10AD900007F11200000E0101321B000E331B000EE2
:10ADA000341B800E351B2EC100F12FC101F130C1C3
:10ADB00002F131C103F132C104F133C105F134C1F3
:10ADC00006F135C107F1F0ECA0F000C12EF101C190
:10ADD0002FF102C130F103C131F11200000E010167
:10ADE0000F6F000E0E6F01EFD7F00DC100F1016B78
:10ADF0000BC102F10CC103F176ECC8F001010E4B5E
:10AE00000F2B0E510925D96E0F510A21DA6EDF5032
:10AE10000D6F0D51D8A40FEFD7F011EFD7F0F5EF6C
:10AE2000D6F012009F0E0101086FFF0E096F06C1D8
:10AE30000AF107C10BF108510A2709510B230B51E5
:10AE400007E11A0E0A5DD8B028EFD7F02AEFD7F045
:10AE500030EFD7F05F0E0615066F076B34EFD7F0B3
:10AE600006C106F107C107F11200BF0E056EFF0E05
:10AE7000066E03C007F004C008F005500726065010
:10AE80000822085007E11A0E075CD8B04AEFD7F045
:10AE90004CEFD7F053EFD7F0200E0310036E0450A1
:10AEA000046E57EFD7F003C003F004C004F01200A3
:10AEB000000E1E1A000E1F1A000E201A800E211AF4
:10AEC0001AC001F01BC002F01CC003F01DC004F04A
:10AED0001EC005F01FC006F020C007F021C008F01A
:10AEE00051ECA3F001C01AF002C01BF003C01CF02B
:10AEF00004C01DF012009F0E056EFF0E066E03C00B
:10AF000007F004C008F00550072606500822085034
:10AF100007E11A0E075CD8B090EFD7F092EFD7F0A8
:10AF200098EFD7F05F0E0314036E046A9CEFD7F01E
:10AF300003C003F004C004F01200000E106E000EF7
:10AF40000F6EAEEFD7F00EC001F0026A0CC003F036
:10AF50000DC004F04FECC9F00F4A102A0F500A241C
:10AF6000D96E10500B20DA6EDF500E6E0E50D8A442
:10AF7000BCEFD7F0BEEFD7F0A3EFD7F01200200E52
:10AF800001180210D8B4C7EFD7F0C9EFD7F0E0EF3F
:10AF9000D7F0F70E036EFF0E046E01C005F002C07D
:10AFA00006F00350052604500622065009E1050E5E
:10AFB000055CD8A0DEEFD7F0E0EFD7F0E0EFD7F0F8
:10AFC0001200010113BFEFEFD7F0135106E1120594
:10AFD000D8B0EDEFD7F0EFEFD7F0FDEFD7F012C11B
:10AFE00014F113C115F1141F151F144B152B14C1A7
:10AFF00012F115C113F101EFD8F012C112F113C112
:10B0000013F1120014BE0FEFD8F0145006E1130430
:10B01000D8B00DEFD8F00FEFD8F01DEFD8F013C077
:10B0200015F014C016F0151E161E154A162A15C066
:10B0300013F016C014F021EFD8F013C013F014C0B1
:10B0400014F012009F0E0101026FFF0E036F200E1D
:10B050000011046F000E0111056F02510427035106
:10B06000052305510AE11A0E045DD8A03AEFD8F085
:10B070003DEFD8F0010E3EEFD8F0000E006F016BEF
:10B0800012009F0E0101026FFF0E036F00C104F159
:10B0900001C105F1025104270351052305510AE1BD
:10B0A0001A0E045DD8A057EFD8F05AEFD8F0010E71
:10B0B0005BEFD8F0000E006F016B1200BF0E0101B4
:10B0C000026FFF0E036F00C104F101C105F10251CF
:10B0D00004270351052305510AE11A0E045DD8A087
:10B0E00074EFD8F077EFD8F0010E78EFD8F0000EBB
:10B0F000006F016B120001010051011102110311D7
:10B10000D8B485EFD8F087EFD8F08FEFD8F0000EE5
:10B11000001B000E011B000E021B800E031B00C152
:10B1200000F101C101F102C102F103C103F11200FA
:10B13000D00E0101026FFF0E036F00C104F101C1C7
:10B1400005F1025104270351052305510AE10A0EB6
:10B15000045DD8A0AEEFD8F0B1EFD8F0010EB2EF99
:10B16000D8F0000E006F016B1200015002100310A6
:10B170000410D8B4BEEFD8F0C0EFD8F0C8EFD8F0C4
:10B18000000E011A000E021A000E031A800E041A95
:10B1900001C001F002C002F003C003F004C004F0DB
:10B1A00012003E01F88100F000F03E01F8B1DBEF43
:10B1B000D8F0DDEFD8F0D5EFD8F06F00C0FB5BF032
:10B1C0005C6A5B500101006F3E01EF510001DE6FD0
:10B1D00000C1DFF012000BC100F10CC101F1000E43
:10B1E0000101036F010E026F71ECDAF0000E010134
:10B1F000066F000E076F000E086F000E096F000E3D
:10B200000A6FF0ECDAF0040E12000BC100F10CC171
:10B2100001F1000E0101036F020E026F71ECDAF012
:10B22000000E0101066F000E076F000E086F000E82
:10B23000096F000E0A6FF0ECDAF0020E12000BC17B
:10B2400000F10CC101F1000E0101036F010E026F4C
:10B2500071ECDAF0000E0101066F000E076F000EB0
:10B26000086F000E096F000E0A6FF0ECDAF0020EA4
:10B2700012000BC100F10CC101F1000E0101036FBE
:10B28000020E026F71ECDAF0000E0101066F000E83
:10B29000076F000E086F000E096F000E0A6FF0ECCA
:10B2A000DAF0040E12003D017995600003F46EFDA2
:10B2B000000E6C6F738B79A560EFD9F062EFD9F057
:10B2C0005BEFD9F074AB67EFD9F06AEFD9F0010EFC
:10B2D0006BEFD9F0000E1200010E0101006F0201A8
:10B2E00029B575EFD9F077EFD9F081EFD9F029972B
:10B2F0002269A2ECDBF0D3ECDAF087ECDBF028C2B9
:10B3000000F1010100511200000E0101016F000E59
:10B31000006F00F00101004B012B01BF99EFD9F044
:10B32000015109E1A00E005DD8A099EFD9F09BEF83
:10B33000D9F089EFD9F012003901A3A9A2EFD9F011
:10B34000A4EFD9F09CEFD9F00D0E3D01EA6F390161
:10B35000A3A9ADEFD9F0AFEFD9F0A7EFD9F00A0E5E
:10B360003D01EA6F12003D0173BFB9EFD9F0BBEFA9
:10B37000D9F0C9EFD9F0000E796F000E7A6F000E88
:10B38000766F6C69510E3A016A6F510E6B6F3D0119
:10B39000738F120002012951FC0B0209296F250548
:10B3A0002611D8A4D6EFD9F0D8EFD9F0DAEFD9F03A
:10B3B00043ECCFF0D880020122357BECDBF0040EA9
:10B3C00012000101005102036F00CCFF04F16F0075
:10B3D000D0FF05F100510303F3500527015102038B
:10B3E000F350052704C100F105C101F1120001016C
:10B3F0001B6F1AC11CF1000E01011D6F1C0E156F91
:10B40000010E166F000E186F010E176F1B5119EC0D
:10B41000D4F0A00EE82EFED71200015003026F00F8
:10B42000CCFF05F06F00D0FF06F001500402F3508E
:10B43000062602500302F350062605C001F006C09E
:10B4400002F012000EC100F10FC101F1DAECD4F0EC
:10B45000010100510E25046F01510F21056F10C12C
:10B4600006F111C107F146ECD3F01200A9ECDBF0B4
:10B47000A6ECDBF00009D8B440EFDAF042EFDAF0E6
:10B4800048EFDAF0000E81ECDBF0000E7BECDBF035
:10B49000000E1200BBF61DF8B2F7D8F747F88BF78D
:10B4A000F9F673F807F65BF72BF76DF858F863F8C1
:0BB4B000F3F708F8286E756C6C29009B
:10B4BC00000E3E01C16FC18FC183C181F851F30BE6
:10B4CC000409F86FF889010EF16FC38A3A01508BA9
:10B4DC003E01F88F1200020129A977EFDAF079EF1B
:10B4EC00DAF082EFDAF000C123F201C124F202C1DA
:10B4FC0025F203C126F2299912000101006F88EF91
:10B50C00DAF000F03901A3A98EEFDAF090EFDAF05F
:10B51C0087EFDAF0600003F4EAFD1200030E3D0140
:10B52C007B6F040E736F800E746F000E756F000EC0
:10B53C006C6F7599200E6E6F7995739F1200016E6A
:10B54C00A9EFDAF000F03901A3A9AFEFDAF0B1EF0F
:10B55C00DAF0A8EFDAF0600007F0EAFD1200010162
:10B56C002A6F27C122F101012A517EECCCF028C1AF
:10B57C0020F129C121F1E6ECD3F01200CAEFDAF088
:10B58C0008ECD5F09DECD2F0020129B5D0EFDAF041
:10B59C00D2EFDAF0C6EFDAF01200390193939395FB
:10B5AC00929F93913D017A917A957A9F7A9D7A93A5
:10B5BC00769376957691120006C100F107C101F1E0
:10B5CC0008C102F109C103F10AC104F1020E35EC04
:10B5DC00D0F0120006C100F107C101F108C102F15F
:10B5EC0009C103F10AC104F1000E35ECD0F01200D0
:10B5FC0002012951FC0B0209296F225122257BECF7
:10B60C00DBF0030E12003D0178BB0FEFDBF012EF05
:10B61C00DBF0010E13EFDBF0000E12003D0174BBEA
:10B62C001AEFDBF01DEFDBF0010E1EEFDBF0000E6E
:10B63C0012003D0178B125EFDBF028EFDBF0010EB5
:10B64C0029EFDBF0000E12003D0179B530EFDBF095
:10B65C0033EFDBF0010E34EFDBF0000E12003D0196
:10B66C0076B93BEFDBF03EEFDBF0010E3FEFDBF0AA
:10B67C00000E12003D0179BF46EFDBF049EFDBF025
:0AB68C00010E4AEFDBF0000E120081
:10B698000001E04BE12B000E02015D6F010E5C6FB3
:10B6A8003901A49511008DECDBF002012995020EF9
:10B6B800286F0F0E12008DECDBF002012995000EA9
:10B6C800286F0F0E1200ACECDBF0A9ECDBF075EC88
:10B6D800DBF012000201255181ECDBF0CAECD9F055
:10B6E800120002012995000E286F0F0E12000101A9
:10B6F800006F600003F46BFD12000101006F600031
:10B7080003F46CFD12003D01739F000E796F78857C
:10B7180012003D01739F7885738F1200000EABEC09
:10B72800D4F01200ACECDBF0090E1200AFECDBF049
:10B73800040E1200AFECDBF0030E1200000E3D0108
:10B74800796F12003D016C5112003D01739B12008C
:10B758003D01748D12003D01749D12003D016A5136
:10B7680012003D01738D12003D01739D12003D01D1
:10B77800799512003D01769912003D01799F1200DA
:10B78800010E1200020E1200050E1200010E120028
:0FB79800140012001200120012001200120064BE
:020000040020DA
:10000000FF0FFF0FFF0FFF0FFF0FFF0FFF0FFF0F80
:020000040030CA
:0A0000008CD5FFF78DCFFFDFFFFF67
:00000001FF
